:020000040800F2
:1000000000500020ED500008F14F0008F94F0008A3
:1000100001500008095000081150000800000000BD
:10002000000000000000000000000000195000085F
:100030002550000800000000315000083D50000825
:100040003551000835510008355100083551000878
:100050003551000835510008355100083551000868
:100060003551000835510008355100084D50000841
:100070003551000835510008355100083551000848
:100080003551000835510008355100083551000838
:1000900061500008355100083551000835510008FD
:1000A0003551000835510008355100083551000818
:1000B0003551000835510008355100083551000808
:1000C00035510008355100083551000835510008F8
:1000D00035510008355100083551000835510008E8
:1000E0003551000835510008355100080000000066
:1000F0000000000000000000000000000000000000
:0C01000000000000000000005FF808F1A3
:10010C0010B5054C237833B9044B13B10448AFF345
:10011C0000800123237010BDE001002000000000CE
:10012C000CEE000808B5034B1BB103490348AFF3B1
:10013C00008008BD00000000E40100200CEE000867
:10014C00034613F8012B002AFBD1181A013870470B
:10015C0080B400AF124B1B78DBB2002B1BD0104BC2
:10016C0000221A700F4B1B889AB20F4B1A800D4B42
:10017C005B889AB20D4B1A800A4B9B889AB20C4B37
:10018C001A80084BDB889AB20A4B1A80054B1B89E4
:10019C009AB2094B1A8000BFBD4680BC704700BFA5
:1001AC0029020020080200202A0200202C02002034
:1001BC002E020020300200203202002080B483B0D6
:1001CC0000AF0023FB7110E0FB79214A32F81330A9
:1001DC0099B2FB791F4A52F82320FB790A441D4936
:1001EC0041F82320FB790133FB71FB79042BEBD90C
:1001FC00194B1B780133DAB2174B1A70164B1B785C
:10020C00042B20D90023BB7114E0BB79114A52F89E
:10021C002330124AA2FB03239A08BB7991B2104AED
:10022C0022F81310BB790B4A002142F82310BB793A
:10023C000133BB71BB79042BE7D9074B00221A7031
:10024C00084B01221A7000BF0C37BD4680BC7047AA
:10025C00FC0100201402002028020020CDCCCCCCC4
:10026C00080200202902002080B582B000AF0346AE
:10027C003960FB71FB799BB201339BB2396818462C
:10028C0001F0E4F9034618460837BD4680BD80B539
:10029C0082B000AF03460A46FB711346BB80FB7964
:1002AC009BB201339BB2BA881146184601F0EAF9A9
:1002BC00034618460837BD4680BD90B482B000AFE7
:1002CC000446084611461A462346FB710346BB7189
:1002DC000B467B7113463B71FB792F2B06D9FB79AF
:1002EC00392B03D8FB79303BFB710BE0FB79602B8E
:1002FC0006D9FB79662B03D8FB79573BFB7101E0E0
:10030C00002370E0BB792F2B06D9BB79392B03D88E
:10031C00BB79303BBB710BE0BB79602B06D9BB7949
:10032C00662B03D8BB79573BBB7101E000235AE025
:10033C007B792F2B06D97B79392B03D87B79303BF2
:10034C007B710BE07B79602B06D97B79662B03D80C
:10035C007B79573B7B7101E0002344E03B792F2BE9
:10036C0006D93B79392B03D83B79303B3B710BE0F9
:10037C003B79602B06D93B79662B03D83B79573BED
:10038C003B7101E000232EE0FB799AB23B691A80A5
:10039C003B691B881B019AB23B691A803B691A881E
:1003AC00BB799BB213449AB23B691A803B691B8898
:1003BC001B019AB23B691A803B691A887B799BB204
:1003CC0013449AB23B691A803B691B881B019AB291
:1003DC003B691A803B691A883B799BB213449AB2E9
:1003EC003B691A80012318460837BD4690BC7047FC
:1003FC002DE9F043C1B006AF0DF09EFB0346002B78
:10040C0000F0C8860DF0ACFBC7F8E000D7F8E03080
:10041C00002BC0F2BE86BD4B1B781A46D7F8E030D5
:10042C00D9B2BB4B995400BFB84B1B781A46B84B8A
:10043C001344012118460DF055FC0346012BF3D053
:10044C00D7F8E0300D2B04D0D7F8E0300A2B40F071
:10045C009986AE4B1B78002B00F09086AC4B1B782A
:10046C00493B242B00F2788601A252F823F000BFFE
:10047C00C706000865110008651100086511000821
:10048C006511000865110008651100086511000868
:10049C006511000865110008651100086511000858
:1004AC006511000865110008651100086511000848
:1004BC006511000865110008651100086511000838
:1004CC006511000865110008651100086511000828
:1004DC0065110008EB06000865110008651100089D
:1004EC00F509000865110008651100086511000880
:1004FC001105000865110008651100086511000858
:10050C00AD07000807F11003824918460DF0C8FF2B
:10051C0000BF07F11003052118460DF0E3FB03465D
:10052C00012BF6D000217C4803F0B4FF034698461B
:10053C000421794803F0AEFF03469946082176481A
:10054C0003F0A8FF03461C460C21734803F0A2FFDE
:10055C0003461D460021714803F09CFF03461E46CE
:10056C0004216E4803F096FF03467B6008216B481C
:10057C0003F090FF03463B600C21684803F08AFFB0
:10058C00034607F1100005933A6804927B680393C5
:10059C000296019500944B46424661490DF080FF4E
:1005AC0000BF07F110031846FFF7CAFD03469AB2C5
:1005BC0007F11003114618460DF094FB0346012B6E
:1005CC00EFD0554B1B685B6B7B60534B1B68996B77
:1005DC003960514B1B68DB6B4F4A1268126C4F49E8
:1005EC000968496B4D480068806B4C4C2468E46B7F
:1005FC004A4D2D682D6C07F1100605950494039057
:10060C000291019200933B687A68464930460DF09E
:10061C0047FF00BF07F110031846FFF791FD034693
:10062C009AB207F11003114618460DF05BFB034616
:10063C00012BEFD03C4B1B781D463C4B1B881E46B8
:10064C003B4B1B881A463B4B1B8819463A4B1B8865
:10065C001C463A4B1B8807F110000393029401913E
:10066C00009233462A4636490DF01AFF00BF07F1B7
:10067C0010031846FFF764FD03469AB207F1100306
:10068C00114618460DF02EFB0346012BEFD02D4BD7
:10069C001B781A462C4B1B7807F110002B490DF0D8
:1006AC00FFFE00BF07F110031F2118460DF01AFBC7
:1006BC000346012BF6D000F061BD07F1100324496D
:1006CC0018460DF0EDFE00BF07F110030921184686
:1006DC000DF008FB0346012BF6D000F04FBD0B4B81
:1006EC001B78022B4AD10A4B5B78302B04D1194B67
:1006FC0000221A7000F042BD054B5B78312B2BD1D8
:10070C00144B01221A7000F039BD00BF34020020D6
:10071C003802002024EE000818030020600300209B
:10072C002CEE000844EE0008F00300202A02002002
:10073C002C0200202E020020300200203202002069
:10074C0078EE00085604002054040020B0EE000897
:10075C00D0EE00085804002007F110039B491846FE
:10076C000DF09EFE00BF07F11003052118460DF099
:10077C00B9FA0346012BF6D000F000BD07F11003C7
:10078C00924918460DF08CFE00BF07F110030521AD
:10079C0018460DF0A7FA0346012BF6D000F0EEBC7C
:1007AC008B4B1B78082B40F0FE808A4B5B78302BF0
:1007BC0040F2E880874B5B78342B00F2E380854B6A
:1007CC005B78303BDAB2834B5A70824B5B7887F89C
:1007DC00DF30804B9B78662B03D1002387F8E73002
:1007EC0019E07C4B9B78622B03D1012387F8E7300F
:1007FC0011E007F11003784918460DF051FE00BFC7
:10080C0007F11003102118460DF06CFA0346012B6A
:10081C00F6D000F0B3BC6F4BDB782F2B40F2A180ED
:10082C006C4BDB78392B00F29C806A4B1B792F2B9D
:10083C0040F29780674B1B79392B00F29280654B05
:10084C005B792F2B40F28D80624B5B79392B00F258
:10085C008880604B9B792F2B40F283805D4B9B797A
:10086C00392B7ED85B4BDB792F2B7AD9594BDB7923
:10087C00392B76D8574BDB78303BDAB2554BDA70E4
:10088C00544BDB7887F8DE30524B1B79303BDAB2B5
:10089C00504B1A714F4B1B7987F8DD304D4B5B7900
:1008AC00303BDAB24B4B5A714A4B5B7987F8DC30F0
:1008BC00484B9B79303BDAB2464B9A71454B9B794E
:1008CC0087F8DB30434BDB79303BDAB2414BDA71E2
:1008DC00404BDB7987F8DA3097F8DE309BB2FB813E
:1008EC00FB891A46920013445B009BB2FB8197F87C
:1008FC00DD309AB2FB8913449BB2FB81FB891A460B
:10090C00920013445B009BB2FB8197F8DC309AB2E7
:10091C00FB8913449BB2FB81FB891A46920013445A
:10092C005B009BB2FB8197F8DB309AB2FB891344D6
:10093C009BB2FB81FB891A46920013445B009BB26D
:10094C00FB8197F8DA309AB2FB8913449BB2FB8196
:10095C00FA8997F8E71097F8DF30184603F010FE85
:10096C0032E007F110031D4918460DF099FD00BF48
:10097C0007F11003132118460DF0B4F90346012BAF
:10098C00F6D021E007F11003154918460DF088FD4B
:10099C0000BF07F11003132118460DF0A3F903460D
:1009AC00012BF6D0EAE307F110030E4918460DF0BF
:1009BC0077FD00BF07F110030A2118460DF092F9DC
:1009CC000346012BF6D0D9E3D8E300BFDCEE0008D8
:1009DC003402002038020020E4EE0008F8EE000893
:1009EC0018EF00082CEF0008BB4B1B78012B40F2D2
:1009FC009B83BA4B5B78722B40F08680B64B1B788E
:100A0C00042B69D1B54B9A78B44BD97807F10C0308
:100A1C0000930B4630213020FFF74FFC0346002B90
:100A2C0042D0BB89DBB207F10E0211461846FFF724
:100A3C001BFC0346A7F8D830B7F8D830002B19D1D7
:100A4C00BB891A46FB8907F11000A5490DF028FD5A
:100A5C0000BF07F110031846FFF772FB03469AB26A
:100A6C0007F11003114618460DF03CF90346012B13
:100A7C00EFD082E3B7F8D82007F110039949184654
:100A8C000DF00EFD00BF07F110031846FFF758FBE1
:100A9C0003469AB207F11003114618460DF022F9DD
:100AAC000346012BEFD068E307F110038E4918467B
:100ABC000DF0F6FC00BF07F110031846FFF740FBE2
:100ACC0003469AB207F11003114618460DF00AF9C5
:100ADC000346012BEFD050E307F11003834918466E
:100AEC000DF0DEFC00BF07F110031846FFF728FBE2
:100AFC0003469AB207F11003114618460DF0F2F8AE
:100B0C000346012BEFD038E3744B5B78772B69D11C
:100B1C00714B1B78082B4DD1704B9A786F4BD97851
:100B2C0007F10C0300930B4630213020FFF7C5FB77
:100B3C000346002B37D0694B1879684B5979674BB2
:100B4C009A79664BDC7907F10E0300932346FFF785
:100B5C00B4FB0346002B1FD0BB89DBB2FA891146CC
:100B6C001846FFF794FB0346A7F8D830B7F8D830EF
:100B7C00002B08D1BB891A46FB8907F110005C4990
:100B8C000DF08EFC1CE0B7F8D82007F11003594982
:100B9C0018460DF085FC13E007F110035649184672
:100BAC000DF07EFC0CE007F11003544918460DF0D3
:100BBC0077FC05E007F11003514918460DF070FC65
:100BCC0000BF07F110031846FFF7BAFA03469AB2B2
:100BDC0007F11003114618460DF084F80346012B5B
:100BEC00EFD0CAE23D4B5B78642B40F0A9803A4BC6
:100BFC001B78022B40F08C80002387F8E63046E00F
:100C0C0007F10E0297F8E63011461846FFF72CFB59
:100C1C000346A7F8D830B7F8D830002B19D197F87D
:100C2C00E620FB8907F1100036490DF039FC00BFB6
:100C3C0007F110031846FFF783FA03469AB207F13F
:100C4C001003114618460DF04DF80346012BEFD05A
:100C5C0018E0B7F8D82007F110032B4918460DF00F
:100C6C001FFC00BF07F110031846FFF769FA034693
:100C7C009AB207F11003114618460DF033F80346EB
:100C8C00012BEFD097F8E630013387F8E63097F870
:100C9C00E6301F2BB4D997F8E63003F00303DBB230
:100CAC00002B40F06A8207F11003184918460DF02A
:100CBC00F7FB00BF07F110031846FFF741FA034694
:100CCC009AB207F11003114618460DF00BF80346C3
:100CDC00012BEFD051E200BF34020020380200207B
:100CEC0038EF00084CEF000860EF000874EF0008C4
:100CFC007CEF000890EF0008A4EF0008BCEF0008A0
:100D0C00D0EF0008DCEF0008ECEF0008F8EF00086B
:100D1C0007F110031D4918460DF0C2FB00BF07F187
:100D2C0010031846FFF70CFA03469AB207F11003AA
:100D3C00114618460CF0D6FF0346012BEFD01CE2EF
:100D4C00134B5B78782B29D1124B1B78022B04D1D7
:100D5C0000F0D2FC00F01EFD0FE207F110030E496B
:100D6C0018460DF09DFB00BF07F110031846FFF766
:100D7C00E7F903469AB207F11003114618460CF036
:100D8C00B1FF0346012BEFD0F7E100BFFCEF0008E9
:100D9C00380200203402002004F00008B44B5B78C9
:100DAC00762B40F04C81B34B1B78022B40F02F81FB
:100DBC00B14B1B889C46B14B1B889E46B04B1B8885
:100DCC001A46B04B1B881946AF4B1B881C46AF4BC1
:100DDC001B881D46AE4B1B881E46AE4B1B8807F16D
:100DEC0010000593049603950294019100927346AA
:100DFC006246A9490DF054FB00BF07F110031846D9
:100E0C00FFF79EF903469AB207F1100311461846F4
:100E1C000CF068FF0346012BEFD0A04B1B88194642
:100E2C009F4B1B881C469F4B1B881A469E4B1B884E
:100E3C0007F110000193009223460A469B490DF0DE
:100E4C002FFB00BF07F110031846FFF779F9034693
:100E5C009AB207F11003114618460CF043FF0346F3
:100E6C00012BEFD0924B1B881A46924B1B8807F133
:100E7C00100091490DF014FB00BF07F11003184648
:100E8C00FFF75EF903469AB207F1100311461846B4
:100E9C000CF028FF0346012BEFD0884B1B8819461A
:100EAC00874B1B881C46874B1B881A46864B1B8816
:100EBC0007F110000193009223460A4683490DF076
:100ECC00EFFA00BF07F110031846FFF739F9034694
:100EDC009AB207F11003114618460CF003FF0346B3
:100EEC00012BEFD07A4B1B8819467A4B1B881C467A
:100EFC00794B1B881A46794B1B8807F1100001931C
:100F0C00009223460A4676490DF0CAFA00BF07F153
:100F1C0010031846FFF714F903469AB207F11003B1
:100F2C00114618460CF0DEFE0346012BEFD06D4B3C
:100F3C001B8819466C4B1B881C466C4B1B881A462D
:100F4C006B4B1B8807F110000193009223460A4655
:100F5C0068490DF0A5FA00BF07F110031846FFF71A
:100F6C00EFF803469AB207F11003114618460CF03D
:100F7C00B9FE0346012BEFD05F4B1B8819465F4B24
:100F8C001B881C465E4B1B881A465E4B1B8807F160
:100F9C0010000193009223460A465B490DF080FA3B
:100FAC0000BF07F110031846FFF7CAF803469AB2C0
:100FBC0007F11003114618460CF094FE0346012B62
:100FCC00EFD0524B1B881946514B1B881C46514B7A
:100FDC001B881A46504B1B8807F110000193009296
:100FEC0023460A464D490DF05BFA00BF07F110038A
:100FFC001846FFF7A5F803469AB207F110031146FD
:10100C0018460CF06FFE0346012BEFD0B5E007F14C
:10101C001003434918460DF043FA00BF07F11003C3
:10102C001846FFF78DF803469AB207F110031146E4
:10103C0018460CF057FE0346012BEFD09DE007F14C
:10104C001003384918460DF02BFA00BF07F11003B6
:10105C001846FFF775F803469AB207F110031146CC
:10106C0018460CF03FFE0346012BEFD085E000BF85
:10107C00380200203402002000040020020400206A
:10108C000404002006040020080400200A040020A8
:10109C000C0400200E0400200CF0000810040020AA
:1010AC0012040020140400201604002068F000082C
:1010BC00180400201E040020ACF0000820040020BE
:1010CC00220400202404002026040020C4F0000880
:1010DC00280400202A040020380400203A040020B0
:1010EC00F8F000082C0400202E0400203C04002002
:1010FC003E0400202CF100083004002032040020B3
:10110C00400400204204002060F100083404002058
:10111C0036040020440400204604002094F100080A
:10112C00C8F10008D0F1000807F110031B4918465C
:10113C000DF0B6F900BF07F110031846FFF700F8E1
:10114C0003469AB207F11003114618460CF0CAFD7B
:10115C000346012BEFD010E007F11003104918469D
:10116C000DF09EF900BF07F11003022118460CF098
:10117C00B9FD0346012BF6D000E000BF094B00225D
:10118C001A7007E0074B1B780133DAB2054B1A7063
:10119C0000E000BFEC37BD46BDE8F083E0F100088D
:1011AC00F4F100083402002080B59AB000AF2F4B48
:1011BC001A782F4B1B789A4217D02D4B1A782B4B41
:1011CC001A702B4B1B781A463B1D2A4918460DF0FA
:1011DC0067F93B1D1846FEF7B3FF03469AB2391D5B
:1011EC004FF0FF33244808F06BFB244B1A88244B38
:1011FC001B889A4217D0224B1A88204B1A80204BFE
:10120C001B881A463B1D1F4918460DF049F93B1D1A
:10121C001846FEF795FF03469AB2391D4FF0FF337F
:10122C00154808F04DFB184B1A78184B1B789A424E
:10123C0017D0164B1A78144B1A70144B1B781A468D
:10124C003B1D134918460DF02BF93B1D1846FEF7B4
:10125C0077FF03469AB2391D4FF0FF33064808F06A
:10126C002FFB00BF6837BD4680BD00BF9C0200202D
:10127C00F0030020F8F10008A80300209E020020D3
:10128C005404002008F20008A0020020560400209C
:10129C0018F2000880B582B000AF03463960FB71CC
:1012AC00FB799BB201339BB23968184600F0CEF93A
:1012BC00034618460837BD4680BD80B582B000AFE6
:1012CC0003460A46FB711346BB80FB799BB2013384
:1012DC009BB2BA881146184600F0D4F9034618465A
:1012EC000837BD4680BD80B483B000AF78607B68A2
:1012FC001B889BB218460C37BD4680BC7047B0B5F6
:10130C0084B000AF78600B467B8004F0AFFE7B8826
:10131C0000221C46154622462B467968012004F013
:10132C0035FE0346FB7304F0C7FEFB7B18461037F3
:10133C00BD46B0BD80B588B000AF78600023BB60FF
:10134C0004F094FE0023FB607B687B610123BB618E
:10135C0007F1080207F10C031146184604F06EFF62
:10136C000346FB7704F0A8FEFB7F18462037BD46EA
:10137C0080BD80B487B000AF78607B6802337B613E
:10138C007B6803F580633B610CE07B691B88FB8108
:10139C00FB894FF6FF72934201D17B6908E07B69B0
:1013AC0004337B613B69033B7A699A42EDD300239A
:1013BC0018461C37BD4680BC704780B489B000AF5E
:1013CC00F8600B467A607B81FB680233FB61FB683B
:1013DC0003F580637B610223FB7600233B837B68F0
:1013EC00002B18D1012324E0FB691B887B827B8AAC
:1013FC004FF6FF72934214D0FB6902331B883B8279
:10140C007A8A7B899A4203D13B8A3B830023FB7601
:10141C00FB690433FB617B69043BFA699A42E3D9AB
:10142C0000E000BFFB7E002B02D17B683A8B1A8058
:10143C00FB7E18462437BD4680BC704780B500AF94
:10144C000F48FFF777FF0346002B01D0012315E06F
:10145C000C48FFF76FFF0346002B01D001230DE072
:10146C004AF6AA210648FFF74AFF0346002B01D093
:10147C00012303E0044B024A1A600023184680BD86
:10148C0000F8000800FC00080000002080B483B0C5
:10149C0000AF78607B68054A934201D1044B00E0B1
:1014AC00024B18460C37BD4680BC704700F800084C
:1014BC0000FC000880B588B000AF03460A46FB80EC
:1014CC001346BB803C4B1B687B617869FFF7DEFFE2
:1014DC0038613869FFF72EFF0346002B01D001233A
:1014EC0065E045F255513869FFF709FF0346002BBB
:1014FC0001D001235BE03B690233FB6100237B835A
:10150C003CE07B8B2D4A32F81330FB81FA89FB8847
:10151C009A4202D1BB887B810BE007F10A02FB895E
:10152C0019467869FFF749FF03467B737B7B002BD9
:10153C0020D1FB891946F869FFF7E1FE0346002B21
:10154C0001D0012333E0FB6902337A891146184636
:10155C00FFF7D5FE0346002B01D0012327E0FB69E2
:10156C000433FB613B6903F58063FA699A4202D349
:10157C0003231CE000BF7B8B01337B837B8B3F2BD6
:10158C00BFD97869FFF7D6FE0346002B01D00123A3
:10159C000DE04AF6AA213869FFF7B1FE0346002B8D
:1015AC0001D0012303E0044A3B6913600023184671
:1015BC002037BD4680BD00BF0000002030F500087C
:1015CC0080B582B000AF1E48FFF78DFE0346FB804E
:1015DC001C48FFF788FE0346BB80FB884FF6FF7262
:1015EC00934208D1BB884FF6FF72934203D1FFF7A9
:1015FC0025FF034620E0FB884AF6AA22934209D134
:10160C00BB884FF6FF72934204D10F4B0C4A1A6001
:10161C00002311E0BB884AF6AA22934209D1FB8829
:10162C004FF6FF72934204D1074B064A1A6000230F
:10163C0002E0FFF703FF034618460837BD4680BD9E
:10164C0000F8000800FC00080000002080B584B001
:10165C0000AF03463960FB803B68002B01D10123AE
:10166C000AE0074B1B68F9883A681846FFF7A5FE95
:10167C000346FB73FB7B9BB218461037BD4680BDFF
:10168C000000002080B584B000AF03460A46FB8002
:10169C001346BB80174B1B681846FFF76AFEF860B1
:1016AC00FB68002B17D0FB881946F868FFF727FE5C
:1016BC000346002B01D0012317E0FB680233BA88E4
:1016CC0011461846FFF71BFE0346002B01D00123E1
:1016DC000BE0002309E0BA88FB8811461846FFF797
:1016EC00E9FE0346FB72FB7A9BB218461037BD46E7
:1016FC0080BD00BF0000002080B59AB000AF002371
:10170C0087F8673035E097F867301E4A32F81320B7
:10171C0097F8673011461846FFF7CFFD0346A7F838
:10172C006430B7F86430002B0BD197F8672097F82A
:10173C006730144931F81330384613490CF0B0FEB9
:10174C0006E0B7F864203B46104918460CF0A8FE9A
:10175C003B461846FEF7F4FC03469AB239464FF066
:10176C00FF330B4808F0ACF897F86730013387F873
:10177C00673097F867303F2BC5D900BF00BF68377B
:10178C00BD4680BDB0F4000824F2000830F2000819
:10179C00A8030020F0B5B9B006AFBC490020FFF794
:1017AC0079FDBB490120FFF775FDBA490220FFF70F
:1017BC0071FDB9490320FFF76DFDB8490420FFF70F
:1017CC0069FDB7490520FFF765FDB6490620FFF70F
:1017DC0061FDB5490720FFF75DFDB4490820FFF70F
:1017EC0059FDB3490920FFF755FDB2490A20FFF70F
:1017FC0051FDB1490B20FFF74DFDB0490C20FFF70F
:10180C0049FDAF490D20FFF745FDAE490E20FFF70E
:10181C0041FDAD490F20FFF73DFDAC491820FFF706
:10182C0039FDAB491920FFF735FDAA491A20FFF7FE
:10183C0031FDA9491B20FFF72DFDA8491C20FFF7FE
:10184C0029FDA7491D20FFF725FDA6491E20FFF7FE
:10185C0021FDA5491F20FFF71DFDA4492020FFF7FE
:10186C0019FDA3492120FFF715FDA2492220FFF7FE
:10187C0011FDA1492320FFF70DFDA0492420FFF7FE
:10188C0009FD9F492520FFF705FD9E492620FFF7FE
:10189C0001FD9D492720FFF7FDFC9C492820FFF7FF
:1018AC00F9FC9B492920FFF7F5FC9A492A20FFF700
:1018BC00F1FC99492B20FFF7EDFC98492C20FFF700
:1018CC00E9FC97492D20FFF7E5FC96492E20FFF700
:1018DC00E1FC95492F20FFF7DDFC94493F20FFF7F1
:1018EC00D9FC3B46924918460CF0DAFD3B461846AB
:1018FC00FEF726FC03469AB239464FF0FF338D486B
:10190C0007F0DEFF614B1B889C46614B1B889E4693
:10191C00604B1B881A46604B1B8819465F4B1B8813
:10192C001C465F4B1B881D465E4B1B881E465E4B40
:10193C001B883846059304960395029401910092F6
:10194C00734662467C490CF0ABFD3B461846FEF7ED
:10195C00F7FB03469AB239464FF0FF33754807F050
:10196C00AFFF564B1B881946554B1B881C46554BD5
:10197C001B881A46544B1B88384601930092234609
:10198C000A466E490CF08CFD3B461846FEF7D8FB18
:10199C0003469AB239464FF0FF33664807F090FF82
:1019AC00514B1B881A464F4B1B88384664490CF028
:1019BC0077FD3B461846FEF7C3FB03469AB2394601
:1019CC004FF0FF335B4807F07BFF424B1B881946F7
:1019DC00414B1B881C46414B1B881A46404B1B88AD
:1019EC0038460193009223460A4656490CF058FD9E
:1019FC003B461846FEF7A4FB03469AB239464FF015
:101A0C00FF334C4807F05CFF384B1B881946384BAA
:101A1C001B881C463D4B1B881A463D4B1B88384681
:101A2C000193009223460A4647490CF039FD3B4688
:101A3C001846FEF785FB03469AB239464FF0FF3342
:101A4C003C4807F03DFF2B4B1B8819462A4B1B8843
:101A5C001C46304B1B881A462F4B1B88384601936B
:101A6C00009223460A4639490CF01AFD3B461846AB
:101A7C00FEF766FB03469AB239464FF0FF332D480A
:101A8C0007F01EFF1D4B1B88194661E00004002067
:101A9C000204002004040020060400200804002096
:101AAC000A0400200C0400200E0400204C0400202A
:101ABC004E0400205004002052040020100400208A
:101ACC001204002014040020160400201C04002022
:101ADC001A040020200400202204002024040020EA
:101AEC00260400201E0400201804002028040020D6
:101AFC002A0400202C0400202E0400203004002096
:101B0C003204002034040020360400203804002065
:101B1C003A0400203C0400203E0400204004002035
:101B2C004204002044040020460400204804002005
:101B3C0044F20008A80300204CF20008A8F20008A8
:101B4C00ECF2000804F3000838F300086CF300080A
:101B5C001F4B1B881C461F4B1B881A461E4B1B8891
:101B6C0038460193009223460A461C490CF098FC17
:101B7C003B461846FEF7E4FA03469AB239464FF054
:101B8C00FF33174807F09CFE164B1B881946164B63
:101B9C001B881C46154B1B881A46154B1B88384650
:101BAC000193009223460A4612490CF079FC3B46FD
:101BBC001846FEF7C5FA03469AB239464FF0FF3382
:101BCC00074807F07DFE00BFCC37BD46F0BD00BF17
:101BDC00320400204004002042040020A0F300083E
:101BEC00A803002034040020360400204404002004
:101BFC0046040020D4F3000880B582B000AF7C4BC3
:101C0C001B780133DAB27A4B1A70794B1B78092B9B
:101C1C0040F2E781764B00221A70764B1B78DBB2D0
:101C2C00002B06D0734B1B78DBB2013BDAB2714B45
:101C3C001A70714B1B78DBB2002B06D06E4B1B78E5
:101C4C00DBB2013BDAB26C4B1A706C4B1B78DBB21B
:101C5C00002B06D0694B1B78DBB2013BDAB2674B29
:101C6C001A70674B1B780133DAB2654B1A70644BF0
:101C7C001B7803F00303DAB2614B1A704FF4804106
:101C8C00604804F007FD0346002B0CD15C4B1B781D
:101C9C001A465D4B9B5C5A4A127843F00103D9B249
:101CAC00594B99540BE0564B1B781A46564B9B5C80
:101CBC00534A127823F00103D9B2534B99544FF481
:101CCC000041504804F0E6FC0346002B0CD14C4B71
:101CDC001B781A464C4B9B5C494A127843F0020322
:101CEC00D9B2494B99540BE0454B1B781A46464BDD
:101CFC009B5C434A127823F00203D9B2424B9954AD
:101D0C004FF48051414804F0C5FC0346002B0CD124
:101D1C003B4B1B781A463C4B9B5C394A127843F080
:101D2C000403D9B2384B99540BE0354B1B781A4647
:101D3C00354B9B5C324A127823F00403D9B2324BF8
:101D4C0099544FF40051314804F0A4FC0346002B85
:101D5C000CD12B4B1B781A462B4B9B5C284A1278C8
:101D6C0043F00803D9B2284B99540BE0244B1B7851
:101D7C001A46254B9B5C224A127823F00803D9B2F1
:101D8C00214B99544FF48041204804F083FC0346C6
:101D9C00002B0CD11A4B1B781A461B4B9B5C184A18
:101DAC00127843F01003D9B2174B99540BE0144B33
:101DBC001B781A46144B9B5C114A127823F01003C3
:101DCC00D9B2114B99544FF40041104804F062FC05
:101DDC000346002B1CD10A4B1B781A460A4B9B5C02
:101DEC00074A127843F02003D9B2074B99541BE0F1
:101DFC005A040020040000200500002006000020EA
:101E0C005B040020001001405C040020000C014029
:101E1C00764B1B781A46764B9B5C744A127823F0EF
:101E2C002003D9B2724B9954714B1A78704B5B7872
:101E3C001340DAB26E4B9B781340DAB26C4BDB7802
:101E4C001340DAB26B4B1B781343DAB2694B1A703E
:101E5C00674B1A78664B5B781343DAB2644B9B780A
:101E6C001343DAB2624BDB781343DAB2614B1B7863
:101E7C001340DAB25F4B1A70FEF7A0F95E4B1B7879
:101E8C000133DAB25C4B1A705B4B1B78092B40F2B6
:101E9C00A880594B00221A700023FB7113E0FB79C8
:101EAC00564A32F813309BB2002B09D0FB79534AB7
:101EBC0032F8132092B2013A91B2504A22F8131020
:101ECC00FB790133FB71FB79032BE8D94C4B1B8855
:101EDC009BB24FF6FF72934206D0494B1B889BB2C4
:101EEC0001339AB2464B1A80464B1B889BB2002B8F
:101EFC0006D0444B1B889BB2013B9AB2414B1A80D3
:101F0C00414B1B78DBB2012B27D1404B1B78002BAC
:101F1C0011D03F4B1B78042B06D900224FF40051F3
:101F2C003C4804F0CEFB4FE001224FF400513948FD
:101F3C0004F0C7FB48E0364B1B78042B06D9002273
:101F4C004FF48071344804F0BCFB3DE001224FF4A7
:101F5C008071314804F0B5FB36E02B4B1B78DBB2BB
:101F6C00022B2BD1294B1B78002B13D0284B1B7821
:101F7C0003F00103002B06D000224FF4005125483A
:101F8C0004F09FFB20E001224FF40051214804F0A3
:101F9C0098FB19E01E4B1B7803F00103002B06D0B5
:101FAC0000224FF480711C4804F08BFB0CE00122E2
:101FBC004FF48071184804F084FB05E000224FF4C4
:101FCC008071154804F07DFB114B1B780133DAB29C
:101FDC000F4B1A700E4B1B78092B02D90C4B00229D
:101FEC001A7000BF0837BD4680BD00BF5B040020DF
:101FFC005C040020F003002060040020F4030020A7
:10200C00FC030020FE03002057040020580400208D
:10201C0061040020001001400008014080B500AFB1
:10202C00AC4B1B7803F00103002B13D0AA4B1B788D
:10203C00DBB2002B07D1A94B1B8843F001039AB2EA
:10204C00A64B1A8036E001224FF40051A44804F04C
:10205C0038FB2FE0A14B1B8803F00103002B14D09D
:10206C009E4B1B8823F001039AB29C4B1A809B4B0E
:10207C001B8843F480539AB2984B1A8000224FF479
:10208C000051974804F01DFB11E0934B1B78DBB219
:10209C00BE2B0CD8914B1B8843F002039AB28F4B8A
:1020AC001A8000224FF400518D4804F00AFB8A4B31
:1020BC00C8221A70874B1B7803F00203002B0CD03C
:1020CC00884B1B78DBB2002B24D1844B1B8843F04C
:1020DC0004039AB2814B1A801CE0804B1B8803F0DE
:1020EC000403002B07D07D4B1B8823F004039AB20A
:1020FC007A4B1A800BE07B4B1B78DBB2BE2B06D8DD
:10210C00764B1B8843F008039AB2744B1A80754BBC
:10211C00C8221A70714B1A8841F20F0313409AB2FD
:10212C006E4B1A806D4B1B88002B40F0E080694B86
:10213C001B7803F03C03302B00F2BB8001A252F859
:10214C0023F000BF15220008BF220008BF220008A0
:10215C00BF22000871220008BF220008BF2200081D
:10216C00BF22000823220008BF220008BF2200085B
:10217C00BF220008A5220008BF220008BF220008C9
:10218C00BF2200083D220008BF220008BF22000821
:10219C00BF220008BF220008BF220008BF2200088F
:1021AC00BF220008BF220008BF220008BF2200087F
:1021BC00BF220008BF220008BF220008BF2200086F
:1021CC00BF22000857220008BF220008BF220008C7
:1021DC00BF220008BF220008BF220008BF2200084F
:1021EC00BF220008BF220008BF220008BF2200083F
:1021FC00BF220008BF220008BF220008BF2200082F
:10220C00BF2200088B220008374B64221A70334B14
:10221C0000221A806BE0344B1B78DBB2002B4FD1C1
:10222C002E4B1B8843F010039AB22C4B1A8047E0BC
:10223C002D4B1B78DBB2002B44D1284B1B8843F071
:10224C0020039AB2254B1A803CE0274B1B78DBB25B
:10225C00002B39D1214B1B8843F480739AB21F4B4E
:10226C001A8031E0204B1B78DBB2002B2ED11B4B9C
:10227C001B8843F400739AB2184B1A8026E01A4B51
:10228C001B78DBB2002B23D1144B1B8843F48063E7
:10229C009AB2124B1A801BE0134B1B78DBB2002B4B
:1022AC0024D10E4B1B8843F400639AB20B4B1A805B
:1022BC001CE00D4B64221A70084B00221A8016E0A9
:1022CC0000BF14E000BF12E000BF10E000BF0EE042
:1022DC0000BF0CE0F0030020040000205404002098
:1022EC0000100140050000200600002000BF00BFC8
:1022FC0080BD00BF80B584B002AF9D4B1B78192BFD
:10230C0000F2948601A252F823F000BF812300084A
:10231C00532400089D240008E724000831250008F8
:10232C00B9250008032600084D260008972600084A
:10233C00E12600082B27000875270008BF27000896
:10234C002D28000875280008BD280008052900085C
:10235C004D290008B5290008452A0008E12A000883
:10236C00FB2E00084B2B00080B2E00089B2E0008A0
:10237C00632F00087F4B1B8823F480539AB27D4B4C
:10238C001A807C4B1B8803F00103002B14D07A4B72
:10239C0002221A70794B00221A80754B12221A7085
:1023AC00774B00221A7001F0DFF901F0AFFA01F05F
:1023BC007FFB01F051FC0BE06E4B1B8803F002031A
:1023CC00002B05D06E4B00221A70694B13221A7029
:1023DC006B4B00221A706B4B1A886B4B1B889A4202
:1023EC0023D9674B1B7883F00103DBB2002B1CD085
:1023FC0001224FF40041654804F063F9644B1B88DB
:10240C009BB2002B1DD15D4B00221A805A4B01222E
:10241C001A70574B18221A7001F0F2FC01F0C2FD31
:10242C0001F092FE01F064FF0BE000224FF400413A
:10243C00564804F046F9574B1A88554B1A8000F051
:10244C00F5BD00F0F3BD544B1B88DAB2534B1B881F
:10245C00D9B2534B1B88DBB20A20019000930B4678
:10246C000021012002F07EFB444B1B889AB24D4B9D
:10247C001B889A4202D33E4B11221A704A4B1B788E
:10248C00002B40F0A2853A4B02221A7000F09DBD41
:10249C00414B1B88DAB2414B1B88D9B2404B1B888D
:1024AC00DBB20A20019000930B460021012002F0C0
:1024BC0059FB324B1B889AB23A4B1B889A4202D377
:1024CC002B4B11221A70384B1B78002B00F07F8598
:1024DC00274B11221A7000F07ABD2F4B1B88DAB2F1
:1024EC002E4B1B88D9B22E4B1B88DBB20A200190D5
:1024FC0000930B460121012002F034FB1F4B1B887B
:10250C009AB2284B1B889A4202D3194B11221A708B
:10251C00254B1B78002B40F05C85154B04221A7060
:10252C0000F057BD1C4B1B88DAB21C4B1B88D9B270
:10253C001B4B1B88DBB20A20019000930B46012138
:10254C00012002F00FFB0D4B1B889AB2154B1B8818
:10255C009A4202D3064B11221A70134B1B78002B94
:10256C0000F03985024B11221A7000F034BD00BF07
:10257C00560400205404002057040020FC030020C3
:10258C0059040020320200201C04002000080140E5
:10259C00FE0300201A0400204C040020200400201C
:1025AC001E04002010040020F0030020934B5B88D5
:1025BC00DAB2934B1B88D9B2924B1B88DBB20A2040
:1025CC00019000930B460021022002F0CBFA8E4BB7
:1025DC001B889AB28D4B1B889A4202D38C4B1122CA
:1025EC001A708C4B1B78002B40F0F784884B06221A
:1025FC001A7000F0F2BC814B5B88DAB2804B1B88FE
:10260C00D9B2804B1B88DBB20A20019000930B4699
:10261C000021022002F0A6FA7B4B1B889AB27B4B5E
:10262C001B889A4202D37A4B11221A70794B1B7871
:10263C00002B00F0D484764B11221A7000F0CFBC22
:10264C006E4B5B88DAB26E4B1B88D9B26D4B1B8814
:10265C00DBB20A20019000930B460121022002F00C
:10266C0081FA694B1B889AB2684B1B889A4202D339
:10267C00674B11221A70674B1B78002B40F0B1840A
:10268C00634B08221A7000F0ACBC5C4B5B88DAB26E
:10269C005B4B1B88D9B25B4B1B88DBB20A200190C9
:1026AC0000930B460121022002F05CFA564B1B886A
:1026BC009AB2564B1B889A4202D3554B11221A7070
:1026CC00544B1B78002B00F08E84514B11221A7046
:1026DC0000F089BC494B9B88DAB24F4B1B88D9B2AE
:1026EC00484B1B88DBB20A20019000930B4600215B
:1026FC00032002F037FA444B1B889AB2474B1B88D5
:10270C009A4202D3424B11221A70424B1B78002B77
:10271C0040F06B843E4B0A221A7000F066BC374BBB
:10272C009B88DAB23C4B1B88D9B2364B1B88DBB288
:10273C000A20019000930B460021032002F012FAAC
:10274C00314B1B889AB2354B1B889A4202D3304BC3
:10275C0011221A702F4B1B78002B00F048842C4B45
:10276C0011221A7000F043BC244B9B88DAB22A4B1E
:10277C001B88D9B2234B1B88DBB20A200190009333
:10278C000B460121032002F0EDF91F4B1B889AB276
:10279C00224B1B889A4202D31D4B11221A701D4BDF
:1027AC001B78002B40F02584194B0C221A7000F07A
:1027BC0020BC124B9B88DAB2174B1B88D9B2114B39
:1027CC001B88DBB20A20019000930B4601210320E9
:1027DC0002F0C8F90C4B1B889AB2104B1B889A421A
:1027EC0002D30B4B11221A700A4B1B78002B00F0F2
:1027FC000284074B11221A70FDE300BF4C04002029
:10280C00220400201E040020FC03002012040020DF
:10281C0056040020F003002024040020140400209F
:10282C00A34BDB88DAB2A34B1B88D9B2A24B1B8813
:10283C00DBB20A20019000930B460021042002F029
:10284C0091F99E4B1B889AB29D4B1B889A4202D3DE
:10285C009C4B11221A709C4B1B78002B40F0CD83A3
:10286C00984B0E221A70C8E3914BDB88DAB2914B6D
:10287C001B88D9B2904B1B88DBB20A2001900093C5
:10288C000B460021042002F06DF98C4B1B889AB288
:10289C008B4B1B889A4202D38A4B11221A708A4B9B
:1028AC001B78002B00F0AB83864B11221A70A6E329
:1028BC007F4BDB88DAB27F4B1B88D9B27E4B1B88EF
:1028CC00DBB20A20019000930B460121042002F098
:1028DC0049F97A4B1B889AB2794B1B889A4202D3DE
:1028EC00784B11221A70784B1B78002B40F089839F
:1028FC00744B10221A7084E36D4BDB88DAB26D4B8B
:10290C001B88D9B26C4B1B88DBB20A200190009358
:10291C000B460121042002F025F9684B1B889AB262
:10292C00674B1B889A4202D3664B11221A70664B76
:10293C001B78002B00F06783624B11221A7062E344
:10294C0000220021012001F08DFF00220021022035
:10295C0001F088FF00220021032001F083FF0022F8
:10296C000021042001F07EFF00220121012001F052
:10297C0079FF00220121022001F074FF00220121C5
:10298C00032001F06FFF00220121042001F06AFFF7
:10299C004D4B1B78002B40F038834C4B00221A70A7
:1029AC00484B16221A7030E3444B1B889BB21D2BEC
:1029BC0024D9464B01221A7000F0D6FE0346FB7157
:1029CC0000F0A4FF0346BB7101F072F803467B7163
:1029DC0001F042F903463B71FB79042B0ED1BB7914
:1029EC00042B0BD17B79042B08D13B79042B05D11B
:1029FC00364B00221A70334B16221A70344B1B883C
:102A0C0003F00203002B02D02E4B13221A70304B12
:102A1C001B8803F00103002B00F0F9822C4B1B8860
:102A2C0003F48053002B00F0F282264B14221A7010
:102A3C00224B00221A80EAE200220021012001F040
:102A4C0011FF00220021022001F00CFF00220021C6
:102A5C00032001F007FF00220021042001F002FFF7
:102A6C0000220121012001F0FDFE002201210220A3
:102A7C0001F0F8FE00220121032001F0F3FE0022F8
:102A8C000121042001F0EEFE0F4B1B78002B40F0CF
:102A9C00C0820E4B00221A700A4B00221A700C4B8B
:102AAC001B8823F002039AB2094B1A80B1E200BFD3
:102ABC004C040020260400201E040020FC030020EF
:102ACC001604002056040020F003002057040020B8
:102ADC005404002000220021012001F0C3FE00223A
:102AEC000021022001F0BEFE00220021032001F093
:102AFC00B9FE00220021042001F0B4FE00220121C5
:102B0C00012001F0AFFE00220121022001F0AAFEFB
:102B1C0000220121032001F0A5FE00220121042046
:102B2C0001F0A0FE984B00221A70984B1B889BB2A8
:102B3C00132B40F27082964B16221A706BE2954B57
:102B4C001B8823F480539AB2924B1A808F4B00222D
:102B5C001A80904B1B8803F00103002B0DD08A4B7D
:102B6C0001221A708A4B17221A7001F049F901F0F0
:102B7C0019FA01F0E9FA01F0BBFB874B1A88874B75
:102B8C001B889A4219D901224FF40041844803F062
:102B9C0098FD844B1B889BB2002B18D17A4B0122D9
:102BAC001A707B4B18221A7001F02AF901F0FAF90D
:102BBC0001F0CAFA01F09CFB09E000224FF400413D
:102BCC00774803F07EFD784B1A88764B1A80714B50
:102BDC001B8803F00203002B03D06D4B19221A70D3
:102BEC001BE26C4B1B8803F01003002B17D0664BB9
:102BFC0001221A706D4B1B88DAB26D4B1B88D9B24F
:102C0C006C4B1B88DBB20020019000930B4600211B
:102C1C00012001F0A7FF5E4B01221A70FDE15D4B14
:102C2C001B8803F02003002B17D0574B01221A707E
:102C3C005E4B1B88DAB25E4B1B88D9B25D4B1B888E
:102C4C00DBB20020019000930B460121012001F022
:102C5C0089FF4F4B03221A70DFE14E4B1B8803F0A8
:102C6C004003002B17D0484B01221A704F4B5B8846
:102C7C00DAB2514B1B88D9B24E4B1B88DBB2002009
:102C8C00019000930B460021022001F06BFF404B9A
:102C9C0005221A70C1E13F4B1B8803F08003002B07
:102CAC0017D0394B01221A70404B5B88DAB2424B79
:102CBC001B88D9B23F4B1B88DBB2002001900093DC
:102CCC000B460121022001F04DFF314B07221A70F7
:102CDC00A3E1304B1B8803F48073002B17D02A4BD5
:102CEC0001221A70314B9B88DAB2344B1B88D9B253
:102CFC00304B1B88DBB20020019000930B46002167
:102D0C00032001F02FFF224B09221A7085E1214B81
:102D1C001B8803F40073002B17D01B4B01221A7075
:102D2C00224B9B88DAB2254B1B88D9B2214B1B88CE
:102D3C00DBB20020019000930B460121032001F02F
:102D4C0011FF134B0B221A7067E1124B1B8803F413
:102D5C008063002B34D00C4B01221A70134BDB8890
:102D6C00DAB2164B1B88D9B2124B1B88DBB200208F
:102D7C00019000930B460021042001F0F3FE044B5C
:102D8C000D221A7049E100BF57040020FC030020FB
:102D9C005604002054040020320200201C040020A1
:102DAC0000080140FE0300201A0400204C040020FF
:102DBC00200400201E0400202204002024040020F3
:102DCC009C4B1B8803F40063002B00F026819A4B6C
:102DDC0001221A70994BDB88DAB2994B1B88D9B255
:102DEC00984B1B88DBB20020019000930B4601210D
:102DFC00042001F0B7FE944B0F221A700DE1934B97
:102E0C001B889BB2092B24D900F0FAFF0346FB71F7
:102E1C0001F0C8F80346BB7101F096F903467B71CB
:102E2C0001F066FA03463B71FB79042B11D1BB7997
:102E3C00042B0ED17B79042B0BD13B79042B08D1BD
:102E4C007D4B00221A70804B00221A70804B01229D
:102E5C001A70784B1B8803F00203002B02D07A4BBC
:102E6C0019221A70734B1B8803F00103002B00F01E
:102E7C00D680704B1B8803F48053002B00F0CF805E
:102E8C00714B15221A70714B00221A80C7E06F4BE0
:102E9C001B889BB2092B40F2C48000F0B1FF0346A3
:102EAC00FB7101F07FF80346BB7101F04DF903464D
:102EBC007B7101F01DFA03463B71FB79042B40F04A
:102ECC00B080BB79042B40F0AC807B79042B40F0B4
:102EDC00A8803B79042B40F0A480574B00221A7039
:102EEC00594B00221A705A4B01221A7099E0002299
:102EFC000021012001F0B6FC00220021022001F08B
:102F0C00B1FC00220021032001F0ACFC00220021C6
:102F1C00042001F0A7FC00220121012001F0A2FCF9
:102F2C0000220121022001F09DFC0022012103203E
:102F3C0001F098FC00220121042001F093FC3E4B8F
:102F4C0000221A70414B1B889BB2132B6BD93E4B42
:102F5C0000221A7067E000220021012001F082FC9F
:102F6C0000220021022001F07DFC00220021032020
:102F7C0001F078FC00220021042001F073FC0022F7
:102F8C000121012001F06EFC00220121022001F040
:102F9C0069FC00220121032001F064FC00220121C4
:102FAC00042001F05FFC2B4B1B78002B3DD1224BF6
:102FBC0000221A70244B16221A701E4B1B8823F009
:102FCC0002039AB21B4B1A802FE000BF2EE000BF09
:102FDC002CE000BF2AE000BF28E000BF26E000BFC5
:102FEC0024E000BF22E000BF20E000BF1EE000BFD5
:102FFC001CE000BF1AE000BF18E000BF16E000BFE5
:10300C0014E000BF12E000BF10E000BF0EE000BFF4
:10301C000CE000BF0AE000BF08E000BF06E000BF04
:10302C0004E000BF02E000BF00E000BF00BF0837B3
:10303C00BD4680BD54040020570400204C040020E1
:10304C00240400201E04002056040020FC03002051
:10305C0059040020F003002080B500AF02F066F8A0
:10306C0000F06EF800F0D0FA00F0B0FA0AF0FEFCB6
:10307C0000F03CF900F0DEF900F0C0F800F07CFA4A
:10308C0005222849284802F08BF90021274801F035
:10309C0016FA0421254801F012FA0821234801F000
:1030AC000EFA0C21214801F00AFA0021204801F007
:1030BC0006FA04211E4801F002FA08211C4801F00E
:1030CC00FEF90C211A4801F0FAF9FEF779FA0346D9
:1030DC00002B01D000BFFDE7FEF75CFB154B1B88F6
:1030EC00052B0FD001224FF48071134803F0E9FA3D
:1030FC00FEF702FBFEF74EFB00224FF480710E48E8
:10310C0003F0DFFA0D4B00221A70FDF771F9FDF791
:10311C001FF8FEF783FFFFF7EDF8FEF745F800BF49
:10312C00F3E700BFFC010020A402002018030020DC
:10313C0060030020480400200008014059040020CE
:10314C0080B594B000AF07F128032822002118465F
:10315C000BF0C8F907F1140300221A605A609A6048
:10316C00DA601A613B1D00221A605A609A60DA60BC
:10317C000123BB624FF48033FB6200233B630123CA
:10318C00BB6302237B644FF48033BB644FF4801326
:10319C00FB6407F12803184605F00CF80346002BD6
:1031AC0001D000F0DBFA0F237B610223BB6100230B
:1031BC00FB614FF480633B6200237B6207F11403D5
:1031CC000221184605F078FA0346002B01D000F0D6
:1031DC00C5FA12237B604FF40043FB6000233B6174
:1031EC003B1D184605F0F8FB0346002B01D000F000
:1031FC00B5FA00BF5037BD4680BD000080B584B025
:10320C0000AF3B1D00221A605A609A60354B364A5B
:10321C001A60344B4FF480729A60324B01221A734D
:10322C00304B00221A752F4B4FF46022DA612D4B74
:10323C0000225A602B4B05221A612A4801F0D8FF54
:10324C000346002B01D000F089FA04237B60012394
:10325C00BB600323FB603B1D1946224802F09AF920
:10326C000346002B01D000F079FA05237B60022382
:10327C00BB603B1D19461B4802F08CF90346002B22
:10328C0001D000F06BFA06237B600323BB603B1D6F
:10329C001946144802F07EF90346002B01D000F0C9
:1032AC005DFA07237B600423BB603B1D19460D4868
:1032BC0002F070F90346002B01D000F04FFA0823FE
:1032CC007B600523BB603B1D1946064802F062F982
:1032DC000346002B01D000F041FA00BF1037BD4669
:1032EC0080BD00BFA40200200024014080B58EB038
:1032FC0000AF07F1280300221A605A609A60DA6066
:10330C0007F1200300221A605A603B1D00221A604C
:10331C005A609A60DA601A615A619A61444B4FF0B4
:10332C0080421A60424B00225A60414B00229A6044
:10333C003F4B44F24F62DA603D4B00221A613C4B2A
:10334C0000229A613A4805F0FDFB0346002B01D0A0
:10335C0000F004FA4FF48053BB6207F128031946BE
:10336C00334805F05FFE0346002B01D000F0F6F960
:10337C002F4805F036FC0346002B01D000F0EEF987
:10338C0000233B6200237B6207F120031946284887
:10339C0006F0E8F90346002B01D000F0DFF96023BA
:1033AC007B604FF47A73BB600023FB6004237B616A
:1033BC003B1D002219461E4805F072FD0346002BEA
:1033CC0001D000F0CBF94FF4FA63BB603B1D042233
:1033DC001946174805F064FD0346002B01D000F098
:1033EC00BDF940F6B833BB6000237B613B1D08225E
:1033FC0019460F4805F054FD0346002B01D000F090
:10340C00ADF94FF47A63BB6004237B613B1D0C2246
:10341C001946074805F044FD0346002B01D000F087
:10342C009DF9034801F03EFD00BF3837BD4680BD15
:10343C001803002080B58EB000AF07F128030022DE
:10344C001A605A609A60DA6007F1200300221A6051
:10345C005A603B1D00221A605A609A60DA601A6149
:10346C005A619A61424B434A1A60414B00225A609E
:10347C003F4B00229A603E4B44F24F62DA603C4B69
:10348C0000221A613A4B00229A61394805F05AFB26
:10349C000346002B01D000F061F94FF48053BB625E
:1034AC0007F128031946324805F0BCFD0346002BF2
:1034BC0001D000F053F92E4805F093FB0346002B86
:1034CC0001D000F04BF900233B6200237B6207F133
:1034DC0020031946264806F045F90346002B01D077
:1034EC0000F03CF960237B6041F28833BB60002321
:1034FC00FB6004237B613B1D002219461C4805F030
:10350C00CFFC0346002B01D000F028F941F2707378
:10351C00BB603B1D04221946154805F0C1FC03464F
:10352C00002B01D000F01AF941F65833BB603B1D5B
:10353C00082219460E4805F0B3FC0346002B01D0B7
:10354C0000F00CF94FF4FA53BB603B1D0C221946EA
:10355C00074805F0A5FC0346002B01D000F0FEF84F
:10356C00034801F09FFC00BF3837BD4680BD00BF4B
:10357C00600300200008004080B500AF114B124AD8
:10358C001A60104B4FF4E1325A600E4B00229A60D5
:10359C000C4B0022DA600B4B00221A61094B0C22F7
:1035AC005A61084B00229A61064B0022DA610548E9
:1035BC0006F036F90346002B01D000F0CFF800BF1F
:1035CC0080BD00BFA80300200038014080B582B048
:1035DC0000AF0C4B5B690B4A43F001035361094B81
:1035EC005B6903F001037B607B68002200210B20E8
:1035FC0002F0A1FA0B2002F0BAFA00BF0837BD4660
:10360C0080BD00BF0010024080B588B000AF07F14C
:10361C00100300221A605A609A60DA604B4B9B6967
:10362C004A4A43F010039361484B9B6903F0100323
:10363C00FB60FB68454B9B69444A43F02003936154
:10364C00424B9B6903F02003BB60BB683F4B9B69FB
:10365C003E4A43F0040393613C4B9B6903F0040323
:10366C007B607B68394B9B69384A43F00803936154
:10367C00364B9B6903F008033B603B6800224FF418
:10368C000051334803F01DF8002240F63E4131480A
:10369C0003F017F800224FF401412F4803F011F802
:1036AC004FF400533B6101237B610023BB61022378
:1036BC00FB6107F110031946254802F067FE4FF431
:1036CC0040433B6100237B610023BB6107F1100386
:1036DC0019461F4802F05AFE10233B6103237B61FD
:1036EC0007F1100319461C4802F050FE40F63E4309
:1036FC003B6101237B610023BB610223FB6107F16A
:10370C0010031946134802F041FE4FF470433B611D
:10371C0000237B610023BB6107F1100319460D48A0
:10372C0002F034FE4FF401433B6101237B61002323
:10373C00BB610223FB6107F110031946064802F036
:10374C0025FE00BF2037BD4680BD00BF00100240E3
:10375C0000100140000C01400008014080B400AF93
:10376C0072B600BF00BFFDE780B59CB002AF5D4BE9
:10377C001A785D4B1B789A4217D05B4B1A78594BD1
:10378C001A70594B1B781A463B1D584918460AF0BB
:10379C0087FE3B1D1846FCF7D3FC03469AB2391D35
:1037AC004FF0FF33524806F08BF8524B1B889AB2FD
:1037BC00514B1B889A4202D24B4B00221A704A4B37
:1037CC001B78032B76D801A252F823F0E9370008B6
:1037DC0035380008653800089738000800220021A9
:1037EC00012001F03FF800220121012001F03AF8FC
:1037FC00404B1B889AB2404B1B889A4265D33F4B77
:10380C001B88DAB23E4B1B88D9B23E4B1B88DBB20D
:10381C000020019000930B460021012001F0A2F939
:10382C00314B01221A7050E0344B1B88DAB2344B06
:10383C001B88D9B2334B1B88DBB20A200190009352
:10384C000B460021012001F08DF90346002B3ED1DF
:10385C00254B02221A703AE0264B1B889AB22A4B4F
:10386C001B889A4235D3264B1B88DAB2254B1B8812
:10387C00DBB200210191009300230021012001F013
:10388C0071F9194B03221A7023E01D4B1B88DAB215
:10389C001C4B1B88DBB20A210191009300230021F1
:1038AC00012001F05FF90346002B14D10E4B0422CA
:1038BC001A7010E000220021012000F0D3FF00223A
:1038CC000121012000F0CEFF06E000BF04E000BFA4
:1038DC0002E000BF00E000BF034B1B7818466837BE
:1038EC00BD4680BD070000206204002008F40008DB
:1038FC00A8030020FC030020280400204C04002016
:10390C0000040020180400202A04002080B59CB07C
:10391C0002AF5D4B1A785D4B1B789A4217D05B4B0C
:10392C001A78594B1A70594B1B781A463B1D58493B
:10393C0018460AF0B5FD3B1D1846FCF701FC034682
:10394C009AB2391D4FF0FF33524805F0B9FF524B74
:10395C001B889AB2514B1B889A4202D24B4B0022C5
:10396C001A704A4B1B78032B76D801A252F823F01D
:10397C008D390008D9390008093A00083B3A00088B
:10398C0000220021022000F06DFF00220121022004
:10399C0000F068FF404B1B889AB2404B1B889A4240
:1039AC0065D33F4B5B88DAB23E4B1B88D9B23E4B9A
:1039BC001B88DBB20020019000930B4601210220F2
:1039CC0001F0D0F8314B01221A7050E0344B5B8877
:1039DC00DAB2344B1B88D9B2334B1B88DBB20A20CA
:1039EC00019000930B460121022001F0BBF8034625
:1039FC00002B3ED1254B02221A703AE0264B1B8835
:103A0C009AB22A4B1B889A4235D3264B1B88DAB2C2
:103A1C00254B1B88DBB2002101910093002301216F
:103A2C00022001F09FF8194B03221A7023E01D4B62
:103A3C001B88DAB21C4B1B88DBB20A210191009364
:103A4C0000230121022001F08DF80346002B14D134
:103A5C000E4B04221A7010E000220021022000F00C
:103A6C0001FF00220121022000F0FCFE06E000BF55
:103A7C0004E000BF02E000BF00E000BF034B1B7876
:103A8C0018466837BD4680BD08000020630400203E
:103A9C0014F40008A8030020FC0300202C040020D0
:103AAC004C04002004040020180400202E040020E4
:103ABC0080B59CB002AF5D4B1A785D4B1B789A4277
:103ACC0017D05B4B1A78594B1A70594B1B781A4606
:103ADC003B1D584918460AF0E3FC3B1D1846FCF701
:103AEC002FFB03469AB2391D4FF0FF33524805F0B5
:103AFC00E7FE524B1B889AB2514B1B889A4202D25A
:103B0C004B4B00221A704A4B1B78032B76D801A220
:103B1C0052F823F0313B00087D3B0008AD3B000818
:103B2C00DF3B000800220021032000F09BFE002256
:103B3C000121032000F096FE404B1B889AB2404BAB
:103B4C001B889A4265D33F4B9B88DAB23E4B1B884D
:103B5C00D9B23E4B1B88DBB20020019000930B4680
:103B6C000021032000F0FEFF314B01221A7050E0BF
:103B7C00344B9B88DAB2364B1B88D9B2334B1B883B
:103B8C00DBB20A20019000930B460021032000F0C9
:103B9C00E9FF0346002B3ED1254B02221A703AE076
:103BAC00264B1B889AB22B4B1B889A4235D3284B39
:103BBC001B88DAB2254B1B88DBB2002101910093E4
:103BCC0000230021032000F0CDFF194B03221A70B3
:103BDC0023E01F4B1B88DAB21C4B1B88DBB20A217B
:103BEC000191009300230021032000F0BBFF03464A
:103BFC00002B14D10E4B04221A7010E0002200216D
:103C0C00032000F02FFE00220121032000F02AFEE9
:103C1C0006E000BF04E000BF02E000BF00E000BF10
:103C2C00034B1B7818466837BD4680BD0900002041
:103C3C006404002020F40008A8030020FC030020EA
:103C4C00300400204C040020040400201804002040
:103C5C00080400203204002080B59CB002AF5D4BFC
:103C6C001A785D4B1B789A4217D05B4B1A78594BDC
:103C7C001A70594B1B781A463B1D584918460AF0C6
:103C8C000FFC3B1D1846FCF75BFA03469AB2391D34
:103C9C004FF0FF33524805F013FE524B1B889AB27B
:103CAC00514B1B889A4202D24B4B00221A704A4B42
:103CBC001B78032B76D801A252F823F0D93C0008CC
:103CCC00253D0008553D0008873D000800220021D5
:103CDC00042000F0C7FD00220121042000F0C2FDE9
:103CEC00404B1B889AB2404B1B889A4265D33F4B82
:103CFC00DB88DAB23E4B1B88D9B23E4B1B88DBB259
:103D0C000020019000930B460021042000F02AFFB4
:103D1C00314B01221A7050E0344BDB88DAB2364B4F
:103D2C001B88D9B2334B1B88DBB20A20019000935D
:103D3C000B460021042000F015FF0346002B3ED15A
:103D4C00254B02221A703AE0264B1B889AB22B4B59
:103D5C001B889A4235D3284B1B88DAB2254B1B881B
:103D6C00DBB200210191009300230021042000F01C
:103D7C00F9FE194B03221A7023E01F4B1B88DAB291
:103D8C001C4B1B88DBB20A210191009300230021FC
:103D9C00042000F0E7FE0346002B14D10E4B042246
:103DAC001A7010E000220021042000F05BFD0022BC
:103DBC000121042000F056FD06E000BF04E000BF26
:103DCC0002E000BF00E000BF034B1B7818466837C9
:103DDC00BD4680BD0A000020650400202CF40008BC
:103DEC00A8030020FC030020340400204C04002015
:103DFC0004040020180400200C04002036040020C9
:103E0C0080B59CB002AF5D4B1A785D4B1B789A4223
:103E1C0017D05B4B1A78594B1A70594B1B781A46B2
:103E2C003B1D584918460AF03BFB3B1D1846FCF756
:103E3C0087F903469AB2391D4FF0FF33524805F00B
:103E4C003FFD524B1B889AB2514B1B889A4202D2AF
:103E5C004B4B00221A704A4B1B78032B76D801A2CD
:103E6C0052F823F0813E0008CD3E0008FD3E0008CC
:103E7C002F3F000800220021012000F0F3FC00225B
:103E8C000121012000F0EEFC404B1B889AB2404B04
:103E9C001B889A4265D33F4B1B88DAB23E4B1B887A
:103EAC00D9B23E4B1B88DBB20020019000930B462D
:103EBC000121012000F056FE314B01221A7050E016
:103ECC00344B1B88DAB2344B1B88D9B2334B1B886A
:103EDC00DBB20A20019000930B460121012000F077
:103EEC0041FE0346002B3ED1254B02221A703AE0CC
:103EFC00264B1B889AB22A4B1B889A4235D3264BE9
:103F0C001B88DAB2254B1B88DBB200210191009390
:103F1C0000230121012000F025FE194B03221A7009
:103F2C0023E01D4B1B88DAB21C4B1B88DBB20A2129
:103F3C000191009300230121012000F013FE0346A0
:103F4C00002B14D10E4B04221A7010E00022002119
:103F5C00012000F087FC00220121012000F082FCEE
:103F6C0006E000BF04E000BF02E000BF00E000BFBD
:103F7C00034B1B7818466837BD4680BD0B000020EC
:103F8C006604002038F40008A8030020FC0300207D
:103F9C00380400204C0400200204002018040020E7
:103FAC003A04002080B59CB002AF5D4B1A785D4B93
:103FBC001B789A4217D05B4B1A78594B1A70594B95
:103FCC001B781A463B1D584918460AF069FA3B1DE6
:103FDC001846FCF7B5F803469AB2391D4FF0FF337B
:103FEC00524805F06DFC524B1B889AB2514B1B8802
:103FFC009A4202D24B4B00221A704A4B1B78032B6D
:10400C0076D801A252F823F0254000087140000830
:10401C00A1400008D340000800220021022000F03B
:10402C0021FC00220121022000F01CFC404B1B88CB
:10403C009AB2404B1B889A4265D33F4B5B88DAB2ED
:10404C003E4B1B88D9B23E4B1B88DBB20020019043
:10405C0000930B460021022000F084FD314B01221D
:10406C001A7050E0344B5B88DAB2344B1B88D9B2EF
:10407C00334B1B88DBB20A20019000930B460021C6
:10408C00022000F06FFD0346002B3ED1254B02228F
:10409C001A703AE0264B1B889AB22A4B1B889A421C
:1040AC0035D3264B1B88DAB2254B1B88DBB200219B
:1040BC000191009300230021022000F053FD194BC5
:1040CC0003221A7023E01D4B1B88DAB21C4B1B8891
:1040DC00DBB20A210191009300230021022000F0A1
:1040EC0041FD0346002B14D10E4B04221A7010E034
:1040FC0000220021022000F0B5FB00220121022049
:10410C0000F0B0FB06E000BF04E000BF02E000BF1F
:10411C0000E000BF034B1B7818466837BD4680BDD6
:10412C000C0000206704002044F40008A8030020C1
:10413C00FC0300203C0400204C040020060400205A
:10414C00180400203E04002080B59CB002AF5D4BEB
:10415C001A785D4B1B789A4217D05B4B1A78594BE7
:10416C001A70594B1B781A463B1D584918460AF0D1
:10417C0097F93B1D1846FBF7E3FF03469AB2391D2E
:10418C004FF0FF33524805F09BFB524B1B889AB201
:10419C00514B1B889A4202D24B4B00221A704A4B4D
:1041AC001B78032B76D801A252F823F0C9410008E2
:1041BC001542000845420008774200080022002101
:1041CC00032000F04FFB00220121032000F04AFBEA
:1041DC00404B1B889AB2404B1B889A4265D33F4B8D
:1041EC009B88DAB23E4B1B88D9B23E4B1B88DBB2A4
:1041FC000020019000930B460121032000F0B2FC3B
:10420C00314B01221A7050E0344B9B88DAB2364B9A
:10421C001B88D9B2334B1B88DBB20A200190009368
:10422C000B460121032000F09DFC0346002B3ED1E0
:10423C00254B02221A703AE0264B1B889AB22B4B64
:10424C001B889A4235D3284B1B88DAB2254B1B8826
:10425C00DBB200210191009300230121032000F027
:10426C0081FC194B03221A7023E01F4B1B88DAB216
:10427C001C4B1B88DBB20A21019100930023012106
:10428C00032000F06FFC0346002B14D10E4B0422CC
:10429C001A7010E000220021032000F0E3FA002243
:1042AC000121032000F0DEFA06E000BF04E000BFAD
:1042BC0002E000BF00E000BF034B1B7818466837D4
:1042CC00BD4680BD0D0000206804002050F400089D
:1042DC00A8030020FC030020400400204C04002014
:1042EC0006040020180400200A04002042040020C8
:1042FC0080B59CB002AF5D4B1A785D4B1B789A422F
:10430C0017D05B4B1A78594B1A70594B1B781A46BD
:10431C003B1D584918460AF0C3F83B1D1846FBF7DD
:10432C000FFF03469AB2391D4FF0FF33524805F088
:10433C00C7FA524B1B889AB2514B1B889A4202D235
:10434C004B4B00221A704A4B1B78032B76D801A2D8
:10435C0052F823F071430008BD430008ED430008F8
:10436C001F44000800220021042000F07BFA0022E8
:10437C000121042000F076FA404B1B889AB2404B86
:10438C001B889A4265D33F4BDB88DAB23E4B1B88C5
:10439C00D9B23E4B1B88DBB20020019000930B4638
:1043AC000121042000F0DEFB314B01221A7050E099
:1043BC00344BDB88DAB2344B1B88D9B2334B1B88B5
:1043CC00DBB20A20019000930B460121042000F07F
:1043DC00C9FB0346002B3ED1254B02221A703AE052
:1043EC00264B1B889AB22A4B1B889A4235D3264BF4
:1043FC001B88DAB2254B1B88DBB20021019100939C
:10440C0000230121042000F0ADFB194B03221A708C
:10441C0023E01D4B1B88DAB21C4B1B88DBB20A2134
:10442C000191009300230121042000F09BFB034623
:10443C00002B14D10E4B04221A7010E00022002124
:10444C00042000F00FFA00220121042000F00AFAE7
:10445C0006E000BF04E000BF02E000BF00E000BFC8
:10446C00034B1B7818466837BD4680BD0E000020F4
:10447C00690400205CF40008A8030020FC03002061
:10448C00440400204C0400200E04002018040020DA
:10449C004604002080B584B000AF7860396039687C
:1044AC00786804F086FE0346FB73FB7B022B0CBF83
:1044BC0001230023DBB218461037BD4680BD80B502
:1044CC0082B000AF786039603968786804F084FC99
:1044DC0000BF0837BD4680BD80B584B000AFF86022
:1044EC00B9601346FB80BB68002B04D1FB681B68CA
:1044FC00FA885A6313E0BB68042B04D1FB681A6872
:10450C00FB8893630BE0BB68082B04D1FB681A682B
:10451C00FB88D36303E0FB681A68FB881364B968F3
:10452C00F86804F0B7FB00BF1037BD4680BD80B4FF
:10453C0085B000AFF860B9601346FB80BB68002BF8
:10454C0004D1FB681B68FA885A6313E0BB68042B20
:10455C0004D1FB681A68FB8893630BE0BB68082BDB
:10456C0004D1FB681A68FB88D36303E0FB681A6804
:10457C00FB88136400BF1437BD4680BC7047000035
:10458C0080B582B000AF0346FB710B46BB7113467E
:10459C00BB80FB79013B032B00F2588101A252F83E
:1045AC0023F000BFC145000863460008054700081A
:1045BC00AF470008BB79002B26D1BB88002B09D153
:1045CC000021A548FFF77BFF00220221A34802F03F
:1045DC0078F83CE10021A048FFF75CFF0346002B74
:1045EC0006D0BB881A4600219B48FFF7A0FF2EE19E
:1045FC0001220221994802F064F8BB881A46002176
:10460C009548FFF769FF22E1BB88002B09D10421F3
:10461C009148FFF754FF00220221904802F051F814
:10462C0015E104218C48FFF735FF0346002B06D01B
:10463C00BB881A4604218848FFF779FF07E101225D
:10464C000221864802F03DF8BB881A4604218248B4
:10465C00FFF742FFFBE0BB79002B26D1BB88002B78
:10466C0009D108217C48FFF72AFF002204217B484E
:10467C0002F027F8EBE008217748FFF70BFF034621
:10468C00002B06D0BB881A4608217348FFF74FFF52
:10469C00DDE001220421714802F013F8BB881A46B0
:1046AC0008216D48FFF718FFD1E0BB88002B09D11A
:1046BC000C216948FFF703FF00220421674802F030
:1046CC0000F8C4E00C216448FFF7E4FE0346002B1D
:1046DC0006D0BB881A460C215F48FFF728FFB6E0CE
:1046EC00012204215D4801F0ECFFBB881A460C2125
:1046FC005948FFF7F1FEAAE0BB79002B28D1BB8803
:10470C00002B0AD100215648FFF7D9FE00224FF4A6
:10471C008061524801F0D5FF99E000215048FFF725
:10472C00B9FE0346002B06D0BB881A4600214C4824
:10473C00FFF7FDFE8BE001224FF48061474801F04A
:10474C00C0FFBB881A4600214548FFF7C5FE7EE036
:10475C00BB88002B0AD104214148FFF7B0FE002290
:10476C004FF480613D4801F0ACFF70E004213C48FF
:10477C00FFF790FE0346002B06D0BB881A46042197
:10478C003748FFF7D4FE62E001224FF480613348D2
:10479C0001F097FFBB881A4604213148FFF79CFEB5
:1047AC0055E0BB79002B28D1BB88002B0AD10821FE
:1047BC002B48FFF784FE00224FF40061274801F0DC
:1047CC0080FF44E008212648FFF764FE0346002BD7
:1047DC0006D0BB881A4608212148FFF7A8FE36E010
:1047EC0001224FF400611D4801F06BFFBB881A4693
:1047FC0008211B48FFF770FE29E0BB88002B0AD16B
:10480C000C211748FFF75BFE00224FF400611348A0
:10481C0001F057FF1BE00C211148FFF73BFE03464C
:10482C00002B06D0BB881A460C210D48FFF77FFEE3
:10483C000DE001224FF40061084801F042FFBB88F3
:10484C001A460C210648FFF747FE00E000BF00BFE8
:10485C000837BD4680BD00BF18030020000C014086
:10486C006003002080B584B000AF0346FB710B469B
:10487C00BB7113467B717B79FB60FB689B03FB6010
:10488C00FB68B44AA2FB03235B09FB60FB687B81DA
:10489C00FB79013B032B00F2578101A252F823F064
:1048AC00BD4800085F490008014A0008AB4A0008EF
:1048BC00BB79002B26D17B89002B09D10021A6487E
:1048CC00FFF7FDFD00220221A44801F0FAFE3CE1B5
:1048DC000021A148FFF7DEFD0346002B06D07B89A3
:1048EC001A4600219C48FFF722FE2EE101220221EC
:1048FC009A4801F0E6FE7B891A4600219648FFF79C
:10490C00EBFD22E17B89002B09D104219248FFF7B2
:10491C00D6FD00220221914801F0D3FE15E10421BD
:10492C008D48FFF7B7FD0346002B06D07B891A464E
:10493C0004218948FFF7FBFD07E10122022187488A
:10494C0001F0BFFE7B891A4604218348FFF7C4FDA2
:10495C00FBE0BB79002B26D17B89002B09D10821E8
:10496C007D48FFF7ACFD002204217C4801F0A9FE34
:10497C00EBE008217848FFF78DFD0346002B06D0AD
:10498C007B891A4608217448FFF7D1FDDDE001222E
:10499C000421724801F095FE7B891A4608216E4865
:1049AC00FFF79AFDD1E07B89002B09D10C216A48D5
:1049BC00FFF785FD00220421684801F082FEC4E067
:1049CC000C216548FFF766FD0346002B06D07B895A
:1049DC001A460C216048FFF7AAFDB6E0012204211B
:1049EC005E4801F06EFE7B891A460C215A48FFF78F
:1049FC0073FDAAE0BB79002B28D17B89002B0AD14F
:104A0C0000215748FFF75BFD00224FF480615348AB
:104A1C0001F057FE99E000215148FFF73BFD03469A
:104A2C00002B06D07B891A4600214D48FFF77FFDED
:104A3C008BE001224FF48061484801F042FE7B89F3
:104A4C001A4600214648FFF747FD7EE07B89002B84
:104A5C000AD104214248FFF732FD00224FF4806155
:104A6C003E4801F02EFE70E004213D48FFF712FD98
:104A7C000346002B06D07B891A4604213848FFF7E1
:104A8C0056FD62E001224FF48061344801F019FEBA
:104A9C007B891A4604213248FFF71EFD55E0BB798D
:104AAC00002B28D17B89002B0AD108212C48FFF739
:104ABC0006FD00224FF40061284801F002FE44E09C
:104ACC0008212748FFF7E6FC0346002B06D07B891C
:104ADC001A4608212248FFF72AFD36E001224FF43E
:104AEC0000611E4801F0EDFD7B891A4608211C4827
:104AFC00FFF7F2FC29E07B89002B0AD10C21184826
:104B0C00FFF7DDFC00224FF40061144801F0D9FDE1
:104B1C001BE00C211248FFF7BDFC0346002B06D00E
:104B2C007B891A460C210E48FFF701FD0DE001228E
:104B3C004FF40061094801F0C4FD7B891A460C2131
:104B4C000748FFF7C9FC00E000BF00BF1037BD46A7
:104B5C0080BD00BF1F85EB5118030020000C0140E5
:104B6C006003002090B585B000AF0446084611469E
:104B7C001A462346FB710346BB710B467B711346E9
:104B8C003B7197F82430002B02D00A2B16D09DE0F5
:104B9C00FB79013B97F8202091B24F4A084622F846
:104BAC001300FB79013BC9B24C4AD1547A79B979DB
:104BBC00FB791846FFF756FE002388E0FB79013B92
:104BCC00464AD35C1946FB79013B434A32F8133011
:104BDC009BB2994278D0FB79013B3F4A32F81330B3
:104BEC009AB2FB79013BD1B23C4AD154FB79013BDF
:104BFC00394A32F813309BB2002B5DD07A793B796D
:104C0C009A4226D97B799AB23B799BB2D31AFB8113
:104C1C0097F820309AB2FB79013B2F4931F81330C9
:104C2C009BB2D31A9BB2FA8902FB03F3FB81FA897C
:104C3C0097F8203092FBF3F3FB81FB89DBB27A7996
:104C4C00D31ADAB2B979FB791846FFF70BFE0123B8
:104C5C003DE07A793B799A4226D23B799AB27B79BC
:104C6C009BB2D31AFB8197F820309AB2FB79013BA7
:104C7C00194931F813309BB2D31A9BB2FA8902FB53
:104C8C0003F3FB81FA8997F8203092FBF3F3FB8155
:104C9C00FB89DAB27B791344DAB2B979FB7918461D
:104CAC00FFF7E0FD012312E03A79B979FB79184658
:104CBC00FFF7D8FD00230AE03A79B979FB79184659
:104CCC00FFF7D0FD002302E0012300E0002318468B
:104CDC001437BD4690BD00BFF40300206C040020C7
:104CEC0080B485B000AF154B9B69144A43F00103A7
:104CFC009361124B9B6903F00103BB60BB680F4BC4
:104D0C00DB690E4A43F08053D3610C4BDB6903F033
:104D1C0080537B607B680A4B5B68FB60FB6823F00D
:104D2C00E063FB60FB6843F00073FB60044AFB68C4
:104D3C00536000BF1437BD4680BC70470010024062
:104D4C000000014080B58AB000AF786007F118030D
:104D5C0000221A605A609A60DA607B681B68334ADA
:104D6C0093425FD1324B9B69314A43F40073936198
:104D7C002F4B9B6903F400737B617B692C4B9B6904
:104D8C002B4A43F004039361294B9B6903F0040302
:104D9C003B613B69264B9B69254A43F008039361B1
:104DAC00234B9B6903F00803FB60FB68F023BB619A
:104DBC000323FB6107F1180319461E4801F0E6FABC
:104DCC000123BB610323FB6107F1180319461A4841
:104DDC0001F0DCFA194B1A4A1A60184B00225A607F
:104DEC00164B00229A60154B8022DA60134B4FF45D
:104DFC0080721A61114B4FF480625A610F4B202262
:104E0C009A610E4B0022DA610C4800F0D1FE034689
:104E1C00002B01D0FEF7A2FC7B68084A1A62074AF5
:104E2C007B68536200BF2837BD4680BD002401401B
:104E3C000010024000080140000C0140D402002088
:104E4C000800024080B485B000AF78607B681B68B6
:104E5C00B3F1804F0CD1114BDB69104A43F00103C5
:104E6C00D3610E4BDB6903F00103FB60FB6810E0C0
:104E7C007B681B680A4A93420BD1084BDB69074AD3
:104E8C0043F00403D361054BDB6903F00403BB60FF
:104E9C00BB6800BF1437BD4680BC70470010024091
:104EAC000008004080B588B000AF786007F11003AF
:104EBC0000221A605A609A60DA607B681B68B3F152
:104ECC00804F18D11D4B9B691C4A43F0040393611E
:104EDC001A4B9B6903F00403FB60FB680F233B61D7
:104EEC0002237B610223FB6107F11003194614486E
:104EFC0001F04CFA1DE07B681B68124A934218D1F2
:104F0C000E4B9B690D4A43F0080393610B4B9B6955
:104F1C0003F00803BB60BB684FF470733B61022362
:104F2C007B610223FB6107F110031946064801F06F
:104F3C002DFA00BF2037BD4680BD00BF00100240D7
:104F4C000008014000080040000C014080B588B00A
:104F5C0000AF786007F1100300221A605A609A6063
:104F6C00DA607B681B681C4A934231D11B4B9B69EE
:104F7C001A4A43F480439361184B9B6903F48043B2
:104F8C00FB60FB68154B9B69144A43F00403936167
:104F9C00124B9B6903F00403BB60BB684FF40073B6
:104FAC003B6102237B610323FB6107F1100319466C
:104FBC000B4801F0EBF94FF480633B6100237B61FC
:104FCC000023BB6107F110031946054801F0DEF917
:104FDC0000BF2037BD4680BD0038014000100240A4
:104FEC000008014080B400AF00BFFDE780B400AF03
:104FFC0000BFFDE780B400AF00BFFDE780B400AF99
:10500C0000BFFDE780B400AF00BFFDE780B400AF88
:10501C0000BFBD4680BC704780B400AF00BFBD462A
:10502C0080BC704780B400AF00BFBD4680BC7047E9
:10503C0080B500AF00F0C0F800F0B3FD00BF80BD3C
:10504C0080B500AF024800F06DFE00BF80BD00BF10
:10505C00D402002080B500AF024801F066FC00BF0E
:10506C0080BD00BF6412002080B586B000AF7860B0
:10507C00144A154BD31A7B617B693B61134B1B683C
:10508C00002B02D1114B124A1A60104B1A687B6824
:10509C0013443A699A4207D209F02CFA03460C22BF
:1050AC001A604FF0FF3309E0084B1B68FB60074B9D
:1050BC001A687B681344054A1360FB681846183756
:1050CC00BD4680BD0050002000040000700400208C
:1050DC00A818002080B400AF00BFBD4680BC70474C
:1050EC00FFF7F8FF0B480C490C4A002302E0D45898
:1050FC00C4500433C4188C42F9D3094A094C002318
:10510C0001E013600432A242FBD309F0F9F9FDF778
:10511C00A3FF704700000020DC01002020F60008EF
:10512C00E0010020A4180020FEE7000080B500AFCD
:10513C00084B1B68074A43F010031360032000F070
:10514C00EFFC0F2000F008F8FFF7CAFD002318460B
:10515C0080BD00BF0020024080B582B000AF7860F7
:10516C00124B1A68124B1B7819464FF47A73B3FB27
:10517C00F1F3B2FBF3F3184600F007FD0346002BE6
:10518C0001D001230EE07B680F2B0AD8002279682E
:10519C004FF0FF3000F0CFFC064A7B681360002311
:1051AC0000E0012318460837BD4680BD10000020E2
:1051BC00180000201400002080B400AF054B1B78B1
:1051CC001A46054B1B681344034A136000BFBD46C7
:1051DC0080BC7047180000207404002080B400AF1D
:1051EC00024B1B681846BD4680BC704774040020F7
:1051FC0080B586B000AF78600023FB7500233B615F
:10520C000023BB600023FB607B68002B01D10123D2
:10521C00BEE07B689B68002B7B689B6A002B09D1E6
:10522C007B680022DA627B68002283F8242078688D
:10523C00FFF788FD786800F0FFFA0346FB757B6882
:10524C009B6A03F01003002B40F09980FB7D002B30
:10525C0040F095807B689B6A23F4885323F002030B
:10526C0043F002027B689A627B685A687B68DB6950
:10527C001A437B681B7B5B001343BA681343BB6008
:10528C007B689B68B3F5807F03D07B689B68012BA0
:10529C0002D14FF4807300E000233A6913433B6161
:1052AC007B681B7D012B19D17B681B7B002B09D1E3
:1052BC007B689B69013B5A033B69134343F40063CE
:1052CC003B610BE07B689B6A43F020027B689A622F
:1052DC007B68DB6A43F001027B68DA627B681B68DF
:1052EC005B6823F469417B681B683A690A435A601E
:1052FC007B681B689A68284B13407A681268B968F7
:10530C000B4393607B689B68B3F5807F03D07B680D
:10531C009B68012B04D17B681B69013B1B05FB605F
:10532C007B681B68DB6A23F470017B681B68FA6876
:10533C000A43DA627B681B689A68184B1340BA6898
:10534C009A420BD17B680022DA627B689B6A23F05D
:10535C00030343F001027B689A6218E07B689B6A46
:10536C0023F0120343F010027B689A627B68DB6ABD
:10537C0043F001027B68DA620123FB7507E07B686E
:10538C009B6A43F010027B689A620123FB75FB7DDC
:10539C0018461837BD4680BDFDF7E1FFFE0E1FFF16
:1053AC0080B586B000AFF860B9607A600023FB75F9
:1053BC00FB681B68644A934204D0FB681B68634A11
:1053CC00934206D1604B5B6803F47023002B40F0D2
:1053DC00B380FB6893F82430012B01D10223AEE09B
:1053EC00FB68012283F82420F86800F0CBF903460F
:1053FC00FB75FB7D002B40F09A80FB689B6A23F4C5
:10540C00706323F0010343F48072FB689A62FB68BB
:10541C001B684E4A934205D14B4B5B6803F47023D7
:10542C00002B15D1FB689B6A23F48012FB689A62EF
:10543C00FB681B685B6803F48063002B26D0FB6859
:10544C009B6A23F4405343F48052FB689A621DE03C
:10545C00FB689B6A43F48012FB689A62FB681B68CA
:10546C00394A934204D0FB681B68384A93420DD1E9
:10547C00354B5B6803F48063002B07D0FB689B6A99
:10548C0023F4405343F48052FB689A62FB689B6A96
:10549C0003F48053002B06D0FB68DB6A23F0060272
:1054AC00FB68DA6202E0FB680022DA62FB68002229
:1054BC0083F82420FB681B6A254A9A62FB681B6AE6
:1054CC00244ADA62FB681B6A234A1A63FB681B686E
:1054DC006FF002021A60FB681B689A68FB681B6815
:1054EC0042F480729A60FB68186AFB681B684C3344
:1054FC001946BA687B6800F0B5FBFB681B689B68B3
:10550C0003F46023B3F5602F08D1FB681B689A681D
:10551C00FB681B6842F4A0029A600FE0FB681B68F2
:10552C009A68FB681B6842F480129A6006E0FB687C
:10553C00002283F8242001E00123FB75FB7D184633
:10554C001837BD4680BD00BF002401400028014033
:10555C00C7580008435900085F59000880B483B04D
:10556C0000AF786000BF0C37BD4680BC704780B47C
:10557C0083B000AF786000BF0C37BD4680BC70476D
:10558C0080B483B000AF786000BF0C37BD4680BCE0
:10559C007047000080B485B000AF7860396000239C
:1055AC00FB730023BB607B6893F82430012B01D183
:1055BC000223DCE07B68012283F824203B685B68D3
:1055CC00062B1CD87B681B68596B3B685A681346C2
:1055DC009B001344053B1F2202FA03F3DB431940E3
:1055EC003B6818683B685A6813469B001344053B9C
:1055FC0000FA03F27B681B680A435A633CE03B6881
:10560C005B680C2B1CD87B681B68196B3B685A6851
:10561C0013469B001344233B1F2202FA03F3DB4384
:10562C0019403B6818683B685A6813469B00134442
:10563C00233B00FA03F27B681B680A431A631BE0E6
:10564C007B681B68D96A3B685A6813469B001344F5
:10565C00413B1F2202FA03F3DB4319403B681868F5
:10566C003B685A6813469B001344413B00FA03F213
:10567C007B681B680A43DA623B681B68092B1CD9E0
:10568C007B681B68D9683B681A6813465B00134437
:10569C001E3B072202FA03F3DB4319403B68986870
:1056AC003B681A6813465B0013441E3B00FA03F276
:1056BC007B681B680A43DA6019E07B681B68196910
:1056CC003B681A6813465B001344072202FA03F383
:1056DC00DB4319403B6898683B681A6813465B00CB
:1056EC00134400FA03F27B681B680A431A613B6897
:1056FC001B68102B03D03B681B68112B32D17B68C5
:10570C001B681D4A934225D17B681B689B6803F478
:10571C000003002B26D17B681B689A687B681B688A
:10572C0042F400029A603B681B68102B1AD1134B91
:10573C001B68134AA2FB03239A0C13469B001344C9
:10574C005B00BB6002E0BB68013BBB60BB68002B2D
:10575C00F9D107E07B689B6A43F020027B689A6270
:10576C000123FB737B68002283F82420FB7B184603
:10577C001437BD4680BC7047002401401000002047
:10578C0083DE1B4380B584B000AF78600023FB60E0
:10579C000023BB607B681B689B6803F00103012B33
:1057AC0040D07B681B689A687B681B6842F00102DA
:1057BC009A601F4B1B681F4AA2FB03239B0CBB6008
:1057CC0002E0BB68013BBB60BB68002BF9D1FFF763
:1057DC0005FDF8601FE0FFF701FD0246FB68D31AD8
:1057EC00022B18D97B681B689B6803F00103012B03
:1057FC0011D07B689B6A43F010027B689A627B68CD
:10580C00DB6A43F001027B68DA627B68002283F872
:10581C002420012307E07B681B689B6803F00103CD
:10582C00012BD8D1002318461037BD4680BD00BFD0
:10583C001000002083DE1B4380B584B000AF78607D
:10584C000023FB607B681B689B6803F00103012B42
:10585C002ED17B681B689A687B681B6822F001025A
:10586C009A60FFF7BBFCF8601BE0FFF7B7FC024641
:10587C00FB68D31A022B14D97B681B689B6803F056
:10588C000103012B0DD17B689B6A43F010027B68EE
:10589C009A627B68DB6A43F001027B68DA6201235F
:1058AC0007E07B681B689B6803F00103012BDCD0CD
:1058BC00002318461037BD4680BD80B584B000AFBC
:1058CC0078607B685B6AFB60FB689B6A03F0500343
:1058DC00002B27D1FB689B6A43F40072FB689A6229
:1058EC00FB681B689B6803F46023B3F5602F15D12C
:1058FC00FB681B7B002B11D1FB689B6A23F4807225
:10590C00FB689A62FB689B6A03F48053002B05D1F9
:10591C00FB689B6A43F00102FB689A62F868FFF728
:10592C001DFE04E0FB681B6A1B6B7868984700BF80
:10593C001037BD4680BD80B584B000AF78607B6801
:10594C005B6AFB60F868FFF712FE00BF1037BD46BC
:10595C0080BD80B584B000AF78607B685B6AFB600B
:10596C00FB689B6A43F04002FB689A62FB68DB6A47
:10597C0043F00402FB68DA62F868FFF701FE00BF2F
:10598C001037BD4680BD000080B485B000AF786094
:10599C007B6803F00703FB600C4BDB68BB60BA68E9
:1059AC004FF6FF031340BB60FB681A02BB6813433E
:1059BC0043F0BF6343F40033BB60044ABB68D3605D
:1059CC0000BF1437BD4680BC704700BF00ED00E03F
:1059DC0080B400AF044BDB681B0A03F007031846C6
:1059EC00BD4680BC704700BF00ED00E080B483B0C2
:1059FC0000AF0346FB7197F90730002B0BDBFB79EB
:105A0C0003F01F02064997F907305B09012000FAE1
:105A1C0002F241F8232000BF0C37BD4680BC704712
:105A2C0000E100E080B483B000AF03463960FB7145
:105A3C0097F90730002B0ADB3B68DAB20C4997F96F
:105A4C0007301201D2B20B4483F800230AE03B6802
:105A5C00DAB20849FB7903F00F03043B1201D2B20E
:105A6C000B441A7600BF0C37BD4680BC704700BF94
:105A7C0000E100E000ED00E080B489B000AFF86018
:105A8C00B9607A60FB6803F00703FB61FB69C3F143
:105A9C000703042B28BF0423BB61FB690433062BCB
:105AAC0002D9FB69033B00E000237B614FF0FF321E
:105ABC00BB6902FA03F3DA43BB681A407B699A406C
:105ACC004FF0FF317B6901FA03F3D9437B680B403C
:105ADC00134318462437BD4680BC704780B582B04E
:105AEC0000AF78607B68013BB3F1807F01D3012369
:105AFC000FE00A4A7B68013B53600F214FF0FF30E7
:105B0C00FFF790FF054B00229A60044B07221A60A6
:105B1C00002318460837BD4680BD00BF10E000E0EA
:105B2C0080B582B000AF78607868FFF72DFF00BFBA
:105B3C000837BD4680BD80B586B000AF0346B9605E
:105B4C007A60FB7300237B61FFF742FF78617A6810
:105B5C00B9687869FFF790FF024697F90F30114644
:105B6C001846FFF75FFF00BF1837BD4680BD80B5F4
:105B7C0082B000AF0346FB7197F907301846FFF768
:105B8C0035FF00BF0837BD4680BD80B582B000AF81
:105B9C0078607868FFF7A2FF034618460837BD46C1
:105BAC0080BD80B500AFFCF727F800BF80BD0000BA
:105BBC0080B485B000AF78600023FB607B68002B5D
:105BCC0001D1012343E07B681B681A46224B134426
:105BDC00224AA2FB03231B099A007B681A647B6888
:105BEC001F4ADA637B68022283F821207B681B68DA
:105BFC001B68FB60FB6823F47F5323F03003FB60CE
:105C0C007B685A687B689B681A437B68DB681A431D
:105C1C007B681B691A437B685B691A437B689B69C9
:105C2C001A437B68DB691343FA681343FB607B6898
:105C3C001B68FA681A607B6800229A637B680122F1
:105C4C0083F821207B68002283F82020002318464B
:105C5C001437BD4680BC7047F8FFFDBFCDCCCCCC13
:105C6C000000024080B586B000AFF860B9607A6081
:105C7C003B600023FB75FB6893F82030012B01D1AE
:105C8C0002234BE0FB68012283F82020FB6893F889
:105C9C002130DBB2012B3AD1FB68022283F82120A0
:105CAC00FB6800229A63FB681B681A68FB681B6818
:105CBC0022F001021A603B687A68B968F86800F053
:105CCC0037F9FB68DB6A002B08D0FB681B681A6885
:105CDC00FB681B6842F00E021A600FE0FB681B6841
:105CEC001A68FB681B6822F004021A60FB681B68C8
:105CFC001A68FB681B6842F00A021A60FB681B6892
:105D0C001A68FB681B6842F001021A6005E0FB6828
:105D1C00002283F820200223FB75FB7D18461837E0
:105D2C00BD4680BD80B584B000AF78607B68DB6B0E
:105D3C001B68FB607B681B681B68BB607B681B6C0B
:105D4C0004229A40FB681340002B4FD0BB6803F031
:105D5C000403002B4AD07B681B681B6803F02003EC
:105D6C00002B07D17B681B681A687B681B6822F0C4
:105D7C0004021A607B681B68664A934229D07B68D0
:105D8C001B68654A934222D07B681B68634A934226
:105D9C001AD07B681B68624A934212D07B681B68DE
:105DAC00604A93420AD07B681B685F4A934202D1D7
:105DBC004FF480030EE04FF080630BE04FF4802330
:105DCC0008E04FF4804305E04FF4806302E0402389
:105DDC0000E00423554A53607B68DB6A002B00F01B
:105DEC0094807B68DB6A786898478EE07B681B6CD4
:105DFC0002229A40FB681340002B56D0BB6803F07C
:105E0C000203002B51D07B681B681B6803F0200336
:105E1C00002B0BD17B681B681A687B681B6822F00F
:105E2C000A021A607B68012283F821207B681B68B8
:105E3C00384A934229D07B681B68374A934222D058
:105E4C007B681B68354A93421AD07B681B68344ABE
:105E5C00934212D07B681B68324A93420AD07B680B
:105E6C001B68314A934202D14FF400130EE04FF0FD
:105E7C0000730BE04FF4003308E04FF4005305E0DF
:105E8C004FF4007302E0202300E00223274A536002
:105E9C007B68002283F820207B689B6A002B34D01F
:105EAC007B689B6A786898472FE07B681B6C08229C
:105EBC009A40FB681340002B28D0BB6803F0080302
:105ECC00002B23D07B681B681A687B681B6822F048
:105EDC000E021A607B681A6C7B68DB6B012101FA7D
:105EEC0002F25A607B6801229A637B68012283F874
:105EFC0021207B68002283F820207B681B6B002B01
:105F0C0004D07B681B6B7868984700BF00BF1037C4
:105F1C00BD4680BD080002401C000240300002401B
:105F2C0044000240580002406C0002400000024055
:105F3C0080B485B000AFF860B9607A603B60FB68F4
:105F4C001A6CFB68DB6B012101FA02F25A60FB68E8
:105F5C001B683A685A60FB685B68102B08D1FB68B9
:105F6C001B687A689A60FB681B68BA68DA6007E09D
:105F7C00FB681B68BA689A60FB681B687A68DA6011
:105F8C0000BF1437BD4680BC70470000F0B587B029
:105F9C0000AFF860B960C7E900230123FB7500234B
:105FAC00BB7500237B752F4B1B7E012B01D102236C
:105FBC0054E02C4B01221A764CF2503000F0A8F829
:105FCC000346FB75FB7D002B44D1FB68012B02D1F2
:105FDC0001237B7507E0FB68022B02D102237B7542
:105FEC0001E004237B750023BB752DE0BB7D5A00BB
:105FFC00BB6802EB030CBB7D1901D7E90023C1F18F
:10600C002006A1F1200022FA01F403FA06F634432B
:10601C0023FA00F0044323FA01F5A3B219466046B3
:10602C0000F05AF84CF2503000F072F80346FB7551
:10603C000D4B1B690C4A23F001031361FB7D002BF4
:10604C0007D1BB7D0133BB75BA7D7B7D9A42CDD325
:10605C0000E000BF034B00221A76FB7D18461C376C
:10606C00BD46F0BD780400200020024080B483B00F
:10607C0000AF0023FB710D4B1B6903F08003002B59
:10608C000DD00A4B0A4A5A60084B0A4A5A60074B11
:10609C001B6903F08003002B01D00123FB71FB79FA
:1060AC0018460C37BD4680BC704700BF002002402C
:1060BC0023016745AB89EFCD80B400AF054B1B695D
:1060CC00044A43F08003136100231846BD4680BC8C
:1060DC00704700BF0020024080B483B000AF7860EE
:1060EC000B467B80084B0022DA61084B1B69074A80
:1060FC0043F0010313617B687A881A8000BF0C3768
:10610C00BD4680BC704700BF7804002000200240D0
:10611C0080B584B000AF7860FFF760F8F86010E0ED
:10612C007B68B3F1FF3F0CD07B68002B07D0FFF7E7
:10613C0055F80246FB68D31A7A689A4201D20323B7
:10614C0025E0154BDB6803F00103002BE8D1124B63
:10615C00DB6803F02003002B02D00F4B2022DA6007
:10616C000D4BDB6803F01003002B0BD10A4BDB69E2
:10617C0003F00103002B05D1074BDB6803F004038C
:10618C00002B03D000F00AF8012300E0002318468E
:10619C001037BD4680BD00BF0020024080B483B0E4
:1061AC0000AF00237B60234BDB6803F01003002B54
:1061BC0009D0214BDB6943F002031F4AD3617B6892
:1061CC0043F010037B601B4BDB6803F00403002BD4
:1061DC0009D0194BDB6943F00103174AD3617B6883
:1061EC0043F004037B60134BDB6903F00103002BCA
:1061FC000BD0114BDB6943F004030F4AD3610D4BF9
:10620C00DB690C4A23F00103D3617B6840F2011275
:10621C00934206D1074BDB69064A23F00103D36195
:10622C0002E0044A7B68D36000BF0C37BD4680BCDB
:10623C00704700BF002002407804002080B584B075
:10624C0000AF786039600123FB730023BB602F4BD8
:10625C001B7E012B01D1022353E02C4B01221A7619
:10626C007B681B68022B16D14CF25030FFF750FFA5
:10627C000346002B41D1012000F04CF84CF2503079
:10628C00FFF746FF0346FB73214B1B69204A23F0A3
:10629C000403136131E04CF25030FFF739FF034631
:1062AC00002B2AD13B684FF0FF321A607B689B6849
:1062BC00BB6019E0B86800F049F84CF25030FFF7B9
:1062CC0027FF0346FB73124B1B69114A23F0020391
:1062DC001361FB7B002B03D03B68BA681A600CE09F
:1062EC00BB6803F58063BB607B68DB689A027B68E4
:1062FC009B681344BA689A42DCD3044B00221A768A
:10630C00FB7B18461037BD4680BD00BF78040020CB
:10631C000020024080B483B000AF7860094B0022AB
:10632C00DA61094B1B69084A43F004031361064BFD
:10633C001B69054A43F04003136100BF0C37BD468F
:10634C0080BC7047780400200020024080B483B0E9
:10635C0000AF78600B4B0022DA610B4B1B690A4AC9
:10636C0043F002031361084A7B685361064B1B69B7
:10637C00054A43F04003136100BF0C37BD4680BC97
:10638C00704700BF780400200020024080B48BB01E
:10639C0000AF7860396000237B6200233B6269E1C7
:1063AC0001227B6A02FA03F3FB613B681B68FA6902
:1063BC001340BB61BA69FB699A4240F058813B6853
:1063CC005B689A4A93425ED0984A934275D8984A31
:1063DC00934258D0964A93426FD8964A934252D0E1
:1063EC00944A934269D8944A93424CD0924A93422D
:1063FC0063D8924A934246D0904A93425DD8122B6E
:10640C002AD8122B59D801A252F823F09364000811
:10641C006D6400087F640008C1640008C76400084C
:10642C00C7640008C7640008C7640008C764000894
:10643C00C7640008C7640008C7640008C764000884
:10644C00C7640008C7640008C7640008C764000874
:10645C007564000889640008794A934213D02CE0D3
:10646C003B68DB683B6229E03B68DB6804333B62DA
:10647C0024E03B68DB6808333B621FE03B68DB6869
:10648C000C333B621AE03B689B68002B02D104235F
:10649C003B6213E03B689B68012B05D108233B62F0
:1064AC007B68FA691A6109E008233B627B68FA6928
:1064BC005A6103E000233B6200E000BFBB69FF2B85
:1064CC0001D87B6801E07B6804337B61BB69FF2BDF
:1064DC0002D87B6A9B0002E07B6A083B9B003B6115
:1064EC007B691A680F213B6901FA03F3DB431A40FD
:1064FC00396A3B6901FA03F31A437B691A603B68FA
:10650C005B6803F08053002B00F0B1804D4B9B690E
:10651C004C4A43F0010393614A4B9B6903F001031E
:10652C00BB60BB68484A7B6A9B08023352F8233035
:10653C00FB607B6A03F003039B000F2202FA03F358
:10654C00DB43FA681340FB607B68404A934213D0EC
:10655C007B683F4A93420DD07B683E4A934207D0FA
:10656C007B683D4A934201D1032306E0042304E0F7
:10657C00022302E0012300E000237A6A02F0030206
:10658C0092009340FA681343FB602F497B6A9B0887
:10659C000233FA6841F823203B685B6803F48013EC
:1065AC00002B06D02D4B9A682C49BB6913438B608A
:1065BC0006E02A4B9A68BB69DB43284913408B6081
:1065CC003B685B6803F40013002B06D0234BDA689E
:1065DC002249BB691343CB6006E0204BDA68BB69E8
:1065EC00DB431E491340CB603B685B6803F400330C
:1065FC00002B06D0194B5A681849BB6913434B60E2
:10660C0006E0164B5A68BB69DB43144913404B60D8
:10661C003B685B6803F48033002B21D00F4B1A6866
:10662C000E49BB6913430B6021E000BF0000321020
:10663C000000311000002210000021100000121088
:10664C000000111000100240000001400008014041
:10665C00000C0140001001400014014000040140F6
:10666C000B4B1A68BB69DB43094913400B607B6A0F
:10667C0001337B623B681A687B6A22FA03F3002BB6
:10668C007FF48EAE00BF00BF2C37BD4680BC704778
:10669C000004014080B485B000AF78600B467B806D
:1066AC007B689A687B881340002B02D00123FB7314
:1066BC0001E00023FB73FB7B18461437BD4680BCFE
:1066CC00704780B483B000AF78600B467B80134674
:1066DC007B707B78002B03D07A887B681A6103E08F
:1066EC007B881A047B681A6100BF0C37BD4680BCDE
:1066FC00704780B584B000AF78607B68002B01D107
:10670C000123E8E07B6893F89132DBB2002B06D1D1
:10671C007B68002283F89022786807F017FC7B686E
:10672C00032283F891227B6800225A717B681B68D4
:10673C00184603F0BCFA7B6818687B6804330ECBF0
:10674C0003F092FA0346002B05D07B68022283F8F3
:10675C0091220123BFE07B681B680021184603F0DF
:10676C00C0FA0346002B05D07B68022283F89122E5
:10677C000123B0E00023FB733EE0FA7B79681346FB
:10678C009B001344DB000B44113301221A70FA7B7B
:10679C00796813469B001344DB000B441033FA7BDF
:1067AC001A70FA7B796813469B001344DB000B4488
:1067BC00133300221A70FA7B796813469B0013443A
:1067CC00DB000B44203300221A60FA7B79681346F5
:1067DC009B001344DB000B44243300221A60FB7B28
:1067EC0079685A1C13469B001344DB000B440022AF
:1067FC001A60FB7B0133FB737B681B79FA7B9A4233
:10680C00BBD30023FB7344E0FA7B796813469B00EF
:10681C001344DB000B4403F2511300221A70FA7B71
:10682C00796813469B001344DB000B4403F5A873F3
:10683C00FA7B1A70FA7B796813469B001344DB00D1
:10684C000B4403F2531300221A70FA7B7968134637
:10685C009B001344DB000B4403F5B07300221A6059
:10686C00FA7B796813469B001344DB000B4403F559
:10687C00B27300221A60FA7B796813469B001344AA
:10688C00DB000B4403F5B47300221A60FB7B01336D
:10689C00FB737B681B79FA7B9A42B5D37B681868CB
:1068AC007B6804330ECB03F028FA0346002B05D08B
:1068BC007B68022283F8912201230CE07B68002282
:1068CC005A737B68012283F891227B681B681846F7
:1068DC0005F0A7FC002318461037BD4680BD80B5D7
:1068EC0082B000AF78607B6893F89032012B01D1B5
:1068FC00022316E07B68012283F890227B681B68D8
:10690C00184603F0BEF90121786807F092FD7B6808
:10691C001B68184605F07BFC7B68002283F89022EC
:10692C00002318460837BD4680BD80B588B000AF3F
:10693C0078607B681B68184605F07DFCB861BB6904
:10694C0003F40043002B03D0786800F01AFB19E124
:10695C00BB6903F48063002B13D07B681B68B3F80E
:10696C0044309AB27B681B6822F4806292B2A3F81E
:10697C004420786807F065FB0021786800F005F981
:10698C0000E1BB6903F48043002B0CD07B681B68CF
:10699C00B3F844309AB27B681B6822F4804292B2FE
:1069AC00A3F84420EEE0BB6903F40053002B0CD099
:1069BC007B681B68B3F844309AB27B681B6822F47E
:1069CC00005292B2A3F84420DCE0BB6903F480537C
:1069DC00002B27D07B681B68B3F840309AB27B68D9
:1069EC001B6822F0040292B2A3F840207B681B685B
:1069FC00B3F840309AB27B681B6822F0080292B25E
:106A0C00A3F84020786807F055FB7B681B68B3F847
:106A1C0044309AB27B681B6822F4805292B2A3F87D
:106A2C004420AFE0BB6903F40063002B00F08380CB
:106A3C000023FB7710E07B681B681A46FB7F9B00EA
:106A4C001A44FB7F128892B25B0020333B4423F83C
:106A5C00182CFB7F0133FB77FB7F072BEBD97B6873
:106A6C001B68B3F840309AB27B681B6842F0010295
:106A7C0092B2A3F840207B681B68B3F840309AB2FE
:106A8C007B681B6822F0010292B2A3F8402000BF81
:106A9C007B681B68B3F844309BB203F48063002B13
:106AAC00F6D07B681B68B3F844309AB27B681B68DD
:106ABC0022F4806292B2A3F844200023FB770FE00B
:106ACC00FB7F7A6812681146FA7F92000A445B00D9
:106ADC0020333B4433F8183C1380FB7F0133FB77A6
:106AEC00FB7F072BECD97B681B68B3F840309AB25C
:106AFC007B681B6842F0080292B2A3F840207B68C6
:106B0C001B68B3F844309AB27B681B6822F40062AD
:106B1C0092B2A3F844207B681B68B3F840309AB259
:106B2C007B681B6842F0040292B2A3F8402078689C
:106B3C0007F0A6FA26E0BB6903F40073002B0FD014
:106B4C007B681B68B3F844309AB27B681B6822F4EC
:106B5C00007292B2A3F84420786807F064FA11E04E
:106B6C00BB6903F48073002B0CD07B681B68B3F8F3
:106B7C0044309AB27B681B6822F4807292B2A3F8FC
:106B8C00442000BF2037BD4680BD80B582B000AF29
:106B9C0078600B46FB707B6893F89032012B01D127
:106BAC00022312E07B68012283F890227B68FA783A
:106BBC005A737B681B68FA781146184605F014FB6B
:106BCC007B68002283F89022002318460837BD46C4
:106BDC0080BD80B584B000AF7860084611461A4677
:106BEC000346FB700B463B801346BB700023FB72C5
:106BFC0097F90330002B0EDAFB7803F007021346EB
:106C0C009B001344DB0010337A681344FB60FB6871
:106C1C0001225A700EE0FB7803F0070213469B002A
:106C2C001344DB0003F5A8737A681344FB60FB681C
:106C3C0000225A70FB7803F00703DAB2FB681A7073
:106C4C003A88FB681A61FB68BA78DA70BB78022B59
:106C5C0002D1FB6800221A717B6893F89032012BE9
:106C6C0001D102230EE07B68012283F890227B681D
:106C7C001B68F968184603F05DF87B68002283F8FE
:106C8C009022FB7A18461037BD4680BD80B584B083
:106C9C0000AF78600B46FB7097F90330002B0EDACF
:106CAC00FB7803F0070213469B001344DB00103300
:106CBC007A681344FB60FB6801225A700EE0FB7883
:106CCC0003F0070213469B001344DB0003F5A87383
:106CDC007A681344FB60FB6800225A70FB7803F05F
:106CEC000703DAB2FB681A707B6893F89032012BB9
:106CFC0001D102230EE07B68012283F890227B688D
:106D0C001B68F968184603F0D5FB7B68002283F8F2
:106D1C009022002318461037BD4680BD80B586B042
:106D2C0000AFF8607A603B600B46FB72FB7A03F0B5
:106D3C00070213469B001344DB0003F5A873FA68A3
:106D4C0013447B617B697A685A617B693A689A6102
:106D5C007B690022DA617B6900225A70FB7A03F0AE
:106D6C000703DAB27B691A70FB681B6879691846ED
:106D7C0003F08CFD002318461837BD4680BD80B447
:106D8C0083B000AF78600B46FB70FB7803F0070212
:106D9C00796813469B001344DB000B4403F5B67370
:106DAC001B6818460C37BD4680BC704780B586B052
:106DBC0000AFF8607A603B600B46FB72FB7A03F025
:106DCC00070213469B001344DB001033FA6813448C
:106DDC007B617B697A685A617B693A689A617B69E5
:106DEC00012283F824207B693A681A627B690022AD
:106DFC00DA617B6901225A70FB7A03F00703DAB27D
:106E0C007B691A70FB681B687969184603F03EFDB4
:106E1C00002318461837BD4680BD80B584B000AF3E
:106E2C0078600B46FB70FB7803F007037A681279E5
:106E3C00934201D901234CE097F90330002B0EDA71
:106E4C00FB7803F0070213469B001344DB0010335E
:106E5C007A681344FB60FB6801225A700CE0FA78E4
:106E6C0013469B001344DB0003F5A8737A681344A4
:106E7C00FB60FB6800225A70FB6801229A70FB7859
:106E8C0003F00703DAB2FB681A707B6893F8903250
:106E9C00012B01D102231CE07B68012283F8902294
:106EAC007B681B68F968184605F0A1F8FB7803F0BD
:106EBC000703002B08D17B681A687B6803F52673DF
:106ECC001946104605F0C6F97B68002283F890221B
:106EDC00002318461037BD4680BD80B584B000AF86
:106EEC0078600B46FB70FB7803F00F037A6812791D
:106EFC00934201D9012340E097F90330002B0EDABD
:106F0C00FB7803F0070213469B001344DB0010339D
:106F1C007A681344FB60FB6801225A700EE0FB7820
:106F2C0003F0070213469B001344DB0003F5A87320
:106F3C007A681344FB60FB6800225A70FB680022DD
:106F4C009A70FB7803F00703DAB2FB681A707B685F
:106F5C0093F89032012B01D102230EE07B680122C1
:106F6C0083F890227B681B68F968184605F08FF847
:106F7C007B68002283F89022002318461037BD4608
:106F8C0080BD80B596B000AF7860BBE37B681B68B2
:106F9C00B3F84430A7F84E30B7F84E30DBB203F0FC
:106FAC000F0387F84D3097F84D30002B40F075816A
:106FBC00B7F84E3003F01003002B4ED17B681B68E2
:106FCC001B889BB223F4E14323F07003FB817B68A5
:106FDC001A68FB896FEA43436FEA53439BB21380F1
:106FEC007B6810337B657B681B68B3F850309BB2B1
:106FFC001A467B6D1B78DB00134402335B007A6806
:10700C001268134403F580631B88C3F309027B6D7C
:10701C00DA617B6D5A697B6DDB691A447B6D5A6151
:10702C000021786806F0E5FF7B685B7BDBB2002B08
:10703C0000F068837B6D9B69002B40F063837B6859
:10704C005B7BDBB263F07F03DAB27B681B68A3F86F
:10705C004C207B6800225A7354E37B6803F5A873B9
:10706C007B657B681B681B88A7F84A30B7F84A30E9
:10707C0003F40063002B34D07B681B68B3F85030EA
:10708C009BB21A467B6D1B78DB00134406335B0006
:10709C007A681268134403F580631B88C3F30902F2
:1070AC007B6DDA617B6818687B6803F526717B6DF4
:1070BC00DA887B6DDB699BB205F01DF97B681B6878
:1070CC001B889AB240F68F7313403B827B681B6817
:1070DC003A8A42F0800292B21A80786806F05CFF1D
:1070EC0010E3B7F94A30002B80F20C837B681B68E5
:1070FC001B889AB240F68F731340FB837B681B6826
:10710C00FA8B42F0800292B21A807B681B68B3F84B
:10711C0050309BB21A467B6D1B78DB001344063350
:10712C005B007A681268134403F580631B88C3F311
:10713C0009027B6DDA617B6DDB69002B19D07B6DED
:10714C005B69002B15D07B6818687B6D59697B6D6A
:10715C00DA887B6DDB699BB205F0CDF87B6D5A69E3
:10716C007B6DDB691A447B6D5A610021786806F0EF
:10717C0025FF7B681B681B88A7F84A30B7F84A3094
:10718C0003F40063002B40F0BD82B7F84A3003F4DF
:10719C004053B3F5405F00F0B5827B681B68BB6160
:1071AC007B681B68B3F850309BB21A46BB6913441A
:1071BC00BB61BB6903F20C437B617B691B889BB28F
:1071CC00C3F309039AB27B691A807B6D1B693E2B52
:1071DC001DD97B6D1B695B097B647B6D1B6903F09F
:1071EC001F03002B02D17B6C013B7B647B691B88EA
:1071FC009AB27B6C9BB29B029BB213439BB26FEA1D
:10720C0043436FEA53439AB27B691A8026E07B6D45
:10721C001B69002B0AD17B691B889BB26FEA434325
:10722C006FEA53439AB27B691A8017E07B6D1B6936
:10723C005B087B647B6D1B6903F00103002B02D0A0
:10724C007B6C01337B647B691B889AB27B6C9BB231
:10725C009B029BB213439AB27B691A807B681B68B2
:10726C001B889BB223F4804323F070037B827B8AC0
:10727C0083F480537B827B8A83F400537B827B680C
:10728C001A687B8A43F07F4343F47F0343F4004343
:10729C0043F080039BB2138034E27B681B681A4670
:1072AC0097F84D309B0013441B88A7F84A30B7F968
:1072BC004A30002B80F2FC807B681B681A4697F8DA
:1072CC004D309B0013441B889AB240F68F731340C9
:1072DC00A7F848307B681B681A4697F84D309B001E
:1072EC001344B7F8482042F0800292B21A8097F803
:1072FC004D2013469B001344DB0003F5A8737A68FA
:10730C0013447B657B6D1B7B002B25D17B681B6835
:10731C00B3F850309BB21A467B6D1B78DB001344DC
:10732C0006335B007A681268134403F580631B888C
:10733C00C3F30903A7F85030B7F85030002B00F016
:10734C0092807B6818687B6D59697B6DDA88B7F819
:10735C00503004F0D0FF86E07B6DDB78022B0AD135
:10736C00B7F84A301A46796D786800F0D9F90346B7
:10737C00A7F8503077E07B681B681A467B6D1B784A
:10738C009B0013441B889BB223F4E04323F070034F
:10739C00A7F852307B681B681A467B6D1B789B00E4
:1073AC001A44B7F8523043F07F4343F47F0343F45D
:1073BC00004343F0C0039BB213807B681B681A46E2
:1073CC007B6D1B789B0013441B889BB203F480439A
:1073DC00002B24D07B681B68B3F850309BB21A4644
:1073EC007B6D1B78DB00134402335B007A681268F8
:1073FC00134403F580631B88C3F30903A7F85030CB
:10740C00B7F85030002B2ED07B6818687B6D59690B
:10741C007B6D1A89B7F8503004F06DFF23E07B6860
:10742C001B68B3F850309BB21A467B6D1B78DB009F
:10743C00134406335B007A681268134403F58063C7
:10744C001B88C3F30903A7F85030B7F85030002B52
:10745C0009D07B6818687B6D59697B6D5A89B7F8C0
:10746C00503004F048FF7B6DDA69B7F850301A449D
:10747C007B6DDA617B6D5A69B7F850301A447B6DBD
:10748C005A617B6D9B69002B05D0B7F850207B6D42
:10749C001B699A4206D27B6D1B781946786806F0F8
:1074AC008DFD05E07B681B68796D184603F0EEF9DD
:1074BC00B7F84A3003F08003002B00F0238197F8D3
:1074CC004D2013469B001344DB0010337A681344A1
:1074DC007B657B681B681A4697F84D309B001344FC
:1074EC001B889BB223F4E14323F07003A7F84230CE
:1074FC007B681B681A4697F84D309B001A44B7F806
:10750C0042306FEA43436FEA53439BB213807B6D67
:10751C00DB78012B40F0A2807B6D00229A617B6DA1
:10752C001B7B002B00F09380B7F84A3003F040032C
:10753C00002B46D07B6D5B78002B26D17B681B68BB
:10754C007B627B681B68B3F850309BB21A467B6A2F
:10755C0013447B627B6D1B781A017B6A134403F224
:10756C0004433B623B6A1B889BB2C3F309039AB288
:10757C003B6A1A803B6A1B889BB26FEA43436FEAF3
:10758C0053439AB23B6A1A8061E07B6D5B78012BA6
:10759C005DD17B681B68FB627B681B68B3F850305D
:1075AC009BB21A46FB6A1344FB627B6D1B781A0173
:1075BC00FB6A134403F20443BB62BB6A00221A80C9
:1075CC0045E07B681B68FB637B6D5B78002B26D1E9
:1075DC007B681B687B637B681B68B3F850309BB27D
:1075EC001A467B6B13447B637B6D1B781A017B6B98
:1075FC00134403F20C433B633B6B1B889BB2C3F3FA
:10760C0009039AB23B6B1A803B6B1B889BB26FEAE7
:10761C0043436FEA53439AB23B6B1A8017E07B6D7E
:10762C005B78012B13D17B681B68B3F850309BB28D
:10763C001A46FB6B1344FB637B6D1B781A01FB6BC7
:10764C00134403F20C43BB63BB6B00221A807B6DAB
:10765C001B781946786806F0CCFC53E0B7F84A3032
:10766C0003F48073002B46D17B681B68B3F8503051
:10767C009BB21A467B6D1B78DB00134402335B0014
:10768C007A681268134403F580631B88C3F30903FB
:10769C00A7F840307B6D9A69B7F840309A4207D909
:1076AC007B6D9A69B7F84030D21A7B6D9A6102E013
:1076BC007B6D00229A617B6D9B69002B06D17B6DE3
:1076CC001B781946786806F094FC1BE07B6D5A69B0
:1076DC00B7F840301A447B6D5A617B6DDA69B7F8A4
:1076EC0040301A447B6DDA617B681B68796D1846F3
:1076FC0003F0CCF806E0B7F84A301A46796D786892
:10770C0000F01BF97B681B68B3F844309BB21BB2CA
:10771C00002BFFF63BAC002318465837BD4680BD06
:10772C0080B588B000AFF860B9601346FB80FB8869
:10773C0003F48043002B7ED0FB681B68B3F85030F9
:10774C009BB21A46BB681B78DB00134402335B0008
:10775C00FA681268134403F580631B88C3F30903AA
:10776C007B83BB689A697B8B9A4206D3BB689A6908
:10777C007B8BD21ABB689A6102E0BB6800229A61CB
:10778C00BB689B69002B23D1FB681B681A46BB683E
:10779C001B789B0013441B889BB223F4804323F07B
:1077AC0070033B833B8B83F400533B83FB681B6868
:1077BC001A46BB681B789B001A443B8B43F07F43F3
:1077CC0043F47F0343F4004343F080039BB21380E4
:1077DC00FB8803F04003002B1FD0FB681B681A4684
:1077EC00BB681B789B0013441B889BB223F4E043BB
:1077FC0023F07003FB82FB681B681A46BB681B787E
:10780C009B001A44FB8A43F07F4343F47F0343F409
:10781C00004343F0C0039BB213807B8B002B00F022
:10782C008780FB681868BB685969BB681A897B8BB1
:10783C0004F061FD7CE0FB681B68B3F850309BB230
:10784C001A46BB681B78DB00134406335B00FA68EE
:10785C001268134403F580631B88C3F309037B830D
:10786C00BB689A697B8B9A4206D3BB689A697B8BFF
:10787C00D21ABB689A6102E0BB6800229A61BB68AD
:10788C009B69002B23D1FB681B681A46BB681B78CD
:10789C009B0013441B889BB223F4804323F070039A
:1078AC00FB83FB8B83F40053FB83FB681B681A463A
:1078BC00BB681B789B001A44FB8B43F07F4343F45B
:1078CC007F0343F4004343F080039BB21380FB8897
:1078DC0003F04003002B1FD1FB681B681A46BB68E2
:1078EC001B789B0013441B889BB223F4E04323F0CA
:1078FC007003BB83FB681B681A46BB681B789B0034
:10790C001A44BB8B43F07F4343F47F0343F400439F
:10791C0043F0C0039BB213807B8B002B08D0FB6819
:10792C001868BB685969BB685A897B8B04F0E3FC07
:10793C007B8B18462037BD4680BD80B5A4B000AF08
:10794C00F860B9601346FB80FB8803F04003002B02
:10795C0000F0DD81FB681B68B3F850309BB21A460F
:10796C00BB681B78DB00134402335B00FA681268B7
:10797C00134403F580631B88C3F30903A7F886300F
:10798C00BB689A69B7F886309A4207D9BB689A697E
:10799C00B7F88630D21ABB689A6102E0BB68002245
:1079AC009A61BB689B69002B40F0B980BB685B781F
:1079BC00002B26D1FB681B68FB62FB681B68B3F8C5
:1079CC0050309BB21A46FB6A1344FB62BB681B78AF
:1079DC001A01FB6A134403F20443BB62BB6A1B88A3
:1079EC009BB2C3F309039AB2BB6A1A80BB6A1B88A9
:1079FC009BB26FEA43436FEA53439AB2BB6A1A8055
:107A0C001AE0BB685B78012B16D1FB681B687B63A3
:107A1C00FB681B68B3F850309BB21A467B6B13445F
:107A2C007B63BB681B781A017B6B134403F2044322
:107A3C003B633B6B00221A80FB681B687B62BB6854
:107A4C005B78002B26D1FB681B68FB61FB681B680D
:107A5C00B3F850309BB21A46FB691344FB61BB6808
:107A6C001B781A01FB69134403F20C43BB61BB691D
:107A7C001B889BB2C3F309039AB2BB691A80BB691A
:107A8C001B889BB26FEA43436FEA53439AB2BB69BC
:107A9C001A8017E0BB685B78012B13D1FB681B685D
:107AAC00B3F850309BB21A467B6A13447B62BB68B6
:107ABC001B781A017B6A134403F20C433B623B6A4A
:107ACC0000221A80BB681B781946F86806F091FAF8
:107ADC00FB8803F48043002B00F0FC82FB681B68DE
:107AEC001A46BB681B789B0013441B889BB223F47B
:107AFC00E04323F07003FB82FB681B681A46BB68EB
:107B0C001B789B001A44FB8A43F07F4343F47F03AA
:107B1C0043F4404343F080039BB21380DAE2FB88CA
:107B2C0003F48043002B21D0FB681B681A46BB680A
:107B3C001B789B0013441B889BB223F4E04323F077
:107B4C007003A7F88A30FB681B681A46BB681B7861
:107B5C009B001A44B7F88A3043F07F4343F47F0309
:107B6C0043F4404343F080039BB21380BB6893F80B
:107B7C002430012B40F0AE82BB685A69B7F88630CE
:107B8C001A44BB685A61BB68DA69B7F886301A4484
:107B9C00BB68DA61BB681A6ABB681B699A420BD373
:107BAC00BB681B69C7F88C30BB681A6AD7F88C3075
:107BBC00D21ABB681A6217E0BB681B6A002B08D18B
:107BCC00B7F88630C7F88C30BB68002283F82420C5
:107BDC000AE0BB68002283F82420BB681B6AC7F844
:107BEC008C30BB6800221A62BB685B78002B65D1B5
:107BFC00FB681B68FB63FB681B68B3F850309BB2D7
:107C0C001A46FB6B1344FB63BB681B781A01FB6BB6
:107C1C00134403F20443BB63BB6B1B889BB2C3F3DB
:107C2C0009039AB2BB6B1A80D7F88C303E2B1DD946
:107C3C00D7F88C305B09BB64D7F88C3003F01F038A
:107C4C00002B02D1BB6C013BBB64BB6B1B889AB293
:107C5C00BB6C9BB29B029BB213439BB26FEA434338
:107C6C006FEA53439AB2BB6B1A8044E0D7F88C305E
:107C7C00002B0AD1BB6B1B889BB26FEA43436FEAA4
:107C8C0053439AB2BB6B1A8035E0D7F88C305B0843
:107C9C00BB64D7F88C3003F00103002B02D0BB6C13
:107CAC000133BB64BB6B1B889AB2BB6C9BB29B024F
:107CBC009BB213439AB2BB6B1A801CE0BB685B7817
:107CCC00012B18D1FB681B687B64FB681B68B3F83D
:107CDC0050309BB21A467B6C13447B64BB681B7898
:107CEC001A017B6C134403F204433B64D7F88C30C9
:107CFC009AB23B6C1A80FB681868BB685969BB6800
:107D0C001A89D7F88C309BB204F0AFFAE2E1FB6829
:107D1C001B68B3F850309BB21A46BB681B78DB006B
:107D2C00134406335B00FA681268134403F580634E
:107D3C001B88C3F30903A7F88630BB689A69B7F8A8
:107D4C0086309A4207D3BB689A69B7F88630D21A44
:107D5C00BB689A6102E0BB6800229A61BB689B69B0
:107D6C00002B40F0C080BB685B78002B26D1FB68F1
:107D7C001B68FB67FB681B68B3F850309BB21A4654
:107D8C00FB6F1344FB67BB681B781A01FB6F134432
:107D9C0003F20443BB67BB6F1B889BB2C3F309039D
:107DAC009AB2BB6F1A80BB6F1B889BB26FEA4343BE
:107DBC006FEA53439AB2BB6F1A801AE0BB685B78C8
:107DCC00012B16D1FB681B687B66FB681B68B3F83C
:107DDC0050309BB21A467B6E13447B66BB681B7893
:107DEC001A017B6E134403F204433B663B6E002284
:107DFC001A80FB681B687B67BB685B78002B2BD1F8
:107E0C00FB681B68FB66FB681B68B3F850309BB2C1
:107E1C001A46FB6E1344FB66BB681B781A01FB6E9B
:107E2C00134403F20C43C7F88030D7F880301B881A
:107E3C009BB2C3F309039AB2D7F880301A80D7F8F3
:107E4C0080301B889BB26FEA43436FEA53439AB26C
:107E5C00D7F880301A8017E0BB685B78012B13D100
:107E6C00FB681B68B3F850309BB21A467B6F134407
:107E7C007B67BB681B781A017B6F134403F20C43BE
:107E8C003B673B6F00221A80BB681B781946F86869
:107E9C0006F0AFF8FB8803F48043002B40F01A8106
:107EAC00FB681B681A46BB681B789B0013441B8835
:107EBC009BB223F4E04323F07003A7F88830FB68EF
:107ECC001B681A46BB681B789B001A44B7F88830AD
:107EDC0043F07F4343F47F0343F4404343F0800378
:107EEC009BB21380F6E0FB8803F48043002B21D176
:107EFC00FB681B681A46BB681B789B0013441B88E5
:107F0C009BB223F4E04323F07003A7F84E30FB68D8
:107F1C001B681A46BB681B789B001A44B7F84E3096
:107F2C0043F07F4343F47F0343F4404343F0800327
:107F3C009BB21380BB6893F82430012B40F0CA80AD
:107F4C00BB685A69B7F886301A44BB685A61BB687B
:107F5C00DA69B7F886301A44BB68DA61BB681A6A0A
:107F6C00BB681B699A420BD3BB681B69C7F88C3082
:107F7C00BB681A6AD7F88C30D21ABB681A6217E041
:107F8C00BB681B6A002B08D1B7F88630C7F88C3059
:107F9C00BB68002283F824200AE0BB681B6AC7F880
:107FAC008C30BB6800221A62BB68002283F8242044
:107FBC00FB681B687B65BB685B78002B65D1FB6835
:107FCC001B68FB65FB681B68B3F850309BB21A4604
:107FDC00FB6D1344FB65BB681B781A01FB6D1344E6
:107FEC0003F20C43BB65BB6D1B889BB2C3F3090347
:107FFC009AB2BB6D1A80D7F88C303E2B1DD9D7F8AE
:10800C008C305B09BB66D7F88C3003F01F03002B58
:10801C0002D1BB6E013BBB66BB6D1B889AB2BB6EBB
:10802C009BB29B029BB213439BB26FEA43436FEA32
:10803C0053439AB2BB6D1A8041E0D7F88C30002BB9
:10804C000AD1BB6D1B889BB26FEA43436FEA534363
:10805C009AB2BB6D1A8032E0D7F88C305B08BB66E5
:10806C00D7F88C3003F00103002B02D0BB6E013328
:10807C00BB66BB6D1B889AB2BB6E9BB29B029BB25C
:10808C0013439AB2BB6D1A8019E0BB685B78012B65
:10809C0015D1FB681B68B3F850309BB21A467B6D48
:1080AC0013447B65BB681B781A017B6D134403F288
:1080BC000C433B65D7F88C309AB23B6D1A80FB6849
:1080CC001868BB685969BB685A89D7F88C309BB261
:1080DC0004F0CBF8FB681B681A46BB681B789B0046
:1080EC0013441B889BB223F4E04323F04003BB8270
:1080FC00BB8A83F01003BB82BB8A83F02003BB8254
:10810C00FB681B681A46BB681B789B001A44BB8A29
:10811C0043F07F4343F47F0343F4004343F0800375
:10812C009BB21380002318469037BD4680BD80B4A7
:10813C0087B000AFF8607B600B467B8113463B81B8
:10814C007B8903F080039BB2002B0BD07B8903F05F
:10815C00070213469B001344DB001033FA681344E8
:10816C007B6109E07A8913469B001344DB0003F51D
:10817C00A873FA6813447B613B89002B07D17B6998
:10818C0000221A737B689AB27B69DA800BE07B69F8
:10819C0001221A737B689AB27B691A817B681B0C6B
:1081AC009AB27B695A81002318461C37BD4680BCA5
:1081BC007047000080B586B000AF78607B68002BFC
:1081CC0001D1012372E27B681B6803F00103002BD1
:1081DC0000F08780924B5B6803F00C03042B0CD0EF
:1081EC008F4B5B6803F00C03082B12D18C4B5B6834
:1081FC0003F48033B3F5803F0BD1894B1B6803F438
:10820C000033002B6CD07B685B68002B68D101239A
:10821C004CE27B685B68B3F5803F06D1804B1B68F2
:10822C007F4A43F4803313602EE07B685B68002B3D
:10823C000CD17B4B1B687A4A23F480331360784B48
:10824C001B68774A23F4802313601DE07B685B680E
:10825C00B3F5A02F0CD1724B1B68714A43F48023E9
:10826C0013606F4B1B686E4A43F4803313600BE052
:10827C006B4B1B686A4A23F480331360684B1B6892
:10828C00674A23F4802313607B685B68002B13D050
:10829C00FCF7A4FF386108E0FCF7A0FF02463B693D
:1082AC00D31A642B01D9032300E25D4B1B6803F442
:1082BC000033002BF0D014E0FCF790FF386108E09D
:1082CC00FCF78CFF02463B69D31A642B01D90323BC
:1082DC00ECE1534B1B6803F40033002BF0D100E0AE
:1082EC0000BF7B681B6803F00203002B63D04C4B70
:1082FC005B6803F00C03002B0BD0494B5B6803F05D
:10830C000C03082B1CD1464B5B6803F48033002B09
:10831C0016D1434B1B6803F00203002B05D07B687E
:10832C001B69012B01D00123C0E13D4B1B6823F0DD
:10833C00F8027B685B69DB00394913430B603AE058
:10834C007B681B69002B20D0364B01221A60FCF78E
:10835C0045FF386108E0FCF741FF02463B69D31A40
:10836C00022B01D90323A1E12D4B1B6803F002035F
:10837C00002BF0D02A4B1B6823F0F8027B685B695A
:10838C00DB00274913430B6015E0264B00221A60D3
:10839C00FCF724FF386108E0FCF720FF02463B693C
:1083AC00D31A022B01D9032380E11D4B1B6803F068
:1083BC000203002BF0D17B681B6803F00803002B31
:1083CC003AD07B689B69002B19D0174B01221A609D
:1083DC00FCF704FF386108E0FCF700FF02463B693C
:1083EC00D31A022B01D9032360E10D4B5B6A03F016
:1083FC000203002BF0D0012000F0D0FA1CE00A4B55
:10840C0000221A60FCF7EAFE38610FE0FCF7E6FE8A
:10841C0002463B69D31A022B08D9032346E100BF5D
:10842C00001002400000424280044242924B5B6AC0
:10843C0003F00203002BE9D17B681B6803F00403F3
:10844C00002B00F0A6800023FB758B4BDB6903F03F
:10845C008053002B0DD1884BDB69874A43F0805346
:10846C00D361854BDB6903F08053BB60BB68012390
:10847C00FB75824B1B6803F48073002B18D17F4B68
:10848C001B687E4A43F480731360FCF7A7FE3861C7
:10849C0008E0FCF7A3FE02463B69D31A642B01D912
:1084AC00032303E1754B1B6803F48073002BF0D09E
:1084BC007B68DB68012B06D16F4B1B6A6E4A43F05D
:1084CC00010313622DE07B68DB68002B0CD16A4B37
:1084DC001B6A694A23F001031362674B1B6A664AE5
:1084EC0023F0040313621CE07B68DB68052B0CD1C2
:1084FC00614B1B6A604A43F0040313625E4B1B6AB8
:10850C005D4A43F0010313620BE05B4B1B6A5A4A52
:10851C0023F001031362584B1B6A574A23F00403E0
:10852C0013627B68DB68002B15D0FCF757FE3861B3
:10853C000AE0FCF753FE02463B69D31A41F288323B
:10854C00934201D90323B1E04B4B1B6A03F00203A6
:10855C00002BEED014E0FCF741FE38610AE0FCF78A
:10856C003DFE02463B69D31A41F28832934201D94F
:10857C0003239BE0404B1B6A03F00203002BEED15C
:10858C00FB7D012B05D13C4BDB693B4A23F080532F
:10859C00D3617B68DB69002B00F08780364B5B680E
:1085AC0003F00C03082B61D07B68DB69022B46D1EE
:1085BC00334B00221A60FCF711FE386108E0FCF71F
:1085CC000DFE02463B69D31A022B01D903236DE041
:1085DC00294B1B6803F00073002BF0D17B681B6ADE
:1085EC00B3F5803F08D1244B5B6823F400327B68E1
:1085FC009B68214913434B601F4B5B6823F4741237
:10860C007B68196A7B685B6A0B431B4913434B609D
:10861C001B4B01221A60FCF7E1FD386108E0FCF706
:10862C00DDFD02463B69D31A022B01D903233DE041
:10863C00114B1B6803F00073002BF0D035E0104B8E
:10864C0000221A60FCF7CAFD386108E0FCF7C6FD91
:10865C0002463B69D31A022B01D9032326E0064BB1
:10866C001B6803F00073002BF0D11EE07B68DB6904
:10867C00012B07D1012319E00010024000700040CB
:10868C00600042420B4B5B68FB60FB6803F480327A
:10869C007B681B6A9A4206D1FB6803F470127B68F4
:1086AC005B6A9A4201D0012300E000231846183778
:1086BC00BD4680BD0010024080B584B000AF78602C
:1086CC0039607B68002B01D10123D0E06A4B1B6819
:1086DC0003F007033A689A4210D9674B1B6823F0E2
:1086EC00070265493B6813430B60634B1B6803F03F
:1086FC0007033A689A4201D00123B8E07B681B68F3
:10870C0003F00203002B20D07B681B6803F00403EA
:10871C00002B05D0594B5B68584A43F4E063536017
:10872C007B681B6803F00803002B05D0534B5B6878
:10873C00524A43F460535360504B5B6823F0F00291
:10874C007B689B684D4913434B607B681B6803F047
:10875C000103002B40D07B685B68012B07D1474B92
:10876C001B6803F40033002B15D101237FE07B68D9
:10877C005B68022B07D1414B1B6803F00073002B85
:10878C0009D1012373E03D4B1B6803F00203002B5E
:10879C0001D101236BE0394B5B6823F003027B684A
:1087AC005B68364913434B60FCF718FDF8600AE030
:1087BC00FCF714FD0246FB68D31A41F2883293424F
:1087CC0001D9032353E02D4B5B6803F00C027B684B
:1087DC005B689B009A42EBD1274B1B6803F00703A5
:1087EC003A689A4210D2244B1B6823F007022249A4
:1087FC003B6813430B60204B1B6803F007033A687C
:10880C009A4201D0012332E07B681B6803F0040319
:10881C00002B08D0194B5B6823F4E0627B68DB68A3
:10882C00164913434B607B681B6803F00803002B4D
:10883C0009D0124B5B6823F460527B681B69DB0028
:10884C000E4913434B6000F021F802460B4B5B685A
:10885C001B0903F00F030A49CB5C22FA03F3094A04
:10886C001360094B1B681846FCF776FC002318466E
:10887C001037BD4680BD00BF0020024000100240F2
:10888C00B0F50008100000201400002080B487B060
:10889C0000AF0023FB600023BB6000237B6100233F
:1088AC007B6000233B611E4B5B68FB60FB6803F045
:1088BC000C03042B02D0082B03D027E0194B3B618F
:1088CC0027E0FB689B0C03F00F03174AD35C7B601B
:1088DC00FB6803F48033002B10D0114B5B685B0CEE
:1088EC0003F00103114AD35CBB607B680D4A03FBA8
:1088FC0002F2BB68B2FBF3F37B6104E07B680C4AC9
:10890C0002FB03F37B617B693B6102E0094B3B613A
:10891C0000BF3B6918461C37BD4680BC704700BF82
:10892C0000100240001BB700C8F50008D8F500087D
:10893C0000093D0000127A0080B400AF024B1B68A6
:10894C001846BD4680BC70471000002080B500AFB3
:10895C00FFF7F2FF0246054B5B681B0A03F00703A7
:10896C000349CB5C22FA03F3184680BD0010024089
:10897C00C0F5000880B500AFFFF7DEFF0246054BDF
:10898C005B68DB0A03F007030349CB5C22FA03F3B1
:10899C00184680BD00100240C0F5000880B485B0B8
:1089AC0000AF78600A4B1B680A4AA2FB03235B0AE0
:1089BC007A6802FB03F3FB6000BFFB685A1EFA6087
:1089CC00002BF9D100BF00BF1437BD4680BC7047E7
:1089DC0010000020D34D621080B586B000AF7860D7
:1089EC0000233B610023FB607B681B6803F00103E1
:1089FC00002B7DD00023FB754F4BDB6903F08053BC
:108A0C00002B0DD14C4BDB694B4A43F08053D361A7
:108A1C00494BDB6903F08053BB60BB680123FB75DA
:108A2C00464B1B6803F48073002B18D1434B1B6817
:108A3C00424A43F480731360FCF7D0FB386108E0C2
:108A4C00FCF7CCFB02463B69D31A642B01D90323F8
:108A5C006DE03A4B1B6803F48073002BF0D0364B5F
:108A6C001B6A03F44073FB60FB68002B2ED07B6801
:108A7C005B6803F44073FA689A4227D02E4B1B6A4A
:108A8C0023F44073FB602E4B01221A602C4B002206
:108A9C001A60294AFB681362FB6803F00103002B80
:108AAC0014D0FCF79BFB38610AE0FCF797FB0246FD
:108ABC003B69D31A41F28832934201D9032336E041
:108ACC001D4B1B6A03F00203002BEED01A4B1B6AE2
:108ADC0023F440727B685B68174913430B62FB7D80
:108AEC00012B05D1144BDB69134A23F08053D3615E
:108AFC007B681B6803F00203002B08D00E4B5B68ED
:108B0C0023F440427B689B680B4913434B607B68A2
:108B1C001B6803F01003002B08D0074B5B6823F491
:108B2C0080027B68DB68044913434B6000231846C2
:108B3C001837BD4680BD00BF0010024000700040D9
:108B4C004004424280B582B000AF78607B68002B55
:108B5C0001D1012341E07B6893F83D30DBB2002B5F
:108B6C0006D17B68002283F83C207868FCF76AF910
:108B7C007B68022283F83D207B681A687B6804338B
:108B8C001946104600F03EFB7B68012283F8462014
:108B9C007B68012283F83E207B68012283F83F200A
:108BAC007B68012283F840207B68012283F84120F6
:108BBC007B68012283F842207B68012283F84320E2
:108BCC007B68012283F844207B68012283F84520CE
:108BDC007B68012283F83D20002318460837BD46E8
:108BEC0080BD80B582B000AF78607B68002B01D16E
:108BFC00012341E07B6893F83D30DBB2002B06D1BA
:108C0C007B68002283F83C20786800F039F87B6898
:108C1C00022283F83D207B681A687B68043319466E
:108C2C00104600F0EFFA7B68012283F846207B683F
:108C3C00012283F83E207B68012283F83F207B6869
:108C4C00012283F840207B68012283F841207B6855
:108C5C00012283F842207B68012283F843207B6841
:108C6C00012283F844207B68012283F845207B682D
:108C7C00012283F83D20002318460837BD4680BDED
:108C8C0080B483B000AF786000BF0C37BD4680BCA9
:108C9C007047000080B584B000AF786039603B68E5
:108CAC00002B09D17B6893F83E30DBB2012B14BF4B
:108CBC0001230023DBB222E03B68042B09D17B6843
:108CCC0093F83F30DBB2012B14BF01230023DBB23E
:108CDC0015E03B68082B09D17B6893F84030DBB278
:108CEC00012B14BF01230023DBB208E07B6893F84F
:108CFC004130DBB2012B14BF01230023DBB2002B6C
:108D0C0001D001235EE03B68002B04D17B6802227A
:108D1C0083F83E2013E03B68042B04D17B680222CD
:108D2C0083F83F200BE03B68082B04D17B680222C0
:108D3C0083F8402003E07B68022283F841207B68A3
:108D4C001B6801223968184600F0E8FC7B681B6838
:108D5C001E4A934207D17B681B685A6C7B681B6860
:108D6C0042F400425A647B681B68184A93420ED046
:108D7C007B681B68B3F1804F09D07B681B68144A71
:108D8C00934204D07B681B68124A934211D17B68D2
:108D9C001B689B6803F00703FB60FB68062B10D075
:108DAC007B681B681A687B681B6842F001021A60BA
:108DBC0007E07B681B681A687B681B6842F001023D
:108DCC001A60002318461037BD4680BD002C0140A8
:108DDC00000400400008004080B582B000AF78600D
:108DEC0039607B681B6800223968184600F096FCD5
:108DFC007B681B68294A934217D17B681B681A6AE7
:108E0C0041F211131340002B0FD17B681B681A6AB7
:108E1C0040F244431340002B07D17B681B685A6C0B
:108E2C007B681B6822F400425A647B681B681A6AD0
:108E3C0041F211131340002B0FD17B681B681A6A87
:108E4C0040F244431340002B07D17B681B681A681F
:108E5C007B681B6822F001021A603B68002B04D16E
:108E6C007B68012283F83E2013E03B68042B04D17D
:108E7C007B68012283F83F200BE03B68082B04D170
:108E8C007B68012283F8402003E07B68012283F891
:108E9C004120002318460837BD4680BD002C0140F8
:108EAC0080B586B000AFF860B9607A600023FB75BE
:108EBC00FB6893F83C30012B01D10223AEE0FB6838
:108ECC00012283F83C207B680C2B00F29F8001A2CE
:108EDC0052F823F0158F000819900008199000081B
:108EEC0019900008558F0008199000081990000877
:108EFC0019900008978F0008199000081990000825
:108F0C0019900008D78F0008FB681B68B9681846D1
:108F1C0000F0E6F9FB681B689A69FB681B6842F075
:108F2C0008029A61FB681B689A69FB681B6822F04F
:108F3C0004029A61FB681B689969BB681A69FB6833
:108F4C001B680A439A6164E0FB681B68B9681846A1
:108F5C0000F02CFAFB681B689A69FB681B6842F4EA
:108F6C0000629A61FB681B689A69FB681B6822F4B3
:108F7C0080629A61FB681B689969BB681B691A025D
:108F8C00FB681B680A439A6143E0FB681B68B9687D
:108F9C00184600F075FAFB681B68DA69FB681B68F9
:108FAC0042F00802DA61FB681B68DA69FB681B682F
:108FBC0022F00402DA61FB681B68D969BB681A6984
:108FCC00FB681B680A43DA6123E0FB681B68B9681D
:108FDC00184600F0BFFAFB681B68DA69FB681B686F
:108FEC0042F40062DA61FB681B68DA69FB681B6893
:108FFC0022F48062DA61FB681B68D969BB681B6963
:10900C001A02FB681B680A43DA6102E00123FB7554
:10901C0000BFFB68002283F83C20FB7D1846183704
:10902C00BD4680BD80B584B000AF78603960002348
:10903C00FB737B6893F83C30012B01D10223B4E025
:10904C007B68012283F83C207B68022283F83D2058
:10905C007B681B689B68BB60BB6823F07703BB60B5
:10906C00BB6823F47F43BB607B681B68BA689A605B
:10907C003B681B68B3F5005F3ED0B3F5005F00F2B0
:10908C008780B3F5805F00F08680B3F5805F7FD872
:10909C00702B1AD0702B7BD8602B50D0602B77D8CC
:1090AC00502B3CD0502B73D8402B58D0402B6FD822
:1090BC00302B64D0302B6BD8202B60D0202B67D872
:1090CC00002B5CD0102B5AD062E07B6818683B6890
:1090DC0099683B685A683B68DB6800F000FB7B686A
:1090EC001B689B68BB60BB6843F07703BB607B6805
:1090FC001B68BA689A604FE07B6818683B6899688F
:10910C003B685A683B68DB6800F0E9FA7B681B68CF
:10911C009A687B681B6842F480429A603CE07B68EA
:10912C0018683B6859683B68DB681A4600F060FABF
:10913C007B681B685021184600F0B7FA2CE07B685E
:10914C0018683B6859683B68DB681A4600F07EFA81
:10915C007B681B686021184600F0A7FA1CE07B684E
:10916C0018683B6859683B68DB681A4600F040FA9F
:10917C007B681B684021184600F097FA0CE07B686E
:10918C001A683B681B681946104600F08EFA03E01B
:10919C000123FB7300E000BF7B68012283F83D20B4
:1091AC007B68002283F83C20FB7B18461037BD46B9
:1091BC0080BD80B485B000AF786039603B68002B0F
:1091CC0004D17B6893F83E30DBB213E03B68042B90
:1091DC0004D17B6893F83F30DBB20BE03B68082B83
:1091EC0004D17B6893F84030DBB203E07B6893F8E2
:1091FC004130DBB2FB73FB7B18461437BD4680BC99
:10920C007047000080B485B000AF786039607B682F
:10921C001B68FB607B682F4A93420BD07B68B3F1D1
:10922C00804F07D07B682C4A934203D07B682B4A33
:10923C00934208D1FB6823F07003FB603B685B68CA
:10924C00FA681343FB607B68224A93420BD07B681D
:10925C00B3F1804F07D07B681F4A934203D07B68E1
:10926C001E4A934208D1FB6823F44073FB603B68B1
:10927C00DB68FA681343FB60FB6823F080023B68F1
:10928C005B691343FB607B68FA681A603B689A68F9
:10929C007B68DA623B681A687B689A627B680D4A65
:1092AC00934203D13B681A697B681A637B6801227D
:1092BC005A617B681B6903F00103002B05D07B68A6
:1092CC001B6923F001027B681A6100BF1437BD468D
:1092DC0080BC7047002C0140000400400008004096
:1092EC0080B487B000AF786039607B681B6A7B61A3
:1092FC007B681B6A23F001027B681A627B685B68DF
:10930C003B617B689B69FB60FB6823F07003FB602F
:10931C00FB6823F00303FB603B681B68FA6813438C
:10932C00FB607B6923F002037B613B689B687A6975
:10933C0013437B617B681C4A93420CD17B6923F0FD
:10934C0008037B613B68DB687A6913437B617B694B
:10935C0023F004037B617B68134A934211D13B6970
:10936C0023F480733B613B6923F400733B613B68DE
:10937C005B693A6913433B613B689B693A691343E8
:10938C003B617B683A695A607B68FA689A613B6812
:10939C005A687B685A637B687A691A6200BF1C370B
:1093AC00BD4680BC704700BF002C014080B487B024
:1093BC0000AF786039607B681B6A7B617B681B6AD5
:1093CC0023F010027B681A627B685B683B617B68E8
:1093DC009B69FB60FB6823F4E043FB60FB6823F4B0
:1093EC004073FB603B681B681B02FA681343FB600D
:1093FC007B6923F020037B613B689B681B017A69C6
:10940C0013437B617B681D4A93420DD17B6923F02A
:10941C0080037B613B68DB681B017A6913437B61CA
:10942C007B6923F040037B617B68144A934213D120
:10943C003B6923F480633B613B6923F400633B612C
:10944C003B685B699B003A6913433B613B689B69D2
:10945C009B003A6913433B617B683A695A607B68AD
:10946C00FA689A613B685A687B689A637B687A6988
:10947C001A6200BF1C37BD4680BC7047002C0140EF
:10948C0080B487B000AF786039607B681B6A7B6101
:10949C007B681B6A23F480727B681A627B685B684A
:1094AC003B617B68DB69FB60FB6823F07003FB604E
:1094BC00FB6823F00303FB603B681B68FA681343EB
:1094CC00FB607B6923F400737B613B689B681B0228
:1094DC007A6913437B617B681D4A93420DD17B698A
:1094EC0023F400637B613B68DB681B027A691343DE
:1094FC007B617B6923F480637B617B68144A9342B4
:10950C0013D13B6923F480533B613B6923F4005333
:10951C003B613B685B691B013A6913433B613B68E8
:10952C009B691B013A6913433B617B683A695A603A
:10953C007B68FA68DA613B685A687B68DA637B6837
:10954C007A691A6200BF1C37BD4680BC704700BFE9
:10955C00002C014080B487B000AF786039607B6824
:10956C001B6A3B617B681B6A23F480527B681A621E
:10957C007B685B687B617B68DB69FB60FB6823F461
:10958C00E043FB60FB6823F44073FB603B681B68A3
:10959C001B02FA681343FB603B6923F400533B61E5
:1095AC003B689B681B033A6913433B617B680F4A1A
:1095BC00934209D17B6923F480437B613B685B69EF
:1095CC009B017A6913437B617B687A695A607B687B
:1095DC00FA68DA613B685A687B681A647B683A6996
:1095EC001A6200BF1C37BD4680BC7047002C01407E
:1095FC0080B487B000AFF860B9607A60FB681B6A12
:10960C007B61FB681B6A23F00102FB681A62FB6832
:10961C009B693B613B6923F0F0033B617B681B0159
:10962C003A6913433B617B6923F00A037B617A69D6
:10963C00BB6813437B61FB683A699A61FB687A6982
:10964C001A6200BF1C37BD4680BC704780B487B01F
:10965C0000AFF860B9607A60FB681B6A7B61FB68DD
:10966C001B6A23F01002FB681A62FB689B693B6162
:10967C003B6923F470433B617B681B033A691343DA
:10968C003B617B6923F0A0037B61BB681B017A699A
:10969C0013437B61FB683A699A61FB687A691A62C9
:1096AC0000BF1C37BD4680BC704780B485B000AF8E
:1096BC00786039607B689B68FB60FB6823F0700303
:1096CC00FB603A68FB68134343F00703FB607B685D
:1096DC00FA689A6000BF1437BD4680BC704780B4EE
:1096EC0087B000AFF860B9607A603B60FB689B683C
:1096FC007B617B6923F47F437B613B681A027B6847
:10970C001A43BB6813437A6913437B61FB687A691C
:10971C009A6000BF1C37BD4680BC704780B487B0D0
:10972C0000AFF860B9607A60BB6803F01F030122D8
:10973C0002FA03F37B61FB681A6A7B69DB431A400C
:10974C00FB681A62FB681A6ABB6803F01F0379682E
:10975C0001FA03F31A43FB681A6200BF1C37BD46BB
:10976C0080BC704780B485B000AF786039607B688E
:10977C0093F83C30012B01D1022346E07B68012297
:10978C0083F83C207B68022283F83D207B681B68B1
:10979C005B68FB607B681B689B68BB60FB6823F0A5
:1097AC007003FB603B681B68FA681343FB607B68C3
:1097BC001B68FA685A607B681B68164A93420ED085
:1097CC007B681B68B3F1804F09D07B681B68124A19
:1097DC00934204D07B681B68104A93420CD1BB683F
:1097EC0023F08003BB603B685B68BA681343BB60C3
:1097FC007B681B68BA689A607B68012283F83D20FD
:10980C007B68002283F83C20002318461437BD46A1
:10981C0080BC7047002C0140000400400008004050
:10982C0080B582B000AF78607B68002B01D101233A
:10983C0042E07B6893F84130DBB2002B06D17B68A9
:10984C00002283F840207868FBF780FB7B68242299
:10985C0083F841207B681B68DA687B681B6822F4FC
:10986C000052DA60786800F071F97B681B681A693D
:10987C007B681B6822F490421A617B681B685A69EA
:10988C007B681B6822F02A025A617B681B68DA68C5
:10989C007B681B6842F40052DA607B6800225A64D1
:1098AC007B68202283F841207B68202283F84220A9
:1098BC007B6800225A63002318460837BD4680BDDA
:1098CC0080B58AB002AFF860B9603B601346FB808C
:1098DC0000237B61FB6893F84130DBB2202B75D100
:1098EC00BB68002B02D0FB88002B01D101236EE05A
:1098FC00FB6800225A64FB68212283F84120FBF7A5
:10990C006DFC7861FB68FA889A84FB68FA88DA84C3
:10991C00FB689B68B3F5805F08D1FB681B69002B63
:10992C0004D10023FB61BB68BB6103E0BB68FB6136
:10993C000023BB612EE03B6800937B6900228021F1
:10994C00F86800F048F80346002B05D0FB6820228D
:10995C0083F8412003233AE0FB69002B0BD1BB6950
:10996C001B881A46FB681B68C2F308025A60BB6965
:10997C000233BB6107E0FB691A78FB681B685A600D
:10998C00FB690133FB61FB68DB8C9BB2013B9AB238
:10999C00FB68DA84FB68DB8C9BB2002BCBD13B6879
:1099AC0000937B6900224021F86800F014F803460C
:1099BC00002B05D0FB68202283F84120032306E00E
:1099CC00FB68202283F84120002300E00223184684
:1099DC002037BD4680BD80B586B000AFF860B96059
:1099EC003B601346FB713BE03B6AB3F1FF3F37D062
:1099FC00FBF7F4FB02463B68D31A3A6A9A4202D34D
:109A0C003B6A002B01D103233AE0FB681B68DB683F
:109A1C0003F00403002B23D0BB68802B20D0BB6841
:109A2C00402B1DD0FB681B681B6803F00803082B38
:109A3C0016D100237B61FB681B681B687B61FB688C
:109A4C001B685B687B617B69F86800F01DF8FB683C
:109A5C0008225A64FB68002283F8402001230FE09F
:109A6C00FB681B681A68BB681340BA689A420CBF43
:109A7C0001230023DBB21A46FB799A42B4D00023AF
:109A8C0018461837BD4680BD80B495B000AF7860DD
:109A9C007B681B680C337B637B6B53E8003F3B6339
:109AAC003B6B23F49073FB647B681B680C33FA6C80
:109ABC003A64FB63F96B3A6C41E80023BB63BB6B04
:109ACC00002BE5D17B681B6814333B623B6A53E87F
:109ADC00003FFB61FB6923F00103BB647B681B68DF
:109AEC001433BA6CFA62BB62B96AFA6A41E80023B1
:109AFC007B627B6A002BE5D17B681B6B012B19D138
:109B0C007B681B680C33FB60FB6853E8003FBB6051
:109B1C00BB6823F010037B647B681B680C337A6C86
:109B2C00BA617B617969BA6941E800233B613B69A1
:109B3C00002BE5D17B68202283F842207B68002231
:109B4C001A6300BF5437BD4680BC704780B584B0E3
:109B5C0000AF78607B681B681B6923F440517B68FD
:109B6C00DA687B681B680A431A617B689A687B68B1
:109B7C001B691A437B685B691343BB607B681B687A
:109B8C00DB6823F4B05323F00C037A681268B968CD
:109B9C000B43D3607B681B685B6923F440717B6863
:109BAC009A697B681B680A435A617B681B682C4A5C
:109BBC00934203D1FEF7DEFEF86002E0FEF7C6FE2C
:109BCC00F860FA6813469B0013449A001A447B68A9
:109BDC005B689B00B2FBF3F3224AA2FB03235B09F5
:109BEC001901FA6813469B0013449A001A447B68C7
:109BFC005B689B00B2FBF3F21A4BA3FB02035B09FD
:109C0C00642000FB03F3D31A1B013233154AA2FB69
:109C1C0003235B0903F0F0031944FA6813469B0015
:109C2C0013449A001A447B685B689B00B2FBF3F206
:109C3C000C4BA3FB02035B09642000FB03F3D31A58
:109C4C001B013233074AA2FB03235B0903F00F020B
:109C5C007B681B680A449A6000BF1037BD4680BD04
:109C6C00003801401F85EB5180B485B000AFF8601F
:109C7C00384680E80E00002318461437BD4680BCD9
:109C8C00704780B485B000AF78607B680022A3F881
:109C9C0044204FF43F43FB60FB689AB27B68A3F807
:109CAC004020002318461437BD4680BC704780B452
:109CBC0085B000AF78604FF43F43FB607B68B3F82E
:109CCC0040309AB2FB689BB2DB439BB213409AB212
:109CDC007B68A3F84020002318461437BD4680BC8F
:109CEC00704780B483B000AF78600B46FB700023E4
:109CFC0018460C37BD4680BC704780B485B000AFA9
:109D0C00F860384680E80E00FB680122A3F840207A
:109D1C00FB680022A3F84020FB680022A3F8442033
:109D2C00FB680022A3F85020002318461437BD46C8
:109D3C0080BC704780B49DB000AF78603960002360
:109D4C0087F86F307A683B681B789B0013441B883C
:109D5C009BB223F4EC4323F07003A7F86C303B6800
:109D6C00DB78032B1FD801A252F823F0899D000841
:109D7C00A59D0008BB9D0008979D0008B7F86C30A6
:109D8C0043F40073A7F86C3012E0B7F86C3043F46E
:109D9C00C063A7F86C300BE0B7F86C3043F4806309
:109DAC00A7F86C3004E0012387F86F3000E000BFA7
:109DBC007A683B681B789B001A44B7F86C3043F008
:109DCC007F4343F47F0343F4004343F080039BB28F
:109DDC0013807A683B681B789B0013441B889BB2EA
:109DEC0023F4E04323F070039BB23A6812781343D8
:109DFC00A7F866307A683B681B789B001A44B7F862
:109E0C00663043F07F4343F47F0343F4004343F055
:109E1C0080039BB213803B681B7B002B40F0788146
:109E2C003B685B78002B00F084807B68BB617B68AF
:109E3C00B3F850309BB21A46BB691344BB613B6804
:109E4C001B781A01BB69134403F580637B613B6883
:109E5C00DB885B089BB25B009AB27B691A807A68DC
:109E6C003B681B789B0013441B887B827B8A03F026
:109E7C004003002B1BD07A683B681B789B00134473
:109E8C001B889BB223F4E04323F070033B827A6877
:109E9C003B681B789B001A443B8A43F07F4343F496
:109EAC007F0343F4004343F0C0039BB213803B6831
:109EBC00DB78012B20D07A683B681B789B0013441D
:109ECC001B889BB223F4E04323F04003BB81BB8986
:109EDC0083F02003BB817A683B681B789B001A4493
:109EEC00BB8943F07F4343F47F0343F4004343F0C7
:109EFC0080039BB21380D5E27A683B681B789B0089
:109F0C0013441B889BB223F4E04323F04003FB81F2
:109F1C007A683B681B789B001A44FB8943F07F43AB
:109F2C0043F47F0343F4004343F080039BB213805C
:109F3C00B8E27B683B637B68B3F850309BB21A463F
:109F4C003B6B13443B633B681B781A013B6B13441C
:109F5C0003F58163FB623B68DB885B089BB25B00AB
:109F6C009AB2FB6A1A807B68BB627B68B3F850308C
:109F7C009BB21A46BB6A1344BB623B681B781A013E
:109F8C00BB6A134403F20C437B627B6A1B889BB253
:109F9C00C3F309039AB27B6A1A803B681B693E2B98
:109FAC001DD93B681B695B09BB663B681B6903F0E9
:109FBC001F03002B02D1BB6E013BBB667B6A1B8867
:109FCC009AB2BB6E9BB29B029BB213439BB26FEADD
:109FDC0043436FEA53439AB27B6A1A8026E03B688C
:109FEC001B69002B0AD17B6A1B889BB26FEA434327
:109FFC006FEA53439AB27B6A1A8017E03B681B697D
:10A00C005B08BB663B681B6903F00103002B02D0A5
:10A01C00BB6E0133BB667B6A1B889AB2BB6E9BB26C
:10A02C009B029BB213439AB27B6A1A807A683B6894
:10A03C001B789B0013441B887B847B8C03F480432C
:10A04C00002B1BD07A683B681B789B0013441B8841
:10A05C009BB223F4E04323F070033B847A683B68A3
:10A06C001B789B001A443B8C43F07F4343F47F03E3
:10A07C0043F4404343F080039BB213803B681B784E
:10A08C00002B24D17A683B681B789B0013441B88F7
:10A09C009BB223F4804323F07003BB83BB8B83F40C
:10A0AC008053BB83BB8B83F40053BB837A683B68C0
:10A0BC001B789B001A44BB8B43F07F4343F47F0314
:10A0CC0043F4004343F080039BB21380EAE17A68C7
:10A0DC003B681B789B0013441B889BB223F4804382
:10A0EC0023F07003FB83FB8B83F40053FB837A68B0
:10A0FC003B681B789B001A44FB8B43F07F4343F473
:10A10C007F0343F4004343F080039BB21380C9E107
:10A11C003B68DB78022B1ED17A683B681B789B006E
:10A12C0013441B889BB223F4E04323F07003A7F87D
:10A13C0062307A683B681B789B001A44B7F862302F
:10A14C0043F07F4343F47F0343F4014343F0800324
:10A15C009BB213801DE07A683B681B789B0013440C
:10A16C001B889BB223F4E24323F07003A7F86430FE
:10A17C007A683B681B789B001A44B7F8643043F04C
:10A18C007F4343F47F0343F4004343F080039BB2CB
:10A19C0013807B68FB657B68B3F850309BB21A4622
:10A1AC00FB6D1344FB653B681B781A01FB6D134474
:10A1BC0003F58063BB653B681B895B089BB25B0046
:10A1CC009AB2BB6D1A807B687B657B68B3F85030A4
:10A1DC009BB21A467B6D13447B653B681B781A0156
:10A1EC007B6D134403F581633B653B685B895B08BE
:10A1FC009BB25B009AB23B6D1A803B685B78002B7C
:10A20C0040F093807A683B681B789B0013441B8852
:10A21C00A7F84030B7F8403003F48043002B1BD034
:10A22C007A683B681B789B0013441B889BB223F411
:10A23C00E04323F07003FB877A683B681B789B0034
:10A24C001A44FB8F43F07F4343F47F0343F44043B2
:10A25C0043F080039BB213807A683B681B789B00A9
:10A26C0013441B88BB87BB8F03F04003002B1BD010
:10A27C007A683B681B789B0013441B889BB223F4C1
:10A28C00E04323F070037B877A683B681B789B0064
:10A29C001A447B8F43F07F4343F47F0343F4004322
:10A2AC0043F0C0039BB213807A683B681B789B0019
:10A2BC0013441B889BB223F4804323F070033B8729
:10A2CC003B8F83F480533B873B8F83F400533B8756
:10A2DC007A683B681B789B001A443B8F43F07F43A2
:10A2EC0043F47F0343F4004343F080039BB2138099
:10A2FC007A683B681B789B0013441B889BB223F441
:10A30C00E04323F04003FB867A683B681B789B0094
:10A31C001A44FB8E43F07F4343F47F0343F4004322
:10A32C0043F080039BB21380BCE07A683B681B78D7
:10A33C009B0013441B88A7F84E30B7F84E3003F43B
:10A34C008043002B1DD07A683B681B789B0013441C
:10A35C001B889BB223F4E04323F07003A7F84C3026
:10A36C007A683B681B789B001A44B7F84C3043F072
:10A37C007F4343F47F0343F4404343F080039BB299
:10A38C0013807A683B681B789B0013441B88A7F8E2
:10A39C004A30B7F84A3003F04003002B1DD07A68DE
:10A3AC003B681B789B0013441B889BB223F4E0434F
:10A3BC0023F07003A7F848307A683B681B789B0041
:10A3CC001A44B7F8483043F07F4343F47F0343F417
:10A3DC00004343F0C0039BB213803B68DB78012B36
:10A3EC0024D07A683B681B789B0013441B889BB273
:10A3FC0023F4E04323F04003A7F84430B7F844308B
:10A40C0083F02003A7F844307A683B681B789B00E4
:10A41C001A44B7F8443043F07F4343F47F0343F4CA
:10A42C00004343F080039BB213801DE07A683B68C5
:10A43C001B789B0013441B889BB223F4E04323F04E
:10A44C004003A7F846307A683B681B789B001A4497
:10A45C00B7F8463043F07F4343F47F0343F40043A3
:10A46C0043F080039BB213807A683B681B789B0097
:10A47C0013441B889BB223F4804323F07003A7F88A
:10A48C0042307A683B681B789B001A44B7F842301C
:10A49C0043F07F4343F47F0343F4004343F08003D2
:10A4AC009BB2138097F86F3018467437BD4680BC4A
:10A4BC00704700BF80B48DB000AF786039603B68E6
:10A4CC001B7B002B40F08E803B685B78002B44D0CC
:10A4DC007A683B681B789B0013441B88BB81BB8943
:10A4EC0003F04003002B1BD07A683B681B789B0061
:10A4FC0013441B889BB223F4E04323F070037B814D
:10A50C007A683B681B789B001A447B8943F07F4335
:10A51C0043F47F0343F4004343F0C0039BB2138026
:10A52C007A683B681B789B0013441B889BB223F40E
:10A53C00E04323F040033B817A683B681B789B0027
:10A54C001A443B8943F07F4343F47F0343F40043B5
:10A55C0043F080039BB2138092E17A683B681B78CE
:10A56C009B0013441B887B827B8A03F48043002B63
:10A57C001BD07A683B681B789B0013441B889BB2EA
:10A58C0023F4E04323F070033B827A683B681B782A
:10A59C009B001A443B8A43F07F4343F47F0343F40C
:10A5AC00404343F080039BB213807A683B681B786E
:10A5BC009B0013441B889BB223F4804323F070034D
:10A5CC00FB817A683B681B789B001A44FB8943F03B
:10A5DC007F4343F47F0343F4004343F080039BB277
:10A5EC0013804DE13B685B78002B40F0A5807A68C6
:10A5FC003B681B789B0013441B883B843B8C03F407
:10A60C008043002B1BD07A683B681B789B0013445B
:10A61C001B889BB223F4E04323F07003FB837A681E
:10A62C003B681B789B001A44FB8B43F07F4343F43D
:10A63C007F0343F4404343F080039BB213807A685A
:10A64C003B681B789B0013441B88BB83BB8B03F0BC
:10A65C004003002B1BD07A683B681B789B0013448B
:10A66C001B889BB223F4E04323F070037B837A684E
:10A67C003B681B789B001A447B8B43F07F4343F46D
:10A68C007F0343F4004343F0C0039BB213807A680A
:10A69C003B681B789B0013441B889BB223F4E0435C
:10A6AC0023F070033B837A683B681B789B001A4449
:10A6BC003B8B43F07F4343F47F0343F4004343F06D
:10A6CC00C0039BB213807A683B681B789B001344D1
:10A6DC001B889BB223F4804323F07003FB827A68BF
:10A6EC003B681B789B001A44FB8A43F07F4343F47E
:10A6FC007F0343F4004343F080039BB213807A68DA
:10A70C003B681B789B0013441B889BB223F4E043EB
:10A71C0023F04003BB827A683B681B789B001A4489
:10A72C00BB8A43F07F4343F47F0343F4004343F07D
:10A73C0080039BB21380A3E07A683B681B789B0074
:10A74C0013441B88FB85FB8D03F48043002B1BD02B
:10A75C007A683B681B789B0013441B889BB223F4DC
:10A76C00E04323F07003BB857A683B681B789B0041
:10A77C001A44BB8D43F07F4343F47F0343F44043BF
:10A78C0043F080039BB213807A683B681B789B0074
:10A79C0013441B887B857B8D03F04003002B1BD05F
:10A7AC007A683B681B789B0013441B889BB223F48C
:10A7BC00E04323F070033B857A683B681B789B0071
:10A7CC001A443B8D43F07F4343F47F0343F400432F
:10A7DC0043F0C0039BB213807A683B681B789B00E4
:10A7EC0013441B889BB223F4E04323F07003FB84D7
:10A7FC007A683B681B789B001A44FB8C43F07F43C0
:10A80C0043F47F0343F4404343F080039BB2138033
:10A81C007A683B681B789B0013441B889BB223F41B
:10A82C00E04323F04003BB847A683B681B789B00B1
:10A83C001A44BB8C43F07F4343F47F0343F400433F
:10A84C0043F080039BB213807A683B681B789B00B3
:10A85C0013441B889BB223F4804323F070037B8446
:10A86C007A683B681B789B001A447B8C43F07F43CF
:10A87C0043F47F0343F4004343F080039BB2138003
:10A88C00002318463437BD4680BC704780B5C2B033
:10A89C0000AF07F58473A3F58273186007F5847312
:10A8AC00A3F58473196007F58473A3F584731B688F
:10A8BC005B78012B40F0B78607F58473A3F584739E
:10A8CC001B689A6907F58473A3F584731B681B696D
:10A8DC009A4208D907F58473A3F584731B681B6926
:10A8EC00C7F8043107E007F58473A3F584731B687C
:10A8FC009B69C7F8043107F58473A3F584731B684F
:10A90C001B7B002B3AD107F58473A3F584731B686A
:10A91C00596907F58473A3F584731B68DA88D7F833
:10A92C0004319BB207F58470A0F58270006801F0C9
:10A93C009CFC07F58473A3F582731B683B6107F5D8
:10A94C008473A3F582731B68B3F850309BB21A461C
:10A95C003B6913443B6107F58473A3F584731B684F
:10A96C001B781A013B69134403F20443FB60D7F8CC
:10A97C0004319AB2FB681A8000F01FBE07F584738D
:10A98C00A3F584731B68DB78022B40F0628407F517
:10A99C008473A3F584731B681A6A07F58473A3F593
:10A9AC0084731B681B699A4240F2DF8307F584733A
:10A9BC00A3F582731A6807F58473A3F584731B6877
:10A9CC001B789B0013441B889BB223F4E04323F0B9
:10A9DC007003A7F8563007F58473A3F582731A68D1
:10A9EC0007F58473A3F584731B681B789B001A44CA
:10A9FC00B7F8563043F07F4343F47F0343F40143ED
:10AA0C0043F080039BB2138007F58473A3F5847322
:10AA1C001B681A6AD7F80431D21A07F58473A3F5A8
:10AA2C0084731B681A6207F58473A3F582731A6822
:10AA3C0007F58473A3F584731B681B789B00134480
:10AA4C001B889BB203F04003002B00F0C78107F575
:10AA5C008473A3F582731B683B6307F58473A3F5BA
:10AA6C0084731B685B78002B77D107F58473A3F58F
:10AA7C0082731B68BB6207F58473A3F582731B6832
:10AA8C00B3F850309BB21A46BB6A1344BB6207F54D
:10AA9C008473A3F584731B681B781A01BB6A134477
:10AAAC0003F20C437B627B6A1B889BB2C3F30903E2
:10AABC009AB27B6A1A80D7F804313E2B21D9D7F889
:10AACC0004315B09C7F80031D7F8043103F01F03D8
:10AADC00002B04D1D7F80031013BC7F800317B6A59
:10AAEC001B889AB2D7F800319BB29B029BB21343DE
:10AAFC009BB26FEA43436FEA53439AB27B6A1A8064
:10AB0C0050E0D7F80431002B0AD17B6A1B889BB22A
:10AB1C006FEA43436FEA53439AB27B6A1A8041E06F
:10AB2C00D7F804315B08C7F80031D7F8043103F0CB
:10AB3C000103002B04D0D7F800310133C7F80031E2
:10AB4C007B6A1B889AB2D7F800319BB29B029BB2EE
:10AB5C0013439AB27B6A1A8024E007F58473A3F539
:10AB6C0084731B685B78012B1CD107F58473A3F5E8
:10AB7C0082731B68B3F850309BB21A463B6B13447C
:10AB8C003B6307F58473A3F584731B681B781A0168
:10AB9C003B6B134403F20C43FB62D7F804319AB2BB
:10ABAC00FB6A1A8007F58473A3F584731B685B89B1
:10ABBC00A7F8763007F58473A3F584731B6859697D
:10ABCC00D7F804319BB2B7F8762007F58470A0F55E
:10ABDC008270006801F049FB07F58473A3F5847358
:10ABEC001B685A69D7F804311A4407F58473A3F526
:10ABFC0084731B685A6107F58473A3F584731B680F
:10AC0C001A6A07F58473A3F584731B681B699A424F
:10AC1C000FD907F58473A3F584731B681A6AD7F8E8
:10AC2C000431D21A07F58473A3F584731B681A6276
:10AC3C000EE007F58473A3F584731B681B6AC7F8D1
:10AC4C00043107F58473A3F584731B6800221A6220
:10AC5C0007F58473A3F584731B685B78002B77D19D
:10AC6C0007F58473A3F582731B68BB6107F58473C6
:10AC7C00A3F582731B68B3F850309BB21A46BB69BC
:10AC8C001344BB6107F58473A3F584731B681B78AD
:10AC9C001A01BB69134403F204437B617B691B8873
:10ACAC009BB2C3F309039AB27B691A80D7F80431BB
:10ACBC003E2B21D9D7F804315B09C7F8FC30D7F803
:10ACCC00043103F01F03002B04D1D7F8FC30013BF7
:10ACDC00C7F8FC307B691B889AB2D7F8FC309BB262
:10ACEC009B029BB213439BB26FEA43436FEA5343FD
:10ACFC009AB27B691A8056E0D7F80431002B0AD13E
:10AD0C007B691B889BB26FEA43436FEA53439AB249
:10AD1C007B691A8047E0D7F804315B08C7F8FC3030
:10AD2C00D7F8043103F00103002B04D0D7F8FC3022
:10AD3C000133C7F8FC307B691B889AB2D7F8FC301A
:10AD4C009BB29B029BB213439AB27B691A802AE096
:10AD5C0007F58473A3F584731B685B78012B22D1F0
:10AD6C0007F58473A3F582731B683B6207F5847344
:10AD7C00A3F582731B68B3F850309BB21A463B6A3A
:10AD8C0013443B6207F58473A3F584731B681B782B
:10AD9C001A013B6A134403F20443FB61D7F80431F4
:10ADAC009AB2FB691A8007F58473A3F584731B6848
:10ADBC001B89A7F8763007F58473A3F584731B6899
:10ADCC005969D7F804319BB2B7F8762007F584702F
:10ADDC00A0F58270006801F048FAEEE307F5847381
:10ADEC00A3F584731B685B78002B77D107F584730C
:10ADFC00A3F582731B68BB6407F58473A3F5827398
:10AE0C001B68B3F850309BB21A46BB6C1344BB643E
:10AE1C0007F58473A3F584731B681B781A01BB6C4C
:10AE2C00134403F204437B647B6C1B889BB2C3F317
:10AE3C0009039AB27B6C1A80D7F804313E2B21D9C6
:10AE4C00D7F804315B09C7F8F830D7F8043103F0B0
:10AE5C001F03002B04D1D7F8F830013BC7F8F830AA
:10AE6C007B6C1B889AB2D7F8F8309BB29B029BB2D2
:10AE7C0013439BB26FEA43436FEA53439AB27B6C22
:10AE8C001A8056E0D7F80431002B0AD17B6C1B8852
:10AE9C009BB26FEA43436FEA53439AB27B6C1A80BE
:10AEAC0047E0D7F804315B08C7F8F830D7F804311D
:10AEBC0003F00103002B04D0D7F8F8300133C7F8A6
:10AECC00F8307B6C1B889AB2D7F8F8309BB29B0297
:10AEDC009BB213439AB27B6C1A802AE007F58473F9
:10AEEC00A3F584731B685B78012B22D107F584735F
:10AEFC00A3F582731B683B6507F58473A3F5827316
:10AF0C001B68B3F850309BB21A463B6D13443B653B
:10AF1C0007F58473A3F584731B681B781A013B6DCA
:10AF2C00134403F20443FB64D7F804319AB2FB6C6C
:10AF3C001A8007F58473A3F584731B681B89A7F823
:10AF4C00763007F58473A3F584731B685969D7F8B9
:10AF5C0004319BB2B7F8762007F58470A0F58270A7
:10AF6C00006801F082F907F58473A3F584731B68FC
:10AF7C005A69D7F804311A4407F58473A3F584731E
:10AF8C001B685A6107F58473A3F584731B681A6AEE
:10AF9C0007F58473A3F584731B681B699A420FD958
:10AFAC0007F58473A3F584731B681A6AD7F8043108
:10AFBC00D21A07F58473A3F584731B681A620EE02A
:10AFCC0007F58473A3F584731B681B6AC7F80431F7
:10AFDC0007F58473A3F584731B6800221A6207F5C6
:10AFEC008473A3F582731B683B6407F58473A3F524
:10AFFC0084731B685B78002B77D107F58473A3F5FA
:10B00C0082731B68BB6307F58473A3F582731B689B
:10B01C00B3F850309BB21A46BB6B1344BB6307F5B5
:10B02C008473A3F584731B681B781A01BB6B1344E0
:10B03C0003F20C437B637B6B1B889BB2C3F309034A
:10B04C009AB27B6B1A80D7F804313E2B21D9D7F8F2
:10B05C0004315B09C7F8F430D7F8043103F01F034F
:10B06C00002B04D1D7F8F430013BC7F8F4307B6BDC
:10B07C001B889AB2D7F8F4309BB29B029BB2134355
:10B08C009BB26FEA43436FEA53439AB27B6B1A80CD
:10B09C0050E0D7F80431002B0AD17B6B1B889BB294
:10B0AC006FEA43436FEA53439AB27B6B1A8041E0D9
:10B0BC00D7F804315B08C7F8F430D7F8043103F043
:10B0CC000103002B04D0D7F8F4300133C7F8F43067
:10B0DC007B6B1B889AB2D7F8F4309BB29B029BB265
:10B0EC0013439AB27B6B1A8024E007F58473A3F5A3
:10B0FC0084731B685B78012B1CD107F58473A3F553
:10B10C0082731B68B3F850309BB21A463B6C1344E5
:10B11C003B6407F58473A3F584731B681B781A01D1
:10B12C003B6C134403F20C43FB63D7F804319AB223
:10B13C00FB6B1A8007F58473A3F584731B685B891A
:10B14C00A7F8763007F58473A3F584731B685969E7
:10B15C00D7F804319BB2B7F8762007F58470A0F5C8
:10B16C008270006801F081F827E207F58473A3F57B
:10B17C0084731B681B6AC7F8043107F58473A3F545
:10B18C0082731A6807F58473A3F584731B681B78A4
:10B19C009B0013441B889BB223F4E24323F07003FF
:10B1AC00A7F8623007F58473A3F582731A6807F564
:10B1BC008473A3F584731B681B789B001A44B7F83F
:10B1CC00623043F07F4343F47F0343F4004343F086
:10B1DC0080039BB2138007F58473A3F582731B68FD
:10B1EC00FB6507F58473A3F582731B68B3F85030C5
:10B1FC009BB21A46FB6D1344FB6507F58473A3F5EC
:10B20C0084731B681B781A01FB6D134403F204430F
:10B21C00BB65D7F804319AB2BB6D1A8007F58473FD
:10B22C00A3F584731B681B89A7F8763007F5847324
:10B23C00A3F584731B685969D7F804319BB2B7F82E
:10B24C00762007F58470A0F58270006801F00DF887
:10B25C00B3E107F58473A3F584731B681A6AD7F8F6
:10B26C000431D21A07F58473A3F584731B681A6230
:10B27C0007F58473A3F582731A6807F58473A3F535
:10B28C0084731B681B789B0013441B889BB203F0D0
:10B29C004003002B00F0C68007F58473A3F582737E
:10B2AC001B683B6707F58473A3F584731B685B7895
:10B2BC00002B77D107F58473A3F582731B68BB66EB
:10B2CC0007F58473A3F582731B68B3F850309BB2F7
:10B2DC001A46BB6E1344BB6607F58473A3F58473DF
:10B2EC001B681B781A01BB6E134403F20C437B667C
:10B2FC007B6E1B889BB2C3F309039AB27B6E1A80D8
:10B30C00D7F804313E2B21D9D7F804315B09C7F8A3
:10B31C00F030D7F8043103F01F03002B04D1D7F819
:10B32C00F030013BC7F8F0307B6E1B889AB2D7F82F
:10B33C00F0309BB29B029BB213439BB26FEA434328
:10B34C006FEA53439AB27B6E1A8050E0D7F80431FF
:10B35C00002B0AD17B6E1B889BB26FEA43436FEACA
:10B36C0053439AB27B6E1A8041E0D7F804315B08E4
:10B37C00C7F8F030D7F8043103F00103002B04D0E8
:10B38C00D7F8F0300133C7F8F0307B6E1B889AB2D7
:10B39C00D7F8F0309BB29B029BB213439AB27B6EF0
:10B3AC001A8024E007F58473A3F584731B685B781B
:10B3BC00012B1CD107F58473A3F582731B68B3F8BA
:10B3CC0050309BB21A463B6F13443B6707F58473AE
:10B3DC00A3F584731B681B781A013B6F134403F2AB
:10B3EC000C43FB66D7F804319AB2FB6E1A8007F552
:10B3FC008473A3F584731B685B89A7F8763007F513
:10B40C008473A3F584731B685969D7F804319BB214
:10B41C00B7F8762007F58470A0F58270006800F00C
:10B42C0024FFCAE007F58473A3F584731B685B786B
:10B43C00002B77D107F58473A3F582731B68FB6728
:10B44C0007F58473A3F582731B68B3F850309BB275
:10B45C001A46FB6F1344FB6707F58473A3F58473DB
:10B46C001B681B781A01FB6F134403F20443BB6780
:10B47C00BB6F1B889BB2C3F309039AB2BB6F1A80D4
:10B48C00D7F804313E2B21D9D7F804315B09C7F822
:10B49C00EC30D7F8043103F01F03002B04D1D7F89C
:10B4AC00EC30013BC7F8EC30BB6F1B889AB2D7F875
:10B4BC00EC309BB29B029BB213439BB26FEA4343AB
:10B4CC006FEA53439AB2BB6F1A805CE0D7F8043131
:10B4DC00002B0AD1BB6F1B889BB26FEA43436FEA08
:10B4EC0053439AB2BB6F1A804DE0D7F804315B0816
:10B4FC00C7F8EC30D7F8043103F00103002B04D06B
:10B50C00D7F8EC300133C7F8EC30BB6F1B889AB21C
:10B51C00D7F8EC309BB29B029BB213439AB2BB6F31
:10B52C001A8030E007F58473A3F584731B685B788D
:10B53C00012B28D107F58473A3F582731B68C7F818
:10B54C00843007F58473A3F582731B68B3F850300D
:10B55C009BB21A46D7F884301344C7F8843007F5E9
:10B56C008473A3F584731B681B781A01D7F8843095
:10B57C00134403F20443C7F88030D7F804319AB26D
:10B58C00D7F880301A8007F58473A3F584731B6891
:10B59C001B89A7F8763007F58473A3F584731B68B1
:10B5AC005969D7F804319BB2B7F8762007F5847047
:10B5BC00A0F58270006800F058FE07F58473A3F5BF
:10B5CC0082731A6807F58473A3F584731B681B7860
:10B5DC009B0013441B889BB223F4E04323F04003ED
:10B5EC007B817B8983F010037B817B8983F0200333
:10B5FC007B8107F58473A3F582731A6807F584734E
:10B60C00A3F584731B681B789B001A447B8943F059
:10B61C007F4343F47F0343F4004343F080039BB226
:10B62C00138000F0DEBC07F58473A3F584731B68EC
:10B63C001B7B002B40F0BB8007F58473A3F5847350
:10B64C001B689A6907F58473A3F584731B681B69DF
:10B65C009A4217D907F58473A3F584731B681B6989
:10B66C00C7F8043107F58473A3F584731B689A69D2
:10B67C00D7F80431D21A07F58473A3F584731B68C9
:10B68C009A610EE007F58473A3F584731B689B69BC
:10B69C00C7F8043107F58473A3F584731B68002283
:10B6AC009A6107F58473A3F582731B68C7F8903011
:10B6BC0007F58473A3F582731B68B3F850309BB203
:10B6CC001A46D7F890301344C7F8903007F58473B6
:10B6DC00A3F584731B681B781A01D7F890301344B8
:10B6EC0003F20C43C7F88C30D7F88C301B889BB214
:10B6FC00C3F309039AB2D7F88C301A80D7F8043107
:10B70C003E2B24D9D7F804315B09C7F8E830D7F8B9
:10B71C00043103F01F03002B04D1D7F8E830013BB0
:10B72C00C7F8E830D7F88C301B889AB2D7F8E830D5
:10B73C009BB29B029BB213439BB26FEA43436FEAEB
:10B74C0053439AB2D7F88C301A8000F010BCD7F85B
:10B75C000431002B0CD1D7F88C301B889BB26FEACC
:10B76C0043436FEA53439AB2D7F88C301A80FEE306
:10B77C00D7F804315B08C7F8E830D7F8043103F088
:10B78C000103002B04D0D7F8E8300133C7F8E830B8
:10B79C00D7F88C301B889AB2D7F8E8309BB29B0252
:10B7AC009BB213439AB2D7F88C301A80DFE307F5BB
:10B7BC008473A3F584731B68DB78022B40F018822A
:10B7CC0007F58473A3F584731B685B78002B40F03A
:10B7DC009D8007F58473A3F582731B68C7F8AC30A2
:10B7EC0007F58473A3F582731B68B3F850309BB2D2
:10B7FC001A46D7F8AC301344C7F8AC3007F584734D
:10B80C00A3F584731B681B781A01D7F8AC3013446A
:10B81C0003F20443C7F8A830D7F8A8301B889BB2B2
:10B82C00C3F309039AB2D7F8A8301A8007F58473CA
:10B83C00A3F584731B681B693E2B2BD907F5847306
:10B84C00A3F584731B681B695B09C7F8E43007F523
:10B85C008473A3F584731B681B6903F01F03002B0F
:10B86C0004D1D7F8E430013BC7F8E430D7F8A8305E
:10B87C001B889AB2D7F8E4309BB29B029BB213435D
:10B88C009BB26FEA43436FEA53439AB2D7F8A8309E
:10B89C001A8070E007F58473A3F584731B681B6929
:10B8AC00002B0CD1D7F8A8301B889BB26FEA43430E
:10B8BC006FEA53439AB2D7F8A8301A805BE007F5C9
:10B8CC008473A3F584731B681B695B08C7F8E430A9
:10B8DC0007F58473A3F584731B681B6903F00103DC
:10B8EC00002B04D0D7F8E4300133C7F8E430D7F894
:10B8FC00A8301B889AB2D7F8E4309BB29B029BB25B
:10B90C0013439AB2D7F8A8301A8034E007F5847341
:10B91C00A3F584731B685B78012B2CD107F584731A
:10B92C00A3F582731B68C7F8B43007F58473A3F5CD
:10B93C0082731B68B3F850309BB21A46D7F8B430F8
:10B94C001344C7F8B43007F58473A3F584731B68EC
:10B95C001B781A01D7F8B430134403F20443C7F828
:10B96C00B03007F58473A3F584731B681B699AB216
:10B97C00D7F8B0301A8007F58473A3F582731B686F
:10B98C00C7F8A43007F58473A3F584731B685B7840
:10B99C00002B40F09D8007F58473A3F582731B6820
:10B9AC00C7F89C3007F58473A3F582731B68B3F852
:10B9BC0050309BB21A46D7F89C301344C7F89C30D1
:10B9CC0007F58473A3F584731B681B781A01D7F8E9
:10B9DC009C30134403F20C43C7F89830D7F89830D6
:10B9EC001B889BB2C3F309039AB2D7F898301A801C
:10B9FC0007F58473A3F584731B681B693E2B2BD945
:10BA0C0007F58473A3F584731B681B695B09C7F87E
:10BA1C00E03007F58473A3F584731B681B6903F08E
:10BA2C001F03002B04D1D7F8E030013BC7F8E030FE
:10BA3C00D7F898301B889AB2D7F8E0309BB29B02AB
:10BA4C009BB213439BB26FEA43436FEA53439AB2E0
:10BA5C00D7F898301A8069E007F58473A3F58473DE
:10BA6C001B681B69002B0CD1D7F898301B889BB234
:10BA7C006FEA43436FEA53439AB2D7F898301A806F
:10BA8C0054E007F58473A3F584731B681B695B088A
:10BA9C00C7F8E03007F58473A3F584731B681B6942
:10BAAC0003F00103002B04D0D7F8E0300133C7F8C2
:10BABC00E030D7F898301B889AB2D7F8E0309BB2B8
:10BACC009B029BB213439AB2D7F898301A802DE0A0
:10BADC0007F58473A3F584731B685B78012B25D160
:10BAEC0007F58473A3F582731B68B3F850309BB2CF
:10BAFC001A46D7F8A4301344C7F8A43007F584735A
:10BB0C00A3F584731B681B781A01D7F8A43013446F
:10BB1C0003F20C43C7F8A03007F58473A3F58473C4
:10BB2C001B681B699AB2D7F8A0301A8007F584738A
:10BB3C00A3F584731B68DB69002B00F0188207F5F2
:10BB4C008473A3F582731A6807F58473A3F5847361
:10BB5C001B681B789B0013441B88A7F89630B7F81A
:10BB6C00963003F48043002B05D0B7F8963003F0E1
:10BB7C004003002B0DD1B7F8963003F48043002B13
:10BB8C0040F0F581B7F8963003F04003002B40F0FD
:10BB9C00EE8107F58473A3F582731A6807F5847335
:10BBAC00A3F584731B681B789B0013441B889BB202
:10BBBC0023F4E04323F07003A7F8943007F5847363
:10BBCC00A3F582731A6807F58473A3F584731B6855
:10BBDC001B789B001A44B7F8943043F07F4343F42E
:10BBEC007F0343F4004343F0C0039BB21380BEE1D8
:10BBFC0007F58473A3F584731B68DB78012B40F085
:10BC0C00B48107F58473A3F584731B689A6907F5EF
:10BC1C008473A3F584731B681B699A4217D907F5C3
:10BC2C008473A3F584731B681B69C7F8043107F58B
:10BC3C008473A3F584731B689A69D7F80431D21AFC
:10BC4C0007F58473A3F584731B689A610EE007F5FE
:10BC5C008473A3F584731B689B69C7F8043107F5DB
:10BC6C008473A3F584731B6800229A6107F58473AF
:10BC7C00A3F584731B685B78002B40F0858007F577
:10BC8C008473A3F582731B68C7F8CC3007F58473F3
:10BC9C00A3F582731B68B3F850309BB21A46D7F8E1
:10BCAC00CC301344C7F8CC3007F58473A3F58473F8
:10BCBC001B681B781A01D7F8CC30134403F20443E9
:10BCCC00C7F8C830D7F8C8301B889BB2C3F3090338
:10BCDC009AB2D7F8C8301A80D7F804313E2B23D942
:10BCEC00D7F804315B09C7F8DC30D7F8043103F01E
:10BCFC001F03002B04D1D7F8DC30013BC7F8DC3034
:10BD0C00D7F8C8301B889AB2D7F8DC309BB29B02AC
:10BD1C009BB213439BB26FEA43436FEA53439AB20D
:10BD2C00D7F8C8301A8060E0D7F80431002B0CD15A
:10BD3C00D7F8C8301B889BB26FEA43436FEA534372
:10BD4C009AB2D7F8C8301A804FE0D7F804315B08A4
:10BD5C00C7F8DC30D7F8043103F00103002B04D012
:10BD6C00D7F8DC300133C7F8DC30D7F8C8301B8883
:10BD7C009AB2D7F8DC309BB29B029BB213439AB2B7
:10BD8C00D7F8C8301A8030E007F58473A3F58473B4
:10BD9C001B685B78012B28D107F58473A3F582739C
:10BDAC001B68C7F8D43007F58473A3F582731B683E
:10BDBC00B3F850309BB21A46D7F8D4301344C7F8B6
:10BDCC00D43007F58473A3F584731B681B781A01B0
:10BDDC00D7F8D430134403F20443C7F8D030D7F863
:10BDEC0004319AB2D7F8D0301A8007F58473A3F5D2
:10BDFC0082731B68C7F8C43007F58473A3F584738A
:10BE0C001B685B78002B40F0858007F58473A3F5E5
:10BE1C0082731B68C7F8BC3007F58473A3F5827373
:10BE2C001B68B3F850309BB21A46D7F8BC30134499
:10BE3C00C7F8BC3007F58473A3F584731B681B78B3
:10BE4C001A01D7F8BC30134403F20C43C7F8B830CE
:10BE5C00D7F8B8301B889BB2C3F309039AB2D7F852
:10BE6C00B8301A80D7F804313E2B23D9D7F80431D7
:10BE7C005B09C7F8D830D7F8043103F01F03002B47
:10BE8C0004D1D7F8D830013BC7F8D830D7F8B83040
:10BE9C001B889AB2D7F8D8309BB29B029BB2134343
:10BEAC009BB26FEA43436FEA53439AB2D7F8B83068
:10BEBC001A805CE0D7F80431002B0CD1D7F8B830DD
:10BECC001B889BB26FEA43436FEA53439AB2D7F88D
:10BEDC00B8301A804BE0D7F804315B08C7F8D8307B
:10BEEC00D7F8043103F00103002B04D0D7F8D83075
:10BEFC000133C7F8D830D7F8B8301B889AB2D7F8C6
:10BF0C00D8309BB29B029BB213439AB2D7F8B8308D
:10BF1C001A802CE007F58473A3F584731B685B7897
:10BF2C00012B24D107F58473A3F582731B68B3F836
:10BF3C0050309BB21A46D7F8C4301344C7F8C430FB
:10BF4C0007F58473A3F584731B681B781A01D7F863
:10BF5C00C430134403F20C43C7F8C030D7F8043193
:10BF6C009AB2D7F8C0301A8001E001233AE007F505
:10BF7C008473A3F582731A6807F58473A3F584732D
:10BF8C001B681B789B0013441B889BB223F48043D3
:10BF9C0023F07003A7F88A30B7F88A3083F4805303
:10BFAC00A7F88A30B7F88A3083F40053A7F88A30A0
:10BFBC0007F58473A3F582731A6807F58473A3F5E8
:10BFCC0084731B681B789B001A44B7F88A3043F0C3
:10BFDC007F4343F47F0343F4004343F080039BB25D
:10BFEC0013800023184607F58477BD4680BD80B4C6
:10BFFC0085B000AF786039603B685B78002B20D04F
:10C00C007A683B681B789B0013441B889BB223F413
:10C01C00E04323F04003BB81BB8983F01003BB8159
:10C02C007A683B681B789B001A44BB8943F07F43BA
:10C03C0043F47F0343F4004343F080039BB213802B
:10C04C001FE07A683B681B789B0013441B889BB2EB
:10C05C0023F4804323F07003FB81FB8983F480532A
:10C06C00FB817A683B681B789B001A44FB8943F080
:10C07C007F4343F47F0343F4004343F080039BB2BC
:10C08C001380002318461437BD4680BC704780B41B
:10C09C0087B000AF786039603B681B7B002B40F0A9
:10C0AC009D803B685B78002B4CD07A683B681B7892
:10C0BC009B0013441B883B823B8A03F04003002BFC
:10C0CC001BD07A683B681B789B0013441B889BB27F
:10C0DC0023F4E04323F07003FB817A683B681B7800
:10C0EC009B001A44FB8943F07F4343F47F0343F4E2
:10C0FC00004343F0C0039BB213803B68DB78012BF9
:10C10C006CD07A683B681B789B0013441B889BB2ED
:10C11C0023F4E04323F04003BB81BB8983F020036D
:10C12C00BB817A683B681B789B001A44BB8943F03F
:10C13C007F4343F47F0343F4004343F080039BB2FB
:10C14C0013804BE07A683B681B789B0013441B8878
:10C15C00FB82FB8A03F48043002B1BD07A683B687C
:10C16C001B789B0013441B889BB223F4E04323F001
:10C17C007003BB827A683B681B789B001A44BB8AAD
:10C18C0043F07F4343F47F0343F4404343F0800385
:10C19C009BB213807A683B681B789B0013441B8806
:10C1AC009BB223F4804323F070037B827B8A83F45D
:10C1BC0080537B827B8A83F400537B827A683B6852
:10C1CC001B789B001A447B8A43F07F4343F47F0324
:10C1DC0043F4004343F080039BB2138000231846C2
:10C1EC001C37BD4680BC704780B483B000AF78600C
:10C1FC000B46FB70FB78002B03D17B688022A3F8E5
:10C20C004C20002318460C37BD4680BC704780B4C8
:10C21C0083B000AF7860002318460C37BD4680BC55
:10C22C00704780B483B000AF7860002318460C3799
:10C23C00BD4680BC704780B485B000AF78607B6829
:10C24C00B3F844309BB2FB60FB6818461437BD460C
:10C25C0080BC704780B483B000AF78603960002335
:10C26C0018460C37BD4680BC704780B48BB000AF0D
:10C27C00F860B96011461A460B46FB801346BB802A
:10C28C00BB8801335B08BB61FB687B61BB68FB61EE
:10C29C00FB885A007B69134403F580633B62BB69DE
:10C2AC007B621FE0FB691B787B82FB6901331B7887
:10C2BC001BB21B021AB2B7F9123013431BB27B82AA
:10C2CC003B6A7A8A1A803B6A02333B623B6A0233CE
:10C2DC003B62FB690133FB61FB690133FB617B6AE8
:10C2EC00013B7B627B6A002BDCD100BF00BF2C378B
:10C2FC00BD4680BC704780B48BB000AFF860B960AD
:10C30C0011461A460B46FB801346BB80BB885B0864
:10C31C009BB2BB61FB687B61BB68FB61FB885A000D
:10C32C007B69134403F580633B62BB697B621BE052
:10C33C003B6A1B889BB23B613B6A02333B623B69A5
:10C34C00DAB2FB691A70FB690133FB613B691B0AAA
:10C35C00DAB2FB691A70FB690133FB613B6A023389
:10C36C003B627B6A013B7B627B6A002BE0D1BB8822
:10C37C0003F001039BB2002B07D03B6A1B889BB2D6
:10C38C003B613B69DAB2FB691A7000BF2C37BD46C2
:10C39C0080BC704780B584B000AF78600B46FB70F2
:10C3AC000023FB737B681B7C002B15D14FF40073AF
:10C3BC0002228121786801F000FF7B680122DA6299
:10C3CC004FF4007302220121786801F0F6FE7B68BD
:10C3DC000122C3F86C2112E04023022281217868EB
:10C3EC0001F0EBFE7B680122DA624023022201217C
:10C3FC00786801F0E2FE7B680122C3F86C21082307
:10C40C0003228221786801F0D8FE7B6801221A642D
:10C41C004FF4077001F0F8FF02467B68C3F8B822AE
:10C42C007B68D3F8B832002B02D10123FB7326E0D2
:10C43C007B68D3F8B832BB607B68D3F8BC321B681E
:10C44C009847BB680022C3F81422BB680022C3F8CB
:10C45C0018227B681B7C002B09D1BB68D3F8042203
:10C46C004FF400730121786801F097FF07E0BB6877
:10C47C00D3F8042240230121786801F08EFFFB7B66
:10C48C0018461037BD4680BD80B584B000AF7860CB
:10C49C000B46FB700023FB738121786801F0B3FE1F
:10C4AC007B680022DA620121786801F0ACFE7B68BF
:10C4BC000022C3F86C218221786801F0A4FE7B680D
:10C4CC0000221A647B68D3F8B832002B0ED07B683C
:10C4DC00D3F8BC325B6898477B68D3F8B8321846FF
:10C4EC0001F09EFF7B680022C3F8B822FB7B184644
:10C4FC001037BD4680BD80B586B000AF786039601E
:10C50C007B68D3F8B8323B610023FB730023BB81FB
:10C51C000023FB753B681B7803F06003002B39D0BC
:10C52C00202B7FD13B68DB88002B29D03B681B7804
:10C53C005BB2002B11DA7B68D3F8BC329B683A688B
:10C54C00507839693A68D288984739693B68DB88F2
:10C55C001A46786801F006FA6BE03B685A783B693A
:10C56C0083F800223B68DB88DAB23B6983F801224E
:10C57C0039693B68DB881A46786801F021FA58E083
:10C58C007B68D3F8BC329B683A68507800223968D3
:10C59C0098474EE03B685B780B2B2ED00B2B38DC8E
:10C5AC00002B02D00A2B14D033E07B6893F89C321A
:10C5BC00032B07D107F10C0302221946786801F00E
:10C5CC00D1F92EE03968786801F062F90223FB7525
:10C5DC0027E07B6893F89C32032B07D107F10F03FC
:10C5EC0001221946786801F0BDF91AE039687868BB
:10C5FC0001F04EF90223FB7513E07B6893F89C3233
:10C60C00032B0DD03968786801F042F90223FB75D1
:10C61C0006E03968786801F03BF90223FB7500E00D
:10C62C0000BF06E03968786801F032F90223FB7527
:10C63C0000BFFB7D18461837BD4680BD80B584B061
:10C64C0000AF78600B46FB707B68D3F8B832FB60A8
:10C65C007B68D3F8C032BB607B68D3F8B832002B50
:10C66C003AD0FA78796813469B0013449B000B442C
:10C67C001C331B68002B29D0FA78796813469B0071
:10C68C0013449B000B441C331A68F978B8680B46AA
:10C69C009B000B44DB00034420331B68B2FBF3F11B
:10C6AC0001FB03F3D31A002B10D1FA7879681346E7
:10C6BC009B0013449B000B441C3300221A60F97836
:10C6CC0000230022786801F045FE03E0FB6800229D
:10C6DC00C3F81422002300E0022318461037BD468D
:10C6EC0080BD80B584B000AF78600B46FB707B6872
:10C6FC00D3F8B832FB60FB781946786801F070FE0D
:10C70C000246FB68C3F80C227B68D3F8B832002BC6
:10C71C000DD07B68D3F8BC32DB68FA68D2F804021F
:10C72C00FA6802F5037211469847002300E00223D1
:10C73C0018461037BD4680BD80B584B000AF786018
:10C74C007B68D3F8B832FB607B68D3F8BC32002B23
:10C75C0014D0FB6893F80032FF2B0FD07B68D3F812
:10C76C00BC329B68FA6892F80002F968FA6892F891
:10C77C0001229847FB68FF2283F800220023184609
:10C78C001037BD4680BD000080B483B000AF786028
:10C79C007B6843221A80034B18460C37BD4680BC7D
:10C7AC00704700BFA400002080B483B000AF786055
:10C7BC007B6843221A80034B18460C37BD4680BC5D
:10C7CC00704700BF6000002080B483B000AF786079
:10C7DC007B6843221A80034B18460C37BD4680BC3D
:10C7EC00704700BFE800002080B483B000AF7860D1
:10C7FC007B680A221A80034B18460C37BD4680BC56
:10C80C00704700BF1C00002080B485B000AF78607A
:10C81C0039600223FB733B68002B05D07B683A68B8
:10C82C00C3F8BC220023FB73FB7B18461437BD46B0
:10C83C0080BC704780B487B000AFF860B960134615
:10C84C00FB80FB68D3F8B8327B617B69BA68C3F8AC
:10C85C000822FA887B69C3F81022002318461C377B
:10C86C00BD4680BC704780B485B000AF786039603D
:10C87C007B68D3F8B832FB60FB683A68C3F80422D3
:10C88C00002318461437BD4680BC704780B584B071
:10C89C0000AF78607B68D3F8B832FB607B68D3F864
:10C8AC00B832002B1CD0FB68D3F81432002B15D1F6
:10C8BC00FB680122C3F81422FB68D3F810227B68B2
:10C8CC001A63FB68D3F80822FB68D3F810329BB2CA
:10C8DC008121786801F03EFD002302E0012300E095
:10C8EC00022318461037BD4680BD80B584B000AF1A
:10C8FC0078607B68D3F8B832FB607B68D3F8B832C9
:10C90C00002B17D07B681B7C002B09D1FB68D3F85C
:10C91C0004224FF400730121786801F03EFD07E01A
:10C92C00FB68D3F8042240230121786801F035FD1F
:10C93C00002300E0022318461037BD4680BD80B5A9
:10C94C0084B000AFF860B9601346FB71FB68002B34
:10C95C0001D102231AE0FB68D3F8B432002B03D0C8
:10C96C00FB680022C3F8B422BB68002B03D0FB6821
:10C97C00BA68C3F8B022FB68012283F89C22FB68DA
:10C98C00FA791A70F86801F0A3FB002318461037E7
:10C99C00BD4680BD80B485B000AF7860396000239F
:10C9AC00FB733B68002B06D07B683A68C3F8B42253
:10C9BC000023FB7301E00223FB73FB7B1846143747
:10C9CC00BD4680BC704780B582B000AF7860786897
:10C9DC0001F0D8FB002318460837BD4680BD80B453
:10C9EC0083B000AF7860002318460C37BD4680BC7E
:10C9FC00704780B584B000AF78600B46FB700223A3
:10CA0C00FB737B68D3F8B432002B0CD07B68D3F863
:10CA1C00B4321B68FA781146786898470346002BA5
:10CA2C0001D10023FB73FB7B18461037BD4680BD3C
:10CA3C0080B582B000AF78600B46FB707B68D3F892
:10CA4C00B4325B68FA781146786898470023184628
:10CA5C000837BD4680BD80B582B000AF78603960C4
:10CA6C007B6803F52A733968184600F0D8FE7B689A
:10CA7C000122C3F894227B68B3F8AE321A467B6865
:10CA8C00C3F898227B6893F8A83203F01F03022B9B
:10CA9C0016D0022B1CD8002B02D0012B08D017E08B
:10CAAC007B6803F52A731946786800F0CBF91AE015
:10CABC007B6803F52A731946786800F02DFA12E0AA
:10CACC007B6803F52A731946786800F06DFA0AE062
:10CADC007B6893F8A83223F07F03DBB219467868A1
:10CAEC0001F0B0FB00BF002318460837BD4680BDDF
:10CAFC0080B586B000AFF8600B467A60FB72FB7AAB
:10CB0C00002B4BD1FB6803F5AA737B61FB68D3F850
:10CB1C009432032B34D17B69DA687B691B699A42A6
:10CB2C0019D97B69DA687B691B69D21A7B69DA606F
:10CB3C007B69DA687B691B699A4203D27B69DB6883
:10CB4C009BB202E07B691B699BB21A467968F86854
:10CB5C0000F054FF38E0FB68D3F8B4321B69002BAB
:10CB6C000AD0FB6893F89C32032B05D1FB68D3F8F1
:10CB7C00B4321B69F8689847F86800F051FF23E05D
:10CB8C00FB68D3F89432052B1ED1FB680022C3F846
:10CB9C0094220021F86801F055FB15E0FB68D3F8EE
:10CBAC00B4329B69002B0DD0FB6893F89C32032B9D
:10CBBC0008D1FB68D3F8B4329B69FA7A1146F8684D
:10CBCC00984701E0022300E0002318461837BD46C1
:10CBDC0080BD80B586B000AFF8600B467A60FB7202
:10CBEC00FB7A002B7FD1FB6814337B61FB68D3F895
:10CBFC009432022B5CD17B69DA687B691B699A429F
:10CC0C0015D97B69DA687B691B69D21A7B69DA6092
:10CC1C007B69DB689BB21A467968F86800F0BEFE47
:10CC2C00002300220021F86801F0B7FB4EE07B697D
:10CC3C009B687A691269B3FBF2F101FB02F29B1A51
:10CC4C00002B1CD17B699A687B691B699A4216D3AD
:10CC5C007B699A68FB68D3F898329A420FD200220B
:10CC6C000021F86800F09AFEFB680022C3F89822B5
:10CC7C00002300220021F86801F08FFB26E0FB68FE
:10CC8C00D3F8B432DB68002B0AD0FB6893F89C32E3
:10CC9C00032B05D1FB68D3F8B432DB68F8689847EE
:10CCAC008021F86801F0CEFAF86800F0CCFE0DE0B7
:10CCBC00FB68D3F89432042B04D0FB68D3F894327D
:10CCCC00002B03D18021F86801F0BCFAFB6893F8C3
:10CCDC00A032012B1DD1F868FFF781FEFB68002202
:10CCEC0083F8A02215E0FB68D3F8B4325B69002B03
:10CCFC000DD0FB6893F89C32032B08D1FB68D3F85A
:10CD0C00B4325B69FA7A1146F868984701E002235D
:10CD1C0000E0002318461837BD4680BD80B582B0B0
:10CD2C0000AF7860402300220021786801F045FABA
:10CD3C007B680122C3F858217B684022C3F8642128
:10CD4C00402300228021786801F037FA7B680122A9
:10CD5C009A617B6840225A627B68012283F89C228C
:10CD6C007B680022C3F894227B6800225A607B689F
:10CD7C000022C3F8A4227B68D3F8B832002B09D068
:10CD8C007B68D3F8B4325B687A685268D2B21146C9
:10CD9C0078689847002318460837BD4680BD80B494
:10CDAC0083B000AF78600B46FB707B68FA781A741E
:10CDBC00002318460C37BD4680BC704780B483B046
:10CDCC0000AF78607B6893F89C227B6883F89D2287
:10CDDC007B68042283F89C22002318460C37BD463E
:10CDEC0080BC704780B483B000AF78607B6893F8E8
:10CDFC009C32042B05D17B6893F89D227B6883F8C9
:10CE0C009C22002318460C37BD4680BC704780B569
:10CE1C0082B000AF78607B6893F89C32032B0BD107
:10CE2C007B68D3F8B432DB69002B05D07B68D3F870
:10CE3C00B432DB6978689847002318460837BD463A
:10CE4C0080BD000080B584B000AF786039600023ED
:10CE5C00FB733B681B7803F06003402B05D0402B21
:10CE6C004FD8002B09D0202B4BD17B68D3F8B43290
:10CE7C009B6839687868984748E03B685B78092B71
:10CE8C0039D801A252F823F0E5CE0008F9CE0008FB
:10CE9C0003CF0008EFCE000803CF0008C7CE000870
:10CEAC00BDCE000803CF0008DBCE0008D1CE0008B1
:10CEBC003968786800F0DCF922E03968786800F0AD
:10CECC003FFB1DE03968786800F07EFB18E039689C
:10CEDC00786800F007FC13E03968786800F037FCDC
:10CEEC000EE03968786800F065FC09E0396878680C
:10CEFC0000F074FC04E03968786800F0C9FC00BFED
:10CF0C0004E03968786800F0C3FC00BFFB7B18466E
:10CF1C001037BD4680BD00BF80B584B000AF7860CF
:10CF2C0039600023FB733B681B7803F06003402BD4
:10CF3C0005D0402B2ED8002B01D0202B2AD17B687A
:10CF4C0093F89C32013B022B1DD83B689B88DBB2CB
:10CF5C00012B13D87B68D3F8B4329B683968786896
:10CF6C0098470346FB733B68DB88002B10D1FB7B97
:10CF7C00002B0DD1786800F053FD09E03968786812
:10CF8C0000F086FC04E03968786800F081FC00E071
:10CF9C0000BF04E03968786800F07AFC00BF002319
:10CFAC0018461037BD4680BD80B584B000AF7860A0
:10CFBC0039600023FB733B689B88BB733B681B7811
:10CFCC0003F06003402B07D0402B00F24681002B6E
:10CFDC000AD0202B40F041817B68D3F8B4329B6897
:10CFEC003968786898473DE13B681B7803F060032B
:10CFFC00202B0AD17B68D3F8B4329B6839687868E7
:10D00C0098470346FB73FB7B2DE13B685B78032B56
:10D01C0007D0032B00F31B81002B72D0012B3AD0CD
:10D02C0015E17B6893F89C32022B02D0032B15D0B0
:10D03C002BE0BB7B002B0CD0BB7B802B09D0BB7BAC
:10D04C001946786801F0FEF88021786801F0FAF84A
:10D05C0020E03968786800F01BFC1BE03B685B88BB
:10D06C00002B0ED1BB7B002B0BD0BB7B802B08D0B5
:10D07C003B68DB88002B04D1BB7B1946786801F038
:10D08C00E1F8786800F0CCFC04E03968786800F0CE
:10D09C00FFFB00BFE0E07B6893F89C32022B02D0D0
:10D0AC00032B15D026E0BB7B002B0CD0BB7B802B3D
:10D0BC0009D0BB7B1946786801F0C4F880217868E8
:10D0CC0001F0C0F81CE03968786800F0E1FB17E06B
:10D0DC003B685B88002B12D1BB7B03F07F03002BDA
:10D0EC0004D0BB7B1946786801F0CBF8786800F067
:10D0FC0097FC04E03968786800F0CAFB00E000BFD8
:10D10C00AAE07B6893F89C32022B02D0032B32D01E
:10D11C0097E0BB7B002B07D0BB7B802B04D03968FE
:10D12C00786800F0B5FB91E097F90E30002B0BDA24
:10D13C00BB7B03F07F0213469B0013449B00103310
:10D14C007A68134404330BE0BB7B03F07F02134675
:10D15C009B0013449B0003F5A8737A6813440433B3
:10D16C00BB60BB6800221A60BB6802221946786853
:10D17C0000F0F8FB6AE097F90E30002B11DABB7B5C
:10D18C0003F00F02796813469B0013449B000B4479
:10D19C0018331B68002B17D13968786800F078FBBE
:10D1AC0054E0BB7B03F00F02796813469B001344D9
:10D1BC009B000B4403F5AC731B68002B04D139683E
:10D1CC00786800F065FB41E097F90E30002B0BDA24
:10D1DC00BB7B03F07F0213469B0013449B00103370
:10D1EC007A68134404330BE0BB7B03F07F021346D5
:10D1FC009B0013449B0003F5A8737A681344043313
:10D20C00BB60BB7B002B02D0BB7B802B03D1BB68EC
:10D21C0000221A600EE0BB7B1946786801F050F8CA
:10D22C000346002B03D0BB6801221A6002E0BB68E6
:10D23C0000221A60BB6802221946786800F092FB43
:10D24C0004E03968786800F023FB00BF04E039681B
:10D25C00786800F01DFB00BF04E03968786800F0C6
:10D26C0017FB00BFFB7B18461037BD4680BD000086
:10D27C0080B584B000AF7860396000233B81002317
:10D28C00FB600023FB723B685B881B0A9BB2013B73
:10D29C00062B00F2288101A252F823F0C5D2000817
:10D2AC00DDD200081DD30008F3D40008F3D4000825
:10D2BC0093D40008BFD400087B68D3F8B0321B6845
:10D2CC007A68127C07F1080110469847F86012E161
:10D2DC007B681B7C002B0DD17B68D3F8B4329B6A26
:10D2EC0007F1080210469847F860FB6801330222E8
:10D2FC001A7000E17B68D3F8B432DB6A07F10802DC
:10D30C0010469847F860FB68013302221A70F2E06D
:10D31C003B685B88DBB2052B00F2AC8001A252F8B3
:10D32C0023F000BF49D300087DD30008B1D3000817
:10D33C00E5D3000819D400084DD400087B68D3F855
:10D34C00B0325B68002B0BD07B68D3F8B0325B68D3
:10D35C007A68127C07F1080110469847F86091E052
:10D36C003968786800F094FAFB7A0133FB7289E033
:10D37C007B68D3F8B0329B68002B0BD07B68D3F85A
:10D38C00B0329B687A68127C07F108011046984706
:10D39C00F86077E03968786800F07AFAFB7A013344
:10D3AC00FB726FE07B68D3F8B032DB68002B0BD0DC
:10D3BC007B68D3F8B032DB687A68127C07F108011D
:10D3CC0010469847F8605DE03968786800F060FABC
:10D3DC00FB7A0133FB7255E07B68D3F8B0321B69E2
:10D3EC00002B0BD07B68D3F8B0321B697A68127CA7
:10D3FC0007F1080110469847F86043E039687868EF
:10D40C0000F046FAFB7A0133FB723BE07B68D3F801
:10D41C00B0325B69002B0BD07B68D3F8B0325B6900
:10D42C007A68127C07F1080110469847F86029E0E9
:10D43C003968786800F02CFAFB7A0133FB7221E032
:10D44C007B68D3F8B0329B69002B0BD07B68D3F888
:10D45C00B0329B697A68127C07F108011046984734
:10D46C00F8600FE03968786800F012FAFB7A013343
:10D47C00FB7207E03968786800F00AFAFB7A01332E
:10D48C00FB7238E037E07B681B7C002B09D17B6892
:10D49C00D3F8B4325B6B07F1080210469847F8607A
:10D4AC0029E03968786800F0F3F9FB7A0133FB72F4
:10D4BC0021E07B681B7C002B0DD17B68D3F8B43248
:10D4CC001B6B07F1080210469847F860FB680133A4
:10D4DC0007221A700FE03968786800F0D9F9FB7AE6
:10D4EC000133FB7207E03968786800F0D1F9FB7AF8
:10D4FC000133FB7200BFFB7A002B1CD13B89002B44
:10D50C0011D03B68DB88002B0DD03B68DA883B8957
:10D51C00934228BF13469BB23B813B891A46F9685C
:10D52C00786800F01FFA3B68DB88002B04D1786820
:10D53C0000F076FA00E000BF1037BD4680BD00BF9A
:10D54C0080B584B000AF786039603B689B88002B55
:10D55C0030D13B68DB88002B2CD13B685B887F2B60
:10D56C0028D83B685B88DBB203F07F03FB737B68D6
:10D57C0093F89C32032B04D13968786800F088F951
:10D58C001DE07B68FA7B83F89E22FB7B194678684A
:10D59C0000F0C1FE786800F043FAFB7B002B04D04E
:10D5AC007B68022283F89C2209E07B68012283F8C5
:10D5BC009C2204E03968786800F06AF900BF00BF6B
:10D5CC001037BD4680BD000080B582B000AF7860DA
:10D5DC0039603B685B88DAB2414B1A70404B1B7860
:10D5EC00012B04D93968786800F052F975E07B6832
:10D5FC0093F89C32022B02D0032B23D062E0384BE1
:10D60C001B78002B1AD0364B1B781A467B685A6055
:10D61C007B68032283F89C22314B1B78194678686F
:10D62C00FFF7E7F90346022B04D13968786800F05C
:10D63C002FF952E0786800F0F3F94EE0786800F0CA
:10D64C00EFF94AE0264B1B78002B12D17B680222A3
:10D65C0083F89C22224B1B781A467B685A60204B1D
:10D66C001B7819467868FFF7E3F9786800F0D8F969
:10D67C0033E01B4B1B781A467B685B689A421DD0C3
:10D68C007B685B68DBB219467868FFF7D1F9144BFD
:10D69C001B781A467B685A60114B1B7819467868C0
:10D6AC00FFF7A7F90346022B04D13968786800F01C
:10D6BC00EFF812E0786800F0B3F90EE0786800F04B
:10D6CC00AFF90AE03968786800F0E2F8044B1B788F
:10D6DC0019467868FFF7ACF900BF0837BD4680BD26
:10D6EC009804002080B582B000AF786039603B6848
:10D6FC00DB88012B04D03968786800F0C9F822E087
:10D70C007B6893F89C32022B02DC002B03DC15E0C7
:10D71C00032B0BD012E07B6800229A607B680833E5
:10D72C0001221946786800F01DF90CE07B6804337F
:10D73C0001221946786800F015F904E03968786818
:10D74C0000F0A6F800BF00BF0837BD4680BD80B50D
:10D75C0082B000AF786039607B6893F89C32013BF3
:10D76C00022B1ED83B68DB88022B04D03968786802
:10D77C0000F08EF81AE07B680122DA607B68D3F83F
:10D78C00A432002B05D07B68DB6843F002027B6877
:10D79C00DA607B680C3302221946786800F0E2F8F4
:10D7AC0004E03968786800F073F800BF00BF0837F0
:10D7BC00BD4680BD80B582B000AF786039603B68F3
:10D7CC005B88012B06D17B680122C3F8A422786800
:10D7DC0000F026F900BF0837BD4680BD80B582B089
:10D7EC0000AF786039607B6893F89C32013B022B68
:10D7FC000BD83B685B88012B0CD17B680022C3F8EB
:10D80C00A422786800F00CF904E03968786800F01C
:10D81C003FF800E000BF00BF0837BD4680BD80B4B4
:10D82C0083B000AF786039603B681A787B681A70F7
:10D83C003B685A787B685A703B6802331B781A46EF
:10D84C003B6803331B781B029BB213449AB27B6870
:10D85C005A803B6804331B781A463B6805331B78A7
:10D86C001B029BB213449AB27B689A803B680633C6
:10D87C001B781A463B6807331B781B029BB2134478
:10D88C009AB27B68DA8000BF0C37BD4680BC70470B
:10D89C0080B582B000AF786039608021786800F084
:10D8AC00D1FC0021786800F0CDFC00BF0837BD46E4
:10D8BC0080BD80B586B000AFF860B9607A60002397
:10D8CC00FB75FB68002B32D0F86800F034F8034687
:10D8DC0001339BB25B009AB27B681A80FB7D5A1CA9
:10D8EC00FA751A46BB6813447A6812781A70FB7D75
:10D8FC005A1CFA751A46BB68134403221A7012E0BC
:10D90C00FB685A1CFA60FA7D511CF9751146BA680D
:10D91C000A441B781370FB7D5A1CFA751A46BB68B7
:10D92C00134400221A70FB681B78002BE8D100BF4F
:10D93C001837BD4680BD80B485B000AF7860002339
:10D94C00FB7305E0FB7B0133FB737B6801337B606E
:10D95C007B681B78002BF5D1FB7B18461437BD4632
:10D96C0080BC704780B584B000AFF860B9601346D6
:10D97C00FB80FB680222C3F89422FA88FB68DA6108
:10D98C00FA88FB681A62FB88BA680021F86800F014
:10D99C00E1FC002318461037BD4680BD80B584B02D
:10D9AC0000AFF860B9601346FB80FB88BA680021B1
:10D9BC00F86800F0CFFC002318461037BD4680BD38
:10D9CC0080B584B000AFF860B9601346FB80FB688B
:10D9DC000322C3F89422FA88FB68C3F85C21FA8806
:10D9EC00FB68C3F86021FB88BA680021F86800F076
:10D9FC00D4FC002318461037BD4680BD80B584B0DA
:10DA0C0000AFF860B9601346FB80FB88BA68002150
:10DA1C00F86800F0C2FC002318461037BD4680BDE4
:10DA2C0080B582B000AF78607B680422C3F8942282
:10DA3C00002300220021786800F08CFC002318469B
:10DA4C000837BD4680BD80B582B000AF78607B687A
:10DA5C000522C3F89422002300220021786800F0EC
:10DA6C009CFC002318460837BD4680BD80B500AF2E
:10DA7C00002212491248FEF762FF0346002B01D028
:10DA8C00F5F76CFE0F490E48FEF784FF0346002B9A
:10DA9C0001D0F5F763FE0C490948FEF7B5FE0346C5
:10DAAC00002B01D0F5F75AFE0548FEF78CFF034614
:10DABC00002B01D0F5F752FE00BF80BD3C010020C9
:10DACC009C040020280000202C01002080B485B08C
:10DADC0000AF786039601EE0144B1B889BB2013399
:10DAEC009BB2DBB2FB81FA89114B1B889BB2DBB278
:10DAFC009A4203D17B6801337B600CE07B685A1C33
:10DB0C007A600A4A128892B2D2B21978094B9954A7
:10DB1C00064AFB8913803B685A1E3A60002BDBD106
:10DB2C0000BF00BF1437BD4680BC7047601000209A
:10DB3C0062100020600F002080B400AF064B1B88E1
:10DB4C009AB2064B1B889BB2D31A9BB2DBB2184617
:10DB5C00BD4680BC704700BF6010002062100020E2
:10DB6C0080B483B000AF104B1B889AB20F4B1B884C
:10DB7C009BB29A4202D14FF0FF3310E00A4B1B8844
:10DB8C009BB2DBB20A4AD35C7B60074B1B889BB20F
:10DB9C0001339BB2DBB29AB2034B1A807B681846F6
:10DBAC000C37BD4680BC704762100020601000200E
:10DBBC00600F002080B500AF002205490548FEF734
:10DBCC0039FE05490348FEF74EFE0023184680BD7A
:10DBDC00600B00209C0400206007002080B400AF84
:10DBEC0000231846BD4680BC7047000080B483B04B
:10DBFC0000AF03463960FB711346BB80FB79232BC6
:10DC0C004AD801A252F823F0A5DC0008A5DC0008D4
:10DC1C00A5DC0008A5DC0008A5DC0008A5DC0008D4
:10DC2C00A5DC0008A5DC0008A5DC0008A5DC0008C4
:10DC3C00A5DC0008A5DC0008A5DC0008A5DC0008B4
:10DC4C00A5DC0008A5DC0008A5DC0008A5DC0008A4
:10DC5C00A5DC0008A5DC0008A5DC0008A5DC000894
:10DC6C00A5DC0008A5DC0008A5DC0008A5DC000884
:10DC7C00A5DC0008A5DC0008A5DC0008A5DC000874
:10DC8C00A5DC0008A5DC0008A5DC0008A5DC000864
:10DC9C00A5DC0008A5DC000800BF002318460C37E3
:10DCAC00BD4680BC704700BF80B582B000AF7860C5
:10DCBC0039603B681B68002B05D03B681B68194614
:10DCCC007868FFF703FF79680548FEF7CCFD044838
:10DCDC00FEF70BFE002318460837BD4680BD00BF7B
:10DCEC009C04002080B584B000AF78600B467B802C
:10DCFC000023FB730D4BD3F8B832BB60BB68D3F871
:10DD0C001432002B01D001230BE07B881A46796872
:10DD1C000648FEF78FFD0548FEF7B8FD0346FB737A
:10DD2C00FB7B18461037BD4680BD00BF9C0400200D
:10DD3C0080B483B000AF03463960FB713B6812229C
:10DD4C001A80034B18460C37BD4680BC704700BF89
:10DD5C005801002080B483B000AF03463960FB71DA
:10DD6C003B6804221A80034B18460C37BD4680BC16
:10DD7C00704700BF6C01002080B582B000AF034635
:10DD8C003960FB71FB79002B05D13A6807490848CB
:10DD9C00FFF78FFD04E03A6804490548FFF789FD59
:10DDAC00024B18460837BD4680BD00BF64100020EA
:10DDBC0068F4000880B582B000AF03463960FB718F
:10DDCC003A6804490448FFF774FD024B18460837BB
:10DDDC00BD4680BD6410002080F4000880B582B080
:10DDEC0000AF03463960FB713B681A221A8000F0C1
:10DDFC0043F8024B18460837BD4680BD7001002021
:10DE0C0080B582B000AF03463960FB71FB79002B03
:10DE1C0005D13A6807490848FFF74BFD04E03A681A
:10DE2C0004490548FFF745FD024B18460837BD4627
:10DE3C0080BD00BF6410002094F4000880B582B04F
:10DE4C0000AF03463960FB71FB79002B05D13A68B2
:10DE5C0007490848FFF72DFD04E03A6804490548D6
:10DE6C00FFF727FD024B18460837BD4680BD00BFA3
:10DE7C0064100020A0F4000880B584B000AF0F4BF4
:10DE8C001B68FB600E4B1B68BB600E4B1B687B60FA
:10DE9C00FA687B681344FB60FB68002B09D00822EE
:10DEAC000949F86800F014F804220849B86800F031
:10DEBC000FF800BF1037BD4680BD00BFE8F7FF1F4D
:10DECC00ECF7FF1FF0F7FF1F72010020820100200A
:10DEDC0080B487B000AFF860B9601346FB710023C3
:10DEEC00FB750023FB7527E0FB681B0F092B0BD878
:10DEFC00FB681B0FDAB2FB7D5B001946BB680B4459
:10DF0C003032D2B21A700AE0FB681B0FDAB2FB7D1A
:10DF1C005B001946BB680B443732D2B21A70FB68EF
:10DF2C001B01FB60FB7D5B000133BA6813440022CC
:10DF3C001A70FB7D0133FB75FA7DFB799A42D3D3C2
:10DF4C0000BF00BF1C37BD4680BC704780B584B095
:10DF5C0000AF78607B681B680D4A934213D10D4B60
:10DF6C00DB690C4A43F40003D3610A4BDB6903F40D
:10DF7C000003FB60FB68002200211420F7F7DBFD97
:10DF8C001420F7F7F4FD00BF1037BD4680BD00BF6D
:10DF9C00005C00400010024080B582B000AF786099
:10DFAC007B68D3F8D4227B6803F526731946104698
:10DFBC00FEF751FD00BF0837BD4680BD80B582B06D
:10DFCC0000AF78600B46FB707B68D3F8D402FA780C
:10DFDC00796813469B001344DB000B4403F5B273C2
:10DFEC001A68FB781946FEF783FD00BF0837BD465B
:10DFFC0080BD80B582B000AF78600B46FB707B684B
:10E00C00D3F8D402FA78796813469B001344DB00EA
:10E01C000B4424331A68FB781946FEF7DAFD00BF6F
:10E02C000837BD4680BD80B582B000AF78607B6894
:10E03C00D3F8D4321846FEF7EAFE00BF0837BD46C7
:10E04C0080BD80B584B000AF78600123FB737B6822
:10E05C009B79022B01D0F5F781FB7B68D3F8D43286
:10E06C00FA7B11461846FEF79AFE7B68D3F8D43239
:10E07C001846FEF753FE00BF1037BD4680BD0000AA
:10E08C0080B582B000AF78607B68D3F8D432184684
:10E09C00FEF794FE7B689B7A002B05D0044B1B6922
:10E0AC00034A43F00603136100BF0837BD4680BD29
:10E0BC0000ED00E080B582B000AF78607B68D3F8EB
:10E0CC00D4321846FEF78EFE00BF0837BD4680BD21
:10E0DC0080B582B000AF7860284A7B68C2F8D43231
:10E0EC007B68264AC3F8C022244B254A1A60234B6E
:10E0FC0008221A71214B02229A71204B00229A722B
:10E10C001E4B0022DA721D4B00221A731B48F8F7C3
:10E11C00F0FA0346002B01D0F5F720FB7B68D3F80F
:10E12C00C002182300220021FAF701F87B68D3F80B
:10E13C00C002582300228021F9F7F9FF7B68D3F83D
:10E14C00C002C02300228121F9F7F1FF7B68D3F8CC
:10E15C00C0024FF4887300220121F9F7E8FF7B68B5
:10E16C00D3F8C0024FF4807300228221F9F7DFFF4D
:10E17C00002318460837BD4680BD00BF641200203E
:10E18C00005C004080B584B000AF78600023FB7366
:10E19C000023BB737B68D3F8C0321846F8F79FFB9B
:10E1AC000346FB73FB7B184600F04EF90346BB732A
:10E1BC00BB7B18461037BD4680BD80B584B000AF20
:10E1CC007860084611461A460346FB700B46BB7036
:10E1DC0013463B800023FB730023BB737B68D3F88F
:10E1EC00C002BB783A88F978F8F7F3FC0346FB7366
:10E1FC00FB7B184600F028F90346BB73BB7B184623
:10E20C001037BD4680BD80B584B000AF78600B463A
:10E21C00FB700023FB730023BB737B68D3F8C03205
:10E22C00FA7811461846F8F731FD0346FB73FB7B71
:10E23C00184600F009F90346BB73BB7B1846103730
:10E24C00BD4680BD80B584B000AF78600B46FB70D6
:10E25C000023FB730023BB737B68D3F8C032FA78BE
:10E26C0011461846F8F7D9FD0346FB73FB7B18469D
:10E27C0000F0EAF80346BB73BB7B18461037BD466B
:10E28C0080BD80B584B000AF78600B46FB70002376
:10E29C00FB730023BB737B68D3F8C032FA7811464A
:10E2AC001846F8F71AFE0346FB73FB7B184600F082
:10E2BC00CBF80346BB73BB7B18461037BD4680BDFD
:10E2CC0080B485B000AF78600B46FB707B68D3F8E8
:10E2DC00C032FB6097F90330002B0BDAFB7803F0AC
:10E2EC007F02F96813469B001344DB000B44123386
:10E2FC001B780BE0FB7803F07F02F96813469B0058
:10E30C001344DB000B4403F5A9731B781846143730
:10E31C00BD4680BC704780B584B000AF78600B46BA
:10E32C00FB700023FB730023BB737B68D3F8C032F4
:10E33C00FA7811461846F8F728FC0346FB73FB7B6A
:10E34C00184600F081F80346BB73BB7B18461037A8
:10E35C00BD4680BD80B586B000AFF8607A601A46C5
:10E36C000B46FB7213463B810023FB750023BB75E8
:10E37C00FB68D3F8C0023B89F97A7A68F8F716FD86
:10E38C000346FB75FB7D184600F05EF80346BB7533
:10E39C00BB7D18461837BD4680BD80B586B000AF32
:10E3AC00F8607A601A460B46FB7213463B810023D9
:10E3BC00FB750023BB75FB68D3F8C0023B89F97A67
:10E3CC007A68F8F7ABFC0346FB75FB7D184600F04A
:10E3DC003BF80346BB75BB7D18461837BD4680BD60
:10E3EC0080B582B000AF78600B46FB707B68D3F8C9
:10E3FC00C032FA7811461846F8F7C1FC03461846A5
:10E40C000837BD4680BD000080B483B000AF786093
:10E41C00024B18460C37BD4680BC70473C1500209B
:10E42C0080B483B000AF786000BF0C37BD4680BCB1
:10E43C00704780B483B000AF78600B46FB7000BFB0
:10E44C000C37BD4680BC704780B485B000AF034626
:10E45C00FB710023FB73FB79032B17D801A252F835
:10E46C0023F000BF81E4000887E400088DE4000875
:10E47C0093E400080023FB730BE00223FB7308E01A
:10E48C000123FB7305E00223FB7302E00223FB7301
:10E49C0000BFFB7B18461437BD4680BC704700BFDD
:10E4AC000EB46FF0004110B500249DB01FAB02906C
:10E4BC000690079104910948094953F8042B0591DA
:10E4CC00006802A901931B9400F092F9029B1C7046
:10E4DC001DB0BDE8104003B0704700BF8C01002098
:10E4EC000802FFFF03460244934200D1704703F831
:10E4FC00011BF9E7014B1868704700BF8C01002025
:10E50C0070B500260C4D0D4C641BA410A64209D10D
:10E51C0000F076FC00260A4D0A4C641BA410A6429F
:10E52C0005D170BD55F8043B98470136EEE755F818
:10E53C00043B98470136F2E718F6000818F6000875
:10E54C0018F600081CF600087047704738B50546E9
:10E55C00002940D051F8043C0C1F002BB8BFE41824
:10E56C0000F0DEF81C4A136833B963601460284667
:10E57C00BDE8384000F0DAB8A34208D92068211869
:10E58C008B4201BF19685B6809182160EDE71A46D8
:10E59C005B680BB1A342FAD911685018A0420BD199
:10E5AC0020680144501883421160E0D118685B6800
:10E5BC00084410605360DAE702D90C232B60D6E7CD
:10E5CC00206821188B4201BF19685B68091821600B
:10E5DC0063605460CBE738BDA018002070B50F4EB7
:10E5EC000C463168054611B900F0A8FB3060214695
:10E5FC00284600F0A3FB431C03D14FF0FF34204608
:10E60C0070BDC41C24F00304A042F8D0211A284683
:10E61C0000F094FB0130F2D1EFE700BF9C18002012
:10E62C002DE9F843CD1C25F0030508350C2D38BF1A
:10E63C000C25002D064601DBA94204D90C233360BE
:10E64C000020BDE8F883DFF8D48000F069F8D8F832
:10E65C0000301C4644BB29463046FFF7BFFF431C25
:10E66C00044658D1D8F800402746002F43D1002C3F
:10E67C004BD023683946304604EB030900F05EFBAF
:10E68C00814542D1216830466D1A2946FFF7A6FF15
:10E69C0001303AD023682B442360D8F800305A68F4
:10E6AC0062BBC8F800700FE02268521B20D40B2A02
:10E6BC0017D96119A342256018BF5960636808BF58
:10E6CC00C8F8001062514B60304600F02FF804F18E
:10E6DC000B00231D20F00700C21A1CBF1B1AA350ED
:10E6EC00AFE76268A3420CBFC8F800205A60EBE7A2
:10E6FC0023466468AEE73C467F68B6E71A465B681B
:10E70C00A342FBD100235360DEE70C233046336079
:10E71C0000F00CF894E70560D6E700BFA0180020C5
:10E72C000148FFF711BF00BF981800200148FFF700
:10E73C000CBF00BF981800202DE9F0471F468E68CB
:10E74C008246BE420C4690460B682DD8B1F90C207F
:10E75C0012F4906F26D06569096905EB4505A3EBAA
:10E76C00010905EBD5757B1C4B446D109D4238BFE0
:10E77C001D46530527D52946FFF752FF064660B3C1
:10E78C004A46216900F0F8FAA38923F4906343F018
:10E79C008003A38126614E4426603E466561A5EB4D
:10E7AC000905A560BE4200D93E4632464146206866
:10E7BC0000F0AAFA0020A3689B1BA36023683344D3
:10E7CC002360BDE8F0872A4600F0E4FA06460028EC
:10E7DC00E0D150462169FFF7B9FE0C23CAF800308E
:10E7EC00A3894FF0FF3043F04003A381E9E7000019
:10E7FC002DE9F04F98468B8907461B060D461446AB
:10E80C009DB010D50B6973B94021FFF709FF286043
:10E81C00286130B90C233B604FF0FF301DB0BDE8D0
:10E82C00F08F40236B610023099320238DF829304E
:10E83C0030234FF00109CDF80C80DFF898818DF86A
:10E84C002A3023469A4613F8012B0AB1252AF9D10E
:10E85C00BAEB040B0BD05B46224629463846FFF731
:10E86C006BFF013000F0A780099A5A4409929AF87C
:10E87C000030002B00F09F8000234FF0FF32CDE9D9
:10E88C0005230AF1010A049307938DF853301A9368
:10E89C005446052214F8011B4E4800F05FFA049A06
:10E8AC00D8B9D00644BF20238DF85330110744BF8C
:10E8BC002B238DF853309AF800302A2B15D0544660
:10E8CC0000204FF00A0C079A214611F8013B303B0F
:10E8DC00092B4BD9B0B1079214E0A0EB080309FA4D
:10E8EC0003F31343A2460493D2E7039B191D1B6841
:10E8FC000391002BBBBF5B4242F0020207930793CC
:10E90C00B8BF049223782E2B0AD163782A2B32D1EC
:10E91C00039B02341A1D1B68039243EAE3730593AD
:10E92C00DFF8B4A003225046217800F017FA38B172
:10E93C004022049BA0EB0A00824013430134049351
:10E94C0014F8011B062225488DF8281000F006FA51
:10E95C00002836D0224B1BBB039B073323F0070345
:10E96C0008330393099B334409936AE70C4601204F
:10E97C000CFB0232A8E700234FF00A0C19460134B5
:10E98C000593204610F8012B303A092A03D9002BA5
:10E99C00C6D00591C4E7044601230CFB0121F0E726
:10E9AC0003AB00932A4638460E4B04A9AFF3008004
:10E9BC00421C0646D6D1AB895B063FF52DAF0998B4
:10E9CC002CE703AB00932A463846064B04A900F00B
:10E9DC007DF8EDE7DAF50008E0F50008E4F500084D
:10E9EC000000000045E700082DE9F0471646984660
:10E9FC008A680B6907469342B8BF1346336091F897
:10EA0C0043200C46DDF820900AB1013333602368B3
:10EA1C00990642BF336802333360256815F006054A
:10EA2C0006D104F1190AE36832689B1AAB422BDC5D
:10EA3C0094F843302268003B18BF0123920630D46F
:10EA4C004146384604F14302C847013023D02368BD
:10EA5C00226903F00603042B14BF002533684FF022
:10EA6C00000608BFE56804F11A0408BFED1A54F853
:10EA7C00123C08BF25EAE5759342C4BF9B1AED18FA
:10EA8C00B5421AD1002008E00123524641463846CF
:10EA9C00C847013003D14FF0FF30BDE8F087013596
:10EAAC00C1E73020E11881F843005A1C94F8451056
:10EABC002244023382F84310C2E701232246414626
:10EACC003846C8470130E6D00136D9E72DE9FF4773
:10EADC000F7E9146782F80460C469A460C9E01F18B
:10EAEC00430207D8622F0AD8002F00F0D180582F8C
:10EAFC0000F0B88004F1420684F842703AE0A7F1C5
:10EB0C006303152BF6D801A151F823F071EB000823
:10EB1C0085EB000801EB000801EB000801EB000895
:10EB2C0001EB000885EB000801EB000801EB000885
:10EB3C0001EB000801EB000883EC0008AFEB0008C8
:10EB4C003DEC000801EB000801EB0008A5EC000807
:10EB5C0001EB0008AFEB000801EB000801EB00082B
:10EB6C0045EC000833681A1D1B68326004F142063C
:10EB7C0084F8423001239CE033682068191D316011
:10EB8C00060601D51D6803E04506FBD5B3F9005018
:10EB9C00002D03DA2D236D4284F843300A235848A4
:10EBAC0011E021683368080653F8045B02D4490667
:10EBBC0048BFADB26F2F336014BF0A2308235048EF
:10EBCC00002184F843106668002EA66005DB2168DE
:10EBDC002E4321F0040121604BD01646B5FBF3F116
:10EBEC0003FB1157C75D06F8017D2F46BB420D464E
:10EBFC00F4D9082B0BD12368DF0708D5236961688A
:10EC0C009942DEBF302306F8013C06F1FF36921B19
:10EC1C0022614B4621464046CDF800A003AAFFF7DF
:10EC2C00E3FE01304AD14FF0FF3004B0BDE8F0876D
:10EC3C00236843F0200323607827324884F845701A
:10EC4C00236831681F0651F8045B02D45F0648BF85
:10EC5C00ADB23160D90744BF43F0200323601DB12E
:10EC6C001023ADE72648E9E7236823F0200323604F
:10EC7C00F6E71646BDE733682568181D61693060F4
:10EC8C002E061B6801D5196002E06806FBD51980B9
:10EC9C00002316462361BCE7336800211A1D32603D
:10ECAC001E686268304600F059F808B1801B60603D
:10ECBC0063682361002384F84330AAE7324649464F
:10ECCC0040462369D0470130ADD023689B0713D44D
:10ECDC00E068039B9842B8BF1846A6E7012332466A
:10ECEC0049464046D04701309DD00135E368039931
:10ECFC005B1AAB42F2DCEBE7002504F11906F5E7F1
:10ED0C00EBF50008FCF50008884210B501EB020495
:10ED1C0002D98442234607D8431EA14208D011F8D9
:10ED2C00012B03F8012FF8E7014602448A4200D177
:10ED3C0010BD13F8014D02F8014DF7E738B500236B
:10ED4C00054D044608462B60F6F78EF9431C02D19C
:10ED5C002B6803B1236038BD94180020034610B50E
:10ED6C00C9B202449342184601D1002003E0047852
:10ED7C0001338C42F6D110BD0A44914200F1FF33AD
:10ED8C0000D1704710B511F8014B914203F8014FB7
:10ED9C00F9D110BD2DE9F041074614460D4621B9B5
:10EDAC001146BDE8F041FFF73BBC2AB9FFF7CEFB9B
:10EDBC0025462846BDE8F08100F01AF88442064644
:10EDCC0002D8B4EB500FF4D821463846FFF728FC94
:10EDDC00804608B94546ECE7B4422246294628BF8E
:10EDEC003246FFF7C9FF29463846FFF7AFFBF1E77C
:10EDFC0051F8043C181F002BBCBF0B58C0187047AF
:10EE0C00F8B500BFF8BC08BC9E467047F8B500BF0B
:08EE1C00F8BC08BC9E467047DB
:10EE2400696E666F0A0000000A70776D20256425FC
:10EE34006425642564256425642564256400000034
:10EE44000A3078256C78203078256C782030782545
:10EE54006C78203078256C78203078256C782030D8
:10EE640078256C78203078256C78203078256C787B
:10EE7400000000000A503D30782578206368343D56
:10EE840025303564206368353D253035642063685A
:10EE9400363D25303564206368373D2530356420A0
:10EEA4006368383D25303564000000000A737443FC
:10EEB40069636C6F3D2530356420737450756C73D1
:10EEC400616E74693D253035640000000A494430A0
:10EED40030303030300000000A62307C31000000F5
:10EEE4000A3F6D6E73767676767620733D667C6225
:10EEF400000000000A3F6D6E7376767676762030D9
:10EF0400303030303E3D76767676763C3D39393950
:10EF1400393900000A3F6D6E737676767676203145
:10EF24003E3D6D3C3D3400000A3F6D6E737676764F
:10EF3400767600000A6565203078253032783D30D9
:10EF440078253034780000000A65652072656164B4
:10EF5400206572726F722025640000000A3F65729A
:10EF64006161206865782076616C756573000000C6
:10EF74000A3F6572616100000A646F6E6520307833
:10EF8400253032783D307825303478000A656520A4
:10EF94007772697465206572726F7220256400004F
:10EFA4000A3F6577616176767676206865782076A3
:10EFB400616C7565730000000A3F657761612068C4
:10EFC40065782076616C7565730000000A3F65778B
:10EFD40061617676767600000A3078253032783DA5
:10EFE4002535642000000000726465727220256477
:10EFF400200000000A0000000A3F656400000000D1
:10F004000A3F6578000000000A6D3170776D617009
:10F014003D2564206D3170776D63683D2564206DF6
:10F024003270776D61703D2564206D3270776D6349
:10F03400683D2564206D3370776D61703D256420D3
:10F044006D3370776D63683D2564206D3470776D22
:10F0540061703D2564206D3470776D63683D25646F
:10F06400000000000A6D3154696D656F75744D615F
:10F074006E3D2564206D3254696D656F75744D6104
:10F084006E3D2564206D3354696D656F75744D61F3
:10F094006E3D2564206D3454696D656F75744D61E2
:10F0A4006E3D2564200000000A7472616D703D2578
:10F0B40064207472616D706D616E3D2564000000A2
:10F0C4000A6D3170776D4D616E3D2564206D32702F
:10F0D400776D4D616E3D2564206D3370776D4D61A4
:10F0E4006E3D2564206D3470776D4D616E3D2564F1
:10F0F400000000000A61704D3173746172743D2523
:10F10400642061704D3173746F703D2564206368B1
:10F114004D3173746172743D25642063684D31739D
:10F12400746F703D256400000A61704D3273746120
:10F1340072743D25642061704D3273746F703D2587
:10F14400642063684D3273746172743D2564206376
:10F15400684D3273746F703D256400000A61704D10
:10F164003373746172743D25642061704D3373741C
:10F174006F703D25642063684D3373746172743D10
:10F1840025642063684D3373746F703D25640000FB
:10F194000A61704D3473746172743D25642061702A
:10F1A4004D3473746F703D25642063684D347374FB
:10F1B4006172743D25642063684D3473746F703DCF
:10F1C400256400000A3F6576000000000A3F65726E
:10F1D4007C777C647C787C76000000000A3F657252
:10F1E4006161207C20657761617676767600000027
:10F1F4000A3F00000A70756C73616E74693D25588E
:10F20400000000000A737470756C73616E74693D5C
:10F21400255800000A73744369636C6F3D256400CC
:10F224000A646F6E652025643D2564000A656520C7
:10F234007772697465206572726F722025640000AC
:10F244004C6F616445450A000A6D3170776D6170D9
:10F254003D2564206D3170776D63683D2564206DB4
:10F264003270776D61703D2564206D3270776D6307
:10F27400683D2564206D3370776D61703D25642091
:10F284006D3370776D63683D2564206D3470776DE0
:10F2940061703D2564206D3470776D63683D25642D
:10F2A400000000000A6D3154696D656F75744D611D
:10F2B4006E3D2564206D3254696D656F75744D61C2
:10F2C4006E3D2564206D3354696D656F75744D61B1
:10F2D4006E3D2564206D3454696D656F75744D61A0
:10F2E4006E3D2564200000000A7472616D703D2536
:10F2F40064207472616D706D616E3D256400000060
:10F304000A6D3170776D4D616E3D2564206D3270EC
:10F31400776D4D616E3D2564206D3370776D4D6161
:10F324006E3D2564206D3470776D4D616E3D2564AE
:10F33400000000000A61704D3173746172743D25E0
:10F34400642061704D3173746F703D25642063686F
:10F354004D3173746172743D25642063684D31735B
:10F36400746F703D256400000A61704D32737461DE
:10F3740072743D25642061704D3273746F703D2545
:10F38400642063684D3273746172743D2564206334
:10F39400684D3273746F703D256400000A61704DCE
:10F3A4003373746172743D25642061704D337374DA
:10F3B4006F703D25642063684D3373746172743DCE
:10F3C40025642063684D3373746F703D25640000B9
:10F3D4000A61704D3473746172743D2564206170E8
:10F3E4004D3473746F703D25642063684D347374B9
:10F3F4006172743D25642063684D3473746F703D8D
:10F40400256400000A6D3161703D25640000000030
:10F414000A6D3261703D2564000000000A6D33619D
:10F42400703D2564000000000A6D3461703D256460
:10F43400000000000A6D3163683D2564000000008F
:10F444000A6D3263683D2564000000000A6D336371
:10F45400683D2564000000000A6D3463683D25643E
:10F464000000000053544D333220566972747561A4
:10F474006C20436F6D506F727400000053544D69DB
:10F4840063726F656C656374726F6E696373000099
:10F4940043444320436F6E6669670000434443203E
:10F4A400496E7465726661636500000028003C0063
:10F4B40046004600230028002800280014001400F9
:10F4C40014001400E600640082002C0101001B00FB
:10F4D4000A001E000100010000000000F4011400F5
:10F4E4003C0046002800280032000A003601C20110
:10F4F4001E0036015401AE011E00AE010A00400197
:10F504008C00B801140018012800B80101001B0088
:10F514000A001E0001000100000000000000640059
:10F524003C004600280028003200050001000200CB
:10F5340003000400050006000700080009000A0093
:10F544000B000C000D000E000F0010001100120043
:10F5540013001400150016001700180019001A00F3
:10F564001B001C001D001E001F00200021002200A3
:10F5740023002400250026002700280029002A0053
:10F584002B002C002D002E002F0030003100320003
:10F5940033003400350036003700380039003A00B3
:10F5A4003B003C003D003E003F00400000000000E6
:10F5B400000000000102030406070809000000001F
:10F5C4000102030402030405060708090A0B0C0DD3
:10F5D4000E0F10100102232D302B2000686C4C00FC
:10F5E400656667454647003031323334353637383F
:10F5F400394142434445460030313233343536379D
:0CF6040038396162636465660000000034
:08F610003C0BFF7F010000002C
:04F6180031010008B4
:04F61C000D010008D4
:10F6200000F80008C8C864040404040404040400C6
:10F6300000127A0010000000010000000A0600021B
:10F640000000004001000000A1C3000895C40008AC
:10F6500003C500080000000045C7000849C60008AF
:10F66000EFC60008000000000000000000000000DD
:10F67000B5C7000895C70008D5C70008F5C700083A
:10F6800009024300020100C0320904000001020225
:10F6900001000524001001052401000104240202D8
:10F6A0000524060001070582030800100904010073
:10F6B000020A00000007050102000200070581029E
:10F6C0000002000009024300020100C032090400E8
:10F6D00000010202010005240010010524010001BF
:10F6E0000424020205240600010705820308001015
:10F6F00009040100020A00000007050102400000A1
:10F70000070581024000000009074300020104C010
:10F710003209040000010202010005240010010565
:10F7200024010001042402020524060001070582C9
:10F730000308001009040100020A00000007050187
:10F74000024000000705810240000000C1DB000804
:10F75000E9DB0008F9DB0008B5DC00083DDD000846
:10F7600061DD0008C1DD000885DD0008E9DD000875
:10F770000DDE000849DE000812010002020200400E
:10F78000830440570002010203010000040309043E
:10F790001A0300000000000000000000000000004C
:10F7A00000000000000000000000000090010020A8
:10F7B000000000005C170020C41700202C18002057
:10F7C0000000000000000000000000000000000039
:10F7D0000000000000000000000000000000000029
:10F7E0000000000000000000000000000000000019
:0CF7F0000000000000000000000000000D
:04000005080050EDB2
:00000001FF
